:100000000C94A40A0C94D50A0C94D50A0C94D50A25
:100010000C94D50A0C94D50A0C94D50A0C94D50AE4
:100020000C94D50A0C94D50A0C94D50A0C94D50AD4
:100030000C94D50A0C944E570C94D50A0C94D50AFE
:100040000C94D50A0C94D50A0C94D50A0C94D50AB4
:100050000C94D50A0C94D50A0C94D50A0C94C69924
:100060000C94D50A0C94614E0C94384E0C94D50A1D
:100070000C94D50A0C94D50A0C94D50A0C94D50A84
:100080000C94D50A0C94D50A0C94D50A0C94D50A74
:100090000C940E4E0C94E54D0C94D50A0C946258B9
:1000A0000C94D50A0C94D50A0C94D50A0C94D50A54
:1000B0000C94D50A0C94D50A0C94D50A0C94D50A44
:1000C0000C94D50A0C94D50A0C94D50A0C94BB4D0B
:1000D0000C94924D0C94D50A0C94684D0C943F4DA1
:1000E0000C94D50AF21BD91C411C3A1C0A1CFA1BA1
:1000F000D91CF61BD91CD91CD91CD91CD91C610BC5
:10010000CA0B520C8F0D970D710F25104311E5127C
:10011000E11337144C145014D91C92149614011680
:10012000BC17D617FD1860193F1ABF1AC61AB31BA1
:10013000BD3F5640684071407A40834095409E40A4
:10014000CD40DF40E840F140FA4095419E41A74153
:1001500048844B843A843E84448482844F8453840C
:1001600059845D84618467846B846F848284758420
:1001700079847D84084AD73B3BCE016E84BCBFFDA9
:10018000C12F3D6C74319ABD56833DDA3D00C77F67
:1001900011BED9E4BB4C3E916BAAAABE0000008000
:1001A0003F07634236B79BD8A71A39685618AEBACC
:1001B000AB558C1D3CB7CC5763BD6DEDFD753EF660
:1001C000177231BF000000803F08000000BE92247B
:1001D00049123EABAAAA2ABECDCCCC4C3E000000B0
:1001E00080BEABAAAAAA3E00000000BF00000080AB
:1001F0003F0000000000084178D3BB4387D1133D86
:10020000190E3CC3BD4282AD2B3E68EC8276BED94E
:100210008FE1A93E4C80EFFFBE01C4FF7F3F00008D
:10022000000000004E414E494E495459494E46CDBA
:10023000CCCC3D0AD7233C17B7D13877CC2B32959D
:1002400095E6241FB14F0A000020410000C842007B
:10025000401C4620BCBE4CCA1B0E5AAEC59D740045
:10026000407A10F35A00A0724E18090010A5D4E885
:100270000000E87648170000E40B54020000CA9A18
:100280003B000000E1F5050000809698000000406A
:10029000420F000000A086010000001027000000AF
:1002A00000E803000000006400000000000A0000F5
:1002B0000000000100000000002C76D888DC674FA9
:1002C0000823DFC1DFAE59E1B1B796E5E3E453C6D9
:1002D0003AE651997696E8E6C28426EB898C9B62D1
:1002E000ED407C6FFCEFBC9C9F40F2BAA56FA5F47B
:1002F00090055A2AF75C936B6CF9676DC11BFCE0A3
:10030000E40D47FEF520E6B500D0ED902E030094F5
:100310003577050080841E080000204E0A0000008A
:10032000C80C333333330F986E12831141EF8D2194
:1003300014893BE65516CFFEE6DB18D1844B381BFB
:10034000F77C1D901DA4BBE424203284725E2281C0
:1003500000C9F124ECA1E53D274D6F74696F6E0073
:10036000555620496E742E00555620496E74656EA0
:1003700073697479004F3220436F6E6300434F32CC
:1003800020436F6E630053656E736F7220657272E7
:100390006F722100234E6F2073656E736F722100A0
:1003A000434F3220436F6E63004D65617375726910
:1003B0006E6700234E6F2073656E736F7220666FD9
:1003C0007220504D21004E6F2073656E736F722145
:1003D00000206E672F4C00504D313A322E353A31A5
:1003E00030004D6561737572696E672E2E00234E65
:1003F0006F2054422073656E736F723F00234E6FFF
:100400002073656E736F722100536F756E64204C9C
:100410006576656C004D6561737572696E672E2E29
:1004200000234E6F2073656E736F722100536F75DA
:100430006E64204C6576656C00234E6F2073656E8C
:10044000736F7220666F722074656D70202620684D
:10045000756D696469747921004E6F2053656E7300
:100460006F72210020666F722074656D70202620E7
:1004700068756D696469747921002353656E736FC3
:1004800072204572726F72200053656E736F722016
:100490004572726F7221002357726F6E6720736509
:1004A0006E736F7220666F722074656D70202620E7
:1004B00068756D6964697479210057726F6E672081
:1004C00053656E736F72210054656D702048756DB1
:1004D0006964697479004C6967687420496E746551
:1004E0006E7369747900466C616D652049520048ED
:1004F0002D6669656C6400536561726368204469A8
:1005000072656374696F6E00234E6F2070482073AC
:10051000656E736F72210070482076616C7565009E
:1005200023496E76616C6964206B65792100204DEA
:10053000756C746973656E736F7273004D756C744E
:100540006973656E736F72730044697361626C6581
:1005500000456E61626C65005265626F6F74696E12
:10056000672E2E2E002344413A2D3233002372652C
:10057000706C6965733D002353657474696E6773AD
:10058000206F6620616C6C2073656E736F72733AB6
:10059000002353697A65206F66206865616465721F
:1005A000202B20616C6C2073656E736F72733A2020
:1005B000002353697A65206F6620686561646572FF
:1005C0003A20002320616E64207265616479207492
:1005D0006F207573652100206D6F62696C65206CFA
:1005E0006F6767657220737461727465642000437D
:1005F000616C6962726174696F6E205072657373A9
:100600007572653D00536561206C6576656C2050A0
:100610002863616C63293D00234572726F723A70E2
:100620007265737375726520424D503038352C20D9
:10063000636865636B20776972696E672100495250
:100640002054656D702073656E736F7220666F75D0
:100650006E6400504D322E352073656E736F7220BC
:100660006C696B656C7920666F756E6400206D6FC8
:1006700062696C65206C6F67676572207374617264
:10068000746564202E2E2E2000576946692049503B
:100690003A002357694669204950206164647265B5
:1006A00073733A2000456455484B205345534C6FB3
:1006B000676765720053656E736F7220736C6F7439
:1006C00020616E6420747970653A0057656C636FC1
:1006D0006D6520746F20456455484B0023456E645A
:1006E000206F66204D756C746973656E736F722030
:1006F0004379636C6523002354696D6520647572CA
:100700006174696F6E3D002354696D6520696E7474
:10071000657276616C3D00576946692049503A0020
:10072000234D5320456E61626C656400234D532058
:1007300044697361626C6564002352657374207050
:100740006172616D657465727320746F2064656693
:1007500061756C742076616C756573004C6F6767AA
:100760006572204E616D653A200067657453656C53
:10077000665465737442697428293A200069734984
:100780006E74657272757074456E61626C65642812
:1007900031293A2000676574496E7465727275700C
:1007A000744D617070696E672831293A2000676561
:1007B00074496E74657272757074536F7572636587
:1007C0002831293A2000676574496E746572727524
:1007D0007074536F7572636528293A2000676574D9
:1007E0005261746528293A20332E31343135393F2E
:1007F00000616363656C2E69734C6F77506F77652A
:100800007228293A2000616363656C2E6973417315
:100810006C65657028293A2000616363656C2E69F8
:1008200073546170536F757263654F6E5A28293A1D
:100830002000616363656C2E6973546170536F753A
:100840007263654F6E5928293A2000616363656CB5
:100850002E6973546170536F757263654F6E5828BB
:10086000293A2000616363656C2E69734163746982
:1008700076697479536F757263654F6E5A28293A99
:100880002000616363656C2E6973416374697669E6
:100890007479536F757263654F6E5928293A200039
:1008A00069734163746976697479536F75726365AE
:1008B0004F6E5828293A200069735461704465745A
:1008C000656374696F6E4F6E5A28293B2066616CB0
:1008D00073653F2000697354617044657465637487
:1008E000696F6E4F6E5A28293B20747275653F20E0
:1008F000006973546170446574656374696F6E4F09
:100900006E5928293B2066616C73653F200069732E
:10091000546170446574656374696F6E4F6E5928D5
:10092000293B20747275653F2000697354617044DF
:100930006574656374696F6E4F6E5828293B206635
:10094000616C73653F200069735461704465746520
:100950006374696F6E4F6E5828293B2074727565F9
:100960003F200067657453757070726573734269D8
:100970007428293B2066616C73653F2000676574AD
:10098000537570707265737342697428293B2074C3
:100990007275653F20006973416374697669747983
:1009A000416328293A20006973496E61637469764E
:1009B0006974795A456E61626C656428293A200031
:1009C0006973496E616374697669747959456E61BA
:1009D000626C656428293A20006973496E6163740A
:1009E000697669747958456E61626C656428293A44
:1009F0002000697341637469766974795A456E6140
:100A0000626C656428293A200069734163746976D1
:100A100069747959456E61626C656428293A2000D1
:100A20006973416374697669747958456E61626C63
:100A3000656428293A2000676574467265654661D9
:100A40006C6C4475726174696F6E28293A20006776
:100A500065744672656546616C6C5468726573684E
:100A60006F6C6428293A200067657454696D654984
:100A70006E616374697669747928293A2000676524
:100A800074496E61637469766974795468726573C8
:100A9000686F6C6428292000676574416374697607
:100AA0006974795468726573686F6C6428292000D2
:100AB000676574446F75626C6554617057696E64E4
:100AC0006F7728292000676574446F75626C6554E0
:100AD00061704C6174656E637928293A20006765FE
:100AE000745461704475726174696F6E28293A207C
:100AF00000676574417869734F666673657428266C
:100B0000782C2026792C20267A293A2000676574D3
:100B10005461705468726573686F6C6428293A2058
:100B20000058595A2047733A200058595A20434FC9
:100B3000554E54533A2000736574206761696E7393
:100B40005B5D3A006761696E735F6F7269675B5DD9
:100B50003A00696E7075742044535463616C696225
:100B6000726174653A0020766F6C746167653D0050
:100B70002354757262696469747920557070657266
:100B8000204C696D69743A200020766F6C7461673F
:100B9000653D0023547572626964697479204C6FF5
:100BA000776572204C696D69743A20002354757220
:100BB000626964697479204C6F776572204C696D45
:100BC00069742056696E663A20004D617820726122
:100BD0006E67653D0023566F6C74616765207365B1
:100BE0006E736F723A00342D32306D4100414353C1
:100BF000373132204D61783D004143533731322047
:100C00004D61783D3541002343757272656E7420E5
:100C100073656E736F723A00234453205468657293
:100C20006D6F6D657465722063616C696272617469
:100C3000656420666F72202300234E6F206E656509
:100C40006420746F2063616C6962726174652063F3
:100C5000757272656E742073656E736F72210023F6
:100C60004143533731322063757272656E7420735D
:100C7000656E736F72206F666673657420563D00F3
:100C8000235556207A65726F20766F6C74616765A4
:100C9000203D00234F3220766F6C253D00234F32DC
:100CA0002063616C6962726174696F6E3A2000231F
:100CB000566F6C746167652870483D3130293A0081
:100CC00023566F6C746167652870483D34293A007B
:100CD000232D2D2D2D2D2D2D2D2D2D2D2D2D2D2D4E
:100CE0002D2D2D2D2D2D2D2D2D2D2D2D2D2D2D2D34
:100CF0002D2D2D2D2D00235265736F6C7574696F2A
:100D00006E3A20202000234D696E2056616C756577
:100D10003A2020202000234D61782056616C7565B3
:100D20003A202020200023556E69717565204944C2
:100D30003A2020202000234472697665722056658F
:100D4000723A202020002353656E736F723A202080
:100D5000202020202000232D2D2D2D204D61676E79
:100D6000657469632053656E736F72202D2D2D2D70
:100D70002D2D2D2D2D2D2D2D2D2D2D2D2D2D2D2DA3
:100D800000482D6669656C643A20280020202020E8
:100D90002020202020202020202020002020202073
:100DA000202020202020202020202000233A5368CB
:100DB0006F772F48696465204C4344002A3A546891
:100DC00069732048656C700044233A43616C696222
:100DD000726174696F6E00442A3A53657474696E67
:100DE00067730044423A5265736574204C6F6767BD
:100DF00065720044433A436C656172204C43440081
:100E000044443A4D756C746953656E736F72730028
:100E100044393A43757272656E7400566F6C746132
:100E200067652B43757272656E740044383A456C81
:100E30006563747269630044373A4D6F74696F6E0D
:100E40000044363A44532054656D700044353A5599
:100E50005620496E74656E736974790044343A4F54
:100E60003220636F6E632E0044333A434F32206367
:100E70006F6E632E0044323A504D28313A322E358F
:100E80003A3130290044323A504D28313A322E3529
:100E90003A3130292A0044313A54757262696469E2
:100EA00074790044303A566F6C7461676500393A62
:100EB0006F7220334420616363656C2E00393A49B8
:100EC0006E636C2E20616E672E00383A7048207673
:100ED000616C756500373A49522054656D70003772
:100EE0003A49522054656D702A00363A4D61676E5A
:100EF00065746963206669656C6400353A4761739F
:100F0000204C6576656C00343A495220466C616D20
:100F10006500333A4C6967687420496E742E00325C
:100F20003A616E642048656967687400323A5465B6
:100F30006D7020507265737375726500313A546537
:100F40006D702048756D696469747900303A536F2B
:100F5000756E64204C6576656C00303A536F756E23
:100F600064204C6576656C2A0054696D65206C615F
:100F70007073653A00576946692049503A00005E2F
:100F8000BCE2613FDD83C29C7E20A3FD1F41009D2A
:100F900023BE46DB65F88C11AF32CA57E974697419
:100FA00065726174696F6E3D0073656E736F722355
:100FB0003D0043757272656E74207374617475734D
:100FC0003A206379636C653D006E6379636C653DBF
:100FD000006E73656E736F72733D006D61786E7332
:100FE000656E736F72733D00656E61626C65643D22
:100FF00000234D756C746973656E736F7273206D29
:101000006561737572656D656E742073657474695E
:101010006E67733A0046696E64696E672057694669
:1010200069204950007365703D006976616C3D0030
:101030006E697465723D00230043616C2E20466129
:10104000696C65640043616C2E20446F6E65004ED0
:101050006F206E6565642100496E76616C6964205D
:101060005028506129005365614C6576656C2050AD
:10107000285061293A0043616C696272617465208D
:1010800050004453542054656D702073656E736F27
:10109000720043757272656E742073656E736F7241
:1010A000004F322073656E736F7200555620736562
:1010B0006E736F720043616C6962726174650046A1
:1010C00061696C65640054422063616C2E20646F1A
:1010D0006E65005570706572204C696D69743A3E9A
:1010E000004C6F776572204C696D69743A3E00540C
:1010F0007572626964697479004661696C6564003F
:1011000070482063616C2E20646F6E6500704831FA
:101110003020507265737320420070483420507242
:1011200065737320410043616C696272617465008C
:10113000416E676C65732F003E6128782C792C7A9C
:10114000292F673A004E6F2073656E736F7221000E
:1011500049522054656D7065726174757265004DF9
:101160006561737572696E672E2E004E6F20736510
:101170006E736F723F0049522054656D70657261E5
:1011800074757265004D6561737572696E672E2E98
:10119000004F6666206169722D636F6E642100499D
:1011A00074277320746F6F20636F6F6C2100546518
:1011B0006D702069732066696E6521004973206136
:1011C00069722D636F6E64206F6E3F0049742773E0
:1011D00020717569746520686F74210049742773E4
:1011E000207665727920686F742120004F66662032
:1011F0006169722D636F6E642100497427732074D6
:101200006F6F20636F6F6C210054656D7020697380
:101210002066696E6521004973206169722D636FD4
:101220006E64206F6E3F0049742773207175697476
:101230006520686F74210049742773207665727980
:1012400020686F74210054656D702048756D696465
:10125000697479004E6F2053656E736F7221004E72
:101260006F20445320546865726D6F6D65746572AC
:101270002100445320546865726D2E004D6F7469CF
:101280006F6E00556E6B6E6F776E00496E6475738E
:10129000747269616C20342D32306D4100414353CA
:1012A000373132204D61783D3541002343757272EC
:1012B000656E742073656E736F723A0000002100D2
:1012C000240027002A002D00300033000101000017
:1012D000040107010A0100002200250028002B005C
:1012E0002E003100340002010000050108010B014D
:1012F000000020002300260029002C002F003200CF
:1013000000010000030106010901050505050705A7
:1013100008080808020202020A0A08080404040471
:10132000010101010101010103030303030303039D
:10133000040707070C0C0C0C0C0C0C0C020202022C
:1013400006060606060606060B0B0B0B0B0B0B0B15
:1013500001021020200808102040102040800201C7
:1013600002010804020101020408102040808040AC
:1013700020100804020180040201804020100804AB
:101380000201080402010102040810204080010249
:1013900004081020408000000A0B02090C0D0E0802
:1013A000070304010000000000000000000000002E
:1013B000000000000000000000000000000000002D
:1013C00000001211100000000000000000000000EA
:1013D000000000000000000000000000496E76617F
:1013E0006C6964206B65792100202020202020205A
:1013F000202020202020202020002020202020200D
:1014000020202020202020202020002020202020FC
:1014100020202020202020202020200020202020EC
:10142000202020202020202020202020004E455455
:101430003D426C7565746F6F7468204C45004E4575
:10144000543D426C7565746F6F7468004E45543D31
:10145000576946690053657474696E67204661690F
:101460006C65640053657474696E6720446F6E65C3
:10147000004368616E6765204E6574776F726B3EDE
:1014800000547970653A0042542F57694669204EDE
:101490006574776F726B004368616E676520536592
:1014A0006E736F723E0043757272656E7420536581
:1014B0006E736F72004F7468657200496E642E20FF
:1014C000342D32306D4100414353373132203C33AB
:1014D000304100414353373132203C3230410041EA
:1014E0004353373132203C3541003E4D6178205620
:1014F0006F6C743A3E004368616E676520766F6C6E
:10150000746167653E00547970652000566F6C7495
:101510006167652053656E736F72004368616E6723
:1015200065207479706520746F0053656E736F72F7
:101530003D4448540054656D702048756D69646978
:101540007479000035A705A711241FBECFEFD1E2A3
:10155000DEBFCDBF00E00CBF1BE0A0E0B2E0E4EADC
:10156000FCE601E00BBF02C007900D92AA3EB10756
:10157000D9F723E1AAEEBBE001C01D92AF39B20753
:10158000E1F71AE0C3EADAE000E006C021970109BA
:10159000802FFE010E9478B3C23AD10780E008078D
:1015A000A9F70E94559A0C9441B60C9400002F9212
:1015B0003F924F925F926F927F928F929F92AF92E3
:1015C000BF92CF92DF92EF92FF920F931F93CF9330
:1015D000DF93CDB7DEB7C554D1090FB6F894DEBF9F
:1015E0000FBECDBF8C01E090070CF090080C8091ED
:1015F0009713882349F06DE675E08EE09FE00E9426
:10160000734CC8010E942A51680125E0C20ED11C0A
:1016100035E0C316D10420F18091070C9091080C9D
:101620000817190729F10E948D3E0E94FB750C3E98
:101630004FEF140724F01093080C0093070CB80127
:10164000CE0101960E942D50BE016F5F7F4F8AE24E
:1016500092E10E94C04ACE0101960E94A34B08C0AD
:101660000E3F5FEF150721F40E940B760C94CD1D01
:101670006FEB79E08EE192E10E94794BF5E0CF16B5
:10168000D10490F068ED7BE0CE0101960E94074CFA
:101690004AE050E06FEF7FEFCE0101960E94699023
:1016A000CE0101960E94A34BF8017C96E632F1052B
:1016B00010F00C94D91C8827EE58FF4F8F4F0C94D4
:1016C00078B30E948D3E89E390E00E94D67020E0BE
:1016D00030E04AE754E40E9413AFAB01BC0121E0C3
:1016E000CE0101960E94A84B60E178E0CE01809681
:1016F0000E94074CBE016F5F7F4FCE0180960E9413
:10170000234B61EC75E00E940C4BBC018EE192E131
:101710000E948E4BCE0180960E94A34BCE01019673
:101720000E94A34B65EC75E088E192E10E94794B41
:1017300068E172E1CE0101960E94FF4B4AE050E061
:1017400068E070E0CE0101960E94C48FCE01019640
:101750000E94A34B6EE172E1CE0101960E94FF4B05
:101760004AE050E06FEF7FEFCE0101960E947C8D42
:10177000CE0101960E94A34B68E172E18EE192E1F5
:101780000E94BA4A8091430C882311F40C940B1DDB
:101790000C945117C090B702D090B8020E948D3EB1
:1017A00089E390E00E94D67020E030E04AE754E4FC
:1017B0000E9413AF0E949DB1CE0101960E942D5050
:1017C00060E178E0CE0180960E94074CBE016F5F19
:1017D0007F4FCE0180960E94234B61EC75E00E9402
:1017E0000C4BBC018EE192E10E948E4BCE018096A3
:1017F0000E94A34BCE0101960E94A34B809122121E
:1018000090912312099718F423E0F22E02C092E07F
:10181000F92E8091B5108330E4F4C6010E946478FB
:101820004B015C016091B6107091B710072E000C4F
:10183000880B990B0E94B4AEA50194010E9413AFCE
:1018400020E030EC4FE754E40E9404B1AB01BC014E
:1018500003C040E050E0BA012F2DCE0101960E9456
:10186000A84B6AEF75E0CE0180960E94074CBE013E
:101870006F5F7F4FCE0180960E94234B6DEC75E029
:101880000E940C4BBC018EE192E10E94BA4ACE014B
:1018900080960E94A34BCE0101960E94A34B60ED5F
:1018A00075E042CF8091430C882309F42CC184ED6C
:1018B0009DE00E94168E61E0809102020E94AE853A
:1018C00060E0809100020E94AE850E94A3970E9472
:1018D000915B0E94AE5BAB01BC0123E0CE01809620
:1018E0000E94A84BBE01605E7F4FCE0101960E9410
:1018F000FF4B67EF75E0CE0101960E940C4BBC01D7
:1019000088E192E10E948E4BCE0101960E94A34B8A
:10191000CE0180960E94A34B6BEF79E0CE01019639
:101920000E94074C68E172E1CE0101960E94234BB0
:10193000BC018EE192E10E948E4BCE0101960E9485
:10194000A34B0E94AE5B6B017C010E940F864B0192
:101950005C016EE170E080E090E00E9434860E94BD
:10196000AE5B2B013C010E940F869B01AC01281944
:1019700039094A095B0949015A0131ED831637E0FB
:101980009306A104B1040CF441C0A7019601C30160
:10199000B2010E943DB06B017C0120E030E0A90162
:1019A0000E94F3B118165CF426EA3BE944EC5BE3D1
:1019B000C701B6010E94AEAE87FF0BC027C026EA62
:1019C0003BE944EC5BEBC701B6010E94F3B118168A
:1019D000ECF0C501B40128EE33E040E050E00E9495
:1019E000E0AFCA01B9010E94B4AE4B015C0120E036
:1019F00030E04AE754E4C701B6010E9413AFA501E5
:101A000094010E9404B1AB01BC0103C040E050E06E
:101A1000BA0122E0CE0180960E94A84BBE01605E12
:101A20007F4FCE0101960E94FF4B69ED75E0CE011C
:101A300001960E940C4BBC0182E192E10E948E4B08
:101A4000CE0101960E94A34BCE0180960E94A34B2B
:101A50006DED75E0CE0101960E94074C62E172E1E6
:101A6000CE0101960E94234BBC018EE192E10E94BF
:101A7000BA4ACE0101960E94A34B68ED7BE0CE01ED
:101A800001960E94074C62E172E1CE0101960E942C
:101A9000234BBC0188E192E10E94BA4ACE01019633
:101AA0000E94A34B69E573E0CE0101960E94F74BBB
:101AB0004AE050E060E070E0CE0101960E94C48FE1
:101AC000CE0101960E94A34B68E172E1CE0101961E
:101AD0000E94FF4B45E050E06FEF7FEFCE01019693
:101AE0000E947C8DCE0101960E94A34B61EE75E0B1
:101AF0008EE192E10E94AC4A60E0809102020E9475
:101B0000AE850C940B1D6091550270915602809128
:101B10005702909158020E949C790C940B1D809161
:101B20005B0290915C020E949F7B0C940B1D409184
:101B30005D0226964FAF269760E0842F0E94AE8507
:101B40008091430C811109C08091131181110EC045
:101B50008FE090E0A0E0B0E00DC023E030E040E096
:101B600050E02CAF3DAF4EAF5FAF08C083E090E0D8
:101B7000A0E0B0E08CAF9DAFAEAFBFAF68E673E062
:101B80008EE192E10E94344B6EE172E1CE0101964A
:101B90000E94FF4B4AE050E06FEF7FEFCE010196CD
:101BA0000E94C48FCE0101960E94A34B21961FAEC6
:101BB000219725961FAE2597212C312CC12CD12C95
:101BC000760182E3682E712C812C912C540126968B
:101BD0008FAD26970E94EA85092E000CAA0BBB0B3D
:101BE000880E991EAA1EBB1E65E070E080E090E0A2
:101BF0000E94348691E0691A710849F740902102E9
:101C0000509022026090230270902402C501B4011A
:101C10000E94B4AE20E030E040EA50E40E9413AFEE
:101C200020E030E040E85AE30E9413AF20E030E0CB
:101C300048E452E40E9404B1A30192010E943DB025
:101C400020E030E040E751E40E9413AF4B015C011B
:101C5000A30192016AE979E989E390E40E943DB029
:101C60009B01AC01C501B4010E9404B120E030E049
:101C7000A9010E943EB020E030E040E251E40E9421
:101C800013AF4B015C0121962FAD219725963FADF7
:101C90002597A1010E94F3B118163CF421968FAE4E
:101CA000219725969FAE2597150120E030E0A901E8
:101CB000B401C5010E94AEAE87FF04C0812C912CF7
:101CC000A12CB12C22E0A401B501CE0180960E9486
:101CD000A84BBE01605E7F4FCE0101960E94FF4B74
:101CE00064EF75E0CE0101960E940C4BBC0188E1C7
:101CF00092E10E948E4BCE0101960E94A34BCE0131
:101D000080960E94A34B68E172E1CE0101960E9489
:101D1000FF4B4AE050E060E070E0CE0101960E9487
:101D20007C8DCE0101960E94A34B0E9490878090EB
:101D30008F1390909013A0909113B0909213A4E6FB
:101D40008A0E911CA11CB11C86169706A806B9061E
:101D500010F40C942C1D0E9490870E94B2AE4B018F
:101D60005C0160918F137091901380919113909109
:101D700092130E94B4AE20E030E048EC51E40E949F
:101D80003EB09B01AC01C501B4010E94AEAE87FF1D
:101D900002C00C942C1D6CE370E080E090E00E9487
:101DA0003486BFEFCB1ADB0AEB0AFB0A2CAD3DAD44
:101DB0004EAD5FAD2C153D054E055F050CF001CF16
:101DC00064E670E080E090E00E9434860E948D3EE0
:101DD00064E670E080E090E00E94348660E673E0A4
:101DE00088E192E10E94344B68E172E1CE010196F4
:101DF0000E94FF4B44E150E060E070E0CE010196AC
:101E00000E94C48FCE0101960E94A34B22E021962E
:101E10004FAD219725965FAD2597B101CE018096F4
:101E20000E94A84BBE01605E7F4FCE0101960E94CA
:101E3000FF4B64EF75E0CE0101960E940C4BBC0194
:101E400088E192E10E948E4BCE0101960E94A34B45
:101E5000CE0180960E94A34B68E172E1CE0101960B
:101E60000E94FF4B42E350E06FEF7FEFCE010196FF
:101E70000E947C8DCE0101960E94A34B64E170E02C
:101E800080E090E00E9434860E94B13E6EE170E0F6
:101E900080E090E00E9434866EE170E080E090E0A7
:101EA0000E94348669EF75E0CE0101960E94074CCE
:101EB00068E172E1CE0101960E94234B6DEF75E05F
:101EC0000E940C4B6EE172E10E94234BBC018EE13B
:101ED00092E10E948E4BCE0101960E94A34B0C947E
:101EE0000B1D80915F029091600299270E94647897
:101EF0002DE038E643E55BE30E9413AF6B017C0104
:101F0000209181023091820240918302509184029B
:101F10000E94AEAE18164CF06091690270916A0290
:101F200080916B0290916C021BC0209195023091C0
:101F300096024091970250919802C701B6010E9403
:101F4000F3B187FF05C0C701B6010E94A26C08C0AB
:101F500060917D0270917E0280917F02909180025B
:101F600020E030E048EC52E40E9413AF20E030E083
:101F700048EA51E40E9413AF2091250230912602D5
:101F800040912702509128020E9404B16B017C010C
:101F900065E773E088E192E10E94344B68E172E109
:101FA000CE0101960E94FF4B42E350E060E070E0FA
:101FB000CE0101960E94C48FCE0101960E94A34BD0
:101FC00022E0B701A601CE0101960E94A84B67E06E
:101FD00076E0CE0180960E94074CBE016F5F7F4F76
:101FE000CE0180960E94234B61E076E00E940C4B6C
:101FF000BC018EE192E10E948E4BCE0180960E9440
:10200000A34BCE0101960E94A34B6EE172E1CE017B
:1020100001960E94FF4B42E350E06FEF7FEFCE014D
:1020200001960E947C8DCE0101960E94A34B809167
:10203000430C882311F40C940B1D60E273E080E0E4
:1020400090E00E9434860C940B1D0E948D3E69EA3C
:1020500073E08EE192E10E94344B6EE172E1CE01B9
:1020600001960E94FF4B4AE050E060E070E0CE0134
:1020700001960E94C48FCE0101960E94A34B60EA94
:1020800073E088E192E10E94344B68E172E1CE0195
:1020900001960E94FF4B44E150E06FEF7FEFCE01CD
:1020A00001960E947C8DCE0101960E94A34B8091E7
:1020B000EE0B9091EF0B8230910549F40E946C86F3
:1020C00081111AC01092EF0B1092EE0B15C0892BE4
:1020D000C9F40E946C86882339F082E090E09093E6
:1020E000EF0B8093EE0B08C00E946C868111F5CF38
:1020F0000E946C868111F1CF8091EE0B9091EF0BD5
:10210000029741F164E973E08EE192E10E94344B61
:102110006EE172E1CE0101960E94FF4B4AE050E071
:1021200060E070E0CE0101960E94C48FCE0101965E
:102130000E94A34B6EE172E1CE0101960E94FF4B1B
:1021400068ED7BE0CE0101960E940C4B68E172E1E4
:102150000C94321A8AE090E00E9437766B017C0181
:1021600020E030E0A9010E94AEAE181634F08AE0FB
:1021700090E00E9437766B017C01BBE0AB2EB12C66
:1021800020E030E042ED53E4C701B6010E94AEAE5C
:1021900018168CF031E0A31AB10869F068EC70E011
:1021A00080E090E00E94348683E090E00E943776E1
:1021B0006B017C01E5CF20E030E0A901C701B60149
:1021C0000E94AEAE18163CF066E873E08EE192E134
:1021D0000E94344B31C020E030E048EC52E4C701AB
:1021E000B6010E94AEAE87FF02C021E001C020E030
:1021F000B701A601CE0101960E94A84B66E076E0E9
:10220000CE0180960E94074CBE016F5F7F4FCE01CA
:1022100080960E94234B6BE076E00E940C4BBC0141
:102220008EE192E10E948E4BCE0180960E94A34BDC
:10223000CE0101960E94A34B6EE172E1CE010196A0
:102240000E94FF4B42E350E06FEF7FEFCE0101961B
:102250000E947C8DCE0101960E94A34B6DE773E036
:1022600088E192E10E94344B68E172E1CE0101966F
:102270000E94FF4B42E350E060E070E0CE01019627
:102280000E94C48FD0CE0E9490872B013C0184ED28
:102290009DE00E94168E64E670E080E090E00E946F
:1022A000348640E855E260E070E084ED9DE00E94F5
:1022B000816D64E670E080E090E00E94348662EE1A
:1022C00073E088E192E10E94344B68E172E1CE0153
:1022D00001960E94FF4B42E350E06FEF7FEFCE018B
:1022E00001960E94C48FCE0101960E94A34B67ED18
:1022F00073E088E192E10E94344B68E172E1CE0123
:1023000001960E94FF4B42E350E06FEF7FEFCE015A
:1023100001960E947C8DCE0101960E94A34B809174
:102320000D0C90910E0C8D7F1CAEA12CB12CC12CEC
:10233000D12CE12CF12C019709F46FC0AE01405E65
:102340005F4F59AF48AFCE014E969BAF8AAF0E9408
:102350009087DC01CB0184199509A609B709883B50
:102360009B40A105B10508F058C084ED9DE00E9496
:102370005D47892B09F44AC02CED35E040E050E080
:102380002093D80D3093D90D4093DA0D5093DB0D87
:102390000E944D6D97FD06C082349105C9F780E01B
:1023A00090E002C08FEF9FEF892B81F5AE014F5F68
:1023B0005F4F1A014A010E944D6D97FF06C0898147
:1023C0008D3421F520E030E009C0D4018D934D011A
:1023D000E8ADF9ADEA17FB0771F7F1CFD1018D91A7
:1023E0001D01280F311DEAADFBADAE17BF07B1F7D8
:1023F0002E5B3F4F8E8D90E0982F88274F8D840F56
:10240000911D2817390711F40C94301D62E370E018
:1024100080E090E00E9434869ACF0E949087DC0191
:10242000CB0184199509A609B709883B9B40A105F2
:10243000B10518F42CAD2111BDC00E948D3E68E19C
:1024400072E1CE0180960E94FF4B42E350E066E0CD
:1024500070E0CE0180960E94C48FCE0180960E94CB
:10246000A34B3CAD332311F40C94491D82E090E062
:1024700090930E0C80930D0CB501CE0180960E94B6
:102480002D50B601CE0186960E942D50B701CE0187
:10249000C2960E942D50BE016E5C7F4FCE018C967D
:1024A0000E94FF4B66E177E0CE018C960E940C4BB8
:1024B000BE016A5D7F4F0E94234B66E177E00E9478
:1024C0000C4BBE01605E7F4F0E94234BBC018EE12E
:1024D00092E10E948E4BCE018C960E94A34BCE01BE
:1024E000C2960E94A34BCE0186960E94A34BCE01BA
:1024F00080960E94A34B6EE172E1CE0180960E940D
:10250000FF4B4AE050E06FEF7FEFCE0180960E94D4
:102510007C8DCE0180960E94A34B61ED73E08FE12C
:1025200093E10E94734CB501CE0180960E942D501C
:10253000B601CE0186960E942D50B701CE018C9631
:102540000E942D506FE076E0CE01C2960E94074CAB
:10255000BE01645D7F4FCE01C2960E94234B68EDA1
:102560007BE00E940C4BBE016A5D7F4F0E94234BB3
:1025700068ED7BE00E940C4BBE01605E7F4F0E94C5
:10258000234B6FE176E00E940C4BBC018EE192E19F
:102590000E948E4BCE01C2960E94A34BCE018C9618
:1025A0000E94A34BCE0186960E94A34BCE0180963B
:1025B0000E94A34B62E370E080E090E00E943486CA
:1025C00084ED9DE00E94168E12C6E0905902F090B4
:1025D0005A0265E276E088E192E10E94794B0E941E
:1025E0008D3E68E172E1CE0101960E94FF4B4AE008
:1025F00050E06FEF7FEFCE0101960E94C48FCE01B5
:1026000001960E94A34BC7010E94757924966CAF76
:102610007DAF8EAF9FAF249780902F0290903002B5
:10262000A0903102B0903202A501940160912B027A
:1026300070912C0280912D0290912E020E943DB04B
:102640002B013C0120E030E0A9010E94AEAE8823BE
:1026500009F453C0C0903702D0903802E09039029C
:10266000F0903A0220E030E0A901C701B6010E94D3
:10267000AEAE18160CF041C0809133029091340236
:10268000A0913502B09136028CAF9DAFAEAFBFAF17
:102690009C01AD01C701B6010E94AEAE882369F16D
:1026A000A70196016CAD7DAD8EAD9FAD0E9404B1CA
:1026B0000E9439B26CAF7DAF8EAF9FAFA501940180
:1026C00024966CAD7DAD8EAD9FAD24970E943DB03C
:1026D000A30192010E9404B12CAD3DAD4EAD5FADA2
:1026E0000E9413AF0E9471B19B01AC01C701B601FA
:1026F0000E9413AF6B017C0103C0C12CD12C760169
:1027000068E172E1CE0101960E94FF4B4AE050E081
:1027100060E070E0CE0101960E94C48FCE01019668
:102720000E94A34B20E030E64AEE56E4C701B60112
:102730000E94F3B118163CF46EEE73E08EE192E164
:102740000E94344B25C021E0B701A601CE0180963E
:102750000E94A84B6FE276E0CE0101960E94074CE2
:10276000BE01605E7F4FCE0101960E94234B63E362
:1027700076E00E940C4BBC018EE192E10E948E4BF0
:10278000CE0101960E94A34BCE0180960E94A34BDE
:102790006EE172E1CE0101960E94FF4B4AE050E0EB
:1027A0006FEF7FEFCE0101960E947C8DCE010196E6
:1027B0000E94A34B64E670E080E090E00E943486C3
:1027C00036CCE090B702F090B8020E948D3E65E0F2
:1027D00070E080E090E00E9434868091B5108330F4
:1027E000E4F4C7010E9464786B017C016091B6102B
:1027F0007091B710072E000C880B990B0E94B4AE95
:10280000A70196010E9413AF20E030EC4FE754E49B
:102810000E9404B1AB01BC0103C040E050E0BA012A
:1028200023E0CE0101960E94A84B6AEF75E0CE012D
:1028300080960E94074CBE016F5F7F4FCE0180964D
:102840000E94234B6DEC75E00E940C4BBC018EE1A5
:1028500092E10E948E4BCE0180960E94A34BCE0146
:1028600001960E94A34B67E376E00C94940B909141
:10287000060C81E089278093060C8091430C882305
:1028800031F06EE172E187E39DE00E94786968ECC7
:1028900070E080E090E0D5CB1092430C0C940B1DBF
:1028A00081E08093430C809321118091181188233B
:1028B00049F16FEE77E08AE292E10E94794B86EE71
:1028C0009FEF9093080C8093070C20911B1130917F
:1028D0001C1180911D1190911E118217930724F0F5
:1028E00010921E1110921D1110920F1110921011C2
:1028F00010921111109212116CE271E080E090E0E0
:102900000E9434866AE272E180E392E10E948E4B7B
:102910008091070C9091080C90933E0C80933D0C95
:102920000C940B1D0E94E43E0C940B1D81E79EE06D
:102930000E94168E40E052EC61E070E081E79EE07C
:102940000E94816D8CED95E0A0E0B0E08093750E63
:102950009093760EA093770EB093780E64E670E0B5
:1029600080E090E00E9434868091EE0B9091EF0B16
:10297000019759F483E090E00E94D878811140C01B
:102980001092EF0B1092EE0B1AC081E090E00E94C3
:10299000D878882339F081E090E09093EF0B809312
:1029A000EE0B0DC083E090E00E94D8788111F3CF48
:1029B00083E090E00E94D8788111EDCF06C080912D
:1029C000EE0B9091EF0B0197D9F06DE274E088E186
:1029D00092E10E94344B68E172E1CE0101960E94BF
:1029E000FF4B44E150E06FEF7FEFCE0101960E9474
:1029F0007C8DCE0101960E94A34B61E274E0CDC0B4
:102A000065E174E08EE192E10E94344B6EE172E187
:102A1000CE0101960E94FF4BCE0101960E94988F35
:102A2000CE0101960E94A34B62E370E080E090E04B
:102A30000E9434866EE172E1CE0101960E94FF4B46
:102A400042E350E06FEF7FEFCE0101960E94C48F0A
:102A5000CE0101960E94A34B69E074E088E192E107
:102A60000E94344B68E172E1CE0101960E94FF4B57
:102A700044E150E06FEF7FEFCE0101960E947C8D24
:102A8000CE0101960E94A34B8BEB88A38AEA89A30F
:102A900081E08AA3C12CD12C412C512C3201212C54
:102AA000312CC6016AE070E00E9465B3892B49F4BD
:102AB00043E050E0BE01605E7F4F81E79EE00E94F0
:102AC000024765E070E080E090E00E943486BFEF4E
:102AD000CB1ADB0AE12CF12C812C912C540181E7DB
:102AE0009EE00E945D47892B81F4E4E08E169104FC
:102AF000A104B10454F094E02916310464F4A0E96F
:102B0000CA16A1E0DA0669F606C0F6E0EF16F1048F
:102B10000CF4EBC7F0CFC301B2010E94B4AE20E0C9
:102B200030E040E251E40E9404B120E030E040E8AF
:102B30005EE30E9413AF6B017C0120E030E040EACD
:102B400051E40E94F3B1181634F521E0B701A60153
:102B5000CE0101960E94A84B61E677E0CE018096F7
:102B60000E94074CBE016F5F7F4FCE0180960E948E
:102B7000234B6FE376E00E940C4BBC018EE192E1A7
:102B80000E948E4BCE0180960E94A34BCE010196EF
:102B90000E94A34B06C06DEF73E08EE192E10E94AC
:102BA000344B6EE172E1CE0101960E94FF4B4AE088
:102BB00050E060E070E0CE0101960E94C48FCE012B
:102BC00001960E94A34B6EE172E1CE0101960E9434
:102BD000FF4B68ED7BE0CE0101960E940C4B68E153
:102BE00072E10E94234BBC018EE192E10E948E4B68
:102BF000CE0101960E94A34B81E79EE00E94168EB3
:102C000016CA68EC74E0CE0101960E94F74B4AE0C8
:102C100050E06FEF7FEFCE0101960E947C8DCE01D8
:102C200001960E94A34B6091B5027091B60280910B
:102C3000290290912A020E94886EE4E18E2E912C46
:102C4000A12CB12CC12CD12CAFEFCA1ADA0AC501C4
:102C5000B4010E9434866091B5027091B6028091F1
:102C6000290290912A020E94886E7C01B3E0CB1663
:102C7000D10434F08EE1C816D10444F4EF2851F0A9
:102C800094E1890E911CA11CB11CDECFE114F1046A
:102C900009F00CC18091290290912A028B30910594
:102CA000C9F480917C1290917D12A0917E12B09116
:102CB0007F1280933D1390933E13A0933F13B093E4
:102CC00040138091781290917912A0917A12B0916C
:102CD0007B121DC08631910521F30C9701F580917F
:102CE000301390913113A0913213B091331380932C
:102CF0003D1390933E13A0933F13B09340138091E4
:102D00002C1390912D13A0912E13B0912F1380931B
:102D1000391390933A13A0933B13B0933C13409113
:102D20003D1350913E1360913F137091401321E089
:102D3000CE0101960E94A84B6DE07AE0CE0180960C
:102D40000E94074CBE016F5F7F4FCE0180960E94AC
:102D5000234BBC018EE192E10E948E4BCE01809606
:102D60000E94A34BCE0101960E94A34B40913913C0
:102D700050913A1360913B1370913C1321E0CE01C6
:102D800001960E94A84B62E476E0CE0180960E94F4
:102D9000074CBE016F5F7F4FCE0180960E94234B90
:102DA000BC018EE192E10E94BA4ACE0180960E9457
:102DB000A34BCE0101960E94A34B64E076E08EE126
:102DC00092E10E94AC4A6FEB79E0CE0101960E943D
:102DD000074C44E150E060E070E0CE0101960E94B3
:102DE000C48FCE0101960E94A34BC0903D13D0909A
:102DF0003E13E0903F13F090401320E030E0A90133
:102E0000C701B6010E94F3B120E030E040E05FE38B
:102E100087FD05C0C701B6010E943EB004C0C701CE
:102E2000B6010E943DB00E949DB1AB01BC01CE0134
:102E300001960E94326ABE016F5F7F4F88E192E186
:102E40000E94C04ACE0101960E94A34B60E087E039
:102E50000E94076A68E172E18FE193E10E94654C8C
:102E60006FED8FE193E10E945E4C68E476E08FE1C4
:102E700093E10E943E4D6091391370913A13809115
:102E80003B1390913C130E949DB14AE050E08FE1CA
:102E900093E10E94F44C64E076E08FE193E10E94BC
:102EA0003E4D64E670E080E090E0CBC8EFEFEE16B8
:102EB000FE06ACF06AEB74E0CE0101960E94F74B7F
:102EC0004AE050E060E070E0CE0101960E94C48FBD
:102ED000CE0101960E94A34B67E974E048C0FEEF63
:102EE000EF16FFEFFF0679F169E874E0CE01019675
:102EF0000E94F74B4AE050E060E070E0CE0101969E
:102F00000E94C48FCE0101960E94A34B6AE774E031
:102F10008EE192E10E94344BB701CE0101960E94EE
:102F20002D50BE016F5F7F4F8EE192E10E94BA4A41
:102F3000CE0101960E94A34B64E674E08EE192E11B
:102F40000E946A4A68C569E574E0CE0101960E9454
:102F5000F74B4AE050E060E070E0CE0101960E943D
:102F6000C48FCE0101960E94A34B69E374E08EE109
:102F700092E10E94344B4FC580910402882309F4EA
:102F80004AC56FEB79E0CE0101960E94074C4AE0FA
:102F900050E061E070E0CE0101960E94C48FCE0146
:102FA00001960E94A34B0E94028C35C58091430C70
:102FB00081110AC080911311811106C07EE1472E54
:102FC000512C612C712C05C063E0462E512C612CD4
:102FD000712C66ED74E08EE192E10E94344B6EE15B
:102FE00072E1CE0101960E94FF4B4AE050E06FEF84
:102FF0007FEFCE0101960E947C8DCE0101960E944A
:10300000A34B812C912C54011CAE1DAE1EAE1FAEE5
:1030100083E20E94EC6987E090E00E94E7690E94E9
:10302000E56966E970E080E090E00E94348683E222
:103030000E94EC6980E290E00E94E7690E94E569E5
:1030400066E970E080E090E00E94348662E070E023
:1030500083E290E00E94328FC12CD12C76018091C6
:103060006D1390E020916E13821B910918161906BA
:103070006CF48BEA9FE00E94AD55FE2CED2CDC2C0D
:10308000CC24C80ED11CE11CF11CE9CFC701B6014C
:103090000E94B4AE2AE939E949E95FE30E9404B12C
:1030A0000E949DB1AB01BC0184169506A606B70629
:1030B00014F44A015B01CE0180960E94326ABE017F
:1030C000605E7F4FCE0101960E94FF4B6BE476E07D
:1030D000CE0101960E940C4BBC0188E192E10E9456
:1030E0008E4BCE0101960E94A34BCE0180960E948A
:1030F000A34B68E172E1CE0101960E94FF4B4EE1C5
:1031000050E060E070E0CE0101960E946990CE012F
:1031100001960E94A34B2CAD3DAD4EAD5FAD2F5F30
:103120003F4F4F4F5F4F2CAF3DAF4EAF5FAF42169B
:103130005306640675060CF06BCFB501A401CE01F1
:1031400080960E94326ABE01605E7F4FCE0101967A
:103150000E94FF4B6BE476E0CE0101960E940C4B7F
:10316000BC0188E192E10E948E4BCE0101960E9443
:10317000A34BCE0180960E94A34B68E172E1CE0181
:1031800001960E94FF4B4AE050E060E070E0CE0103
:1031900001960E94C48FCE0101960E94A34BB501F7
:1031A000A401CE0101960E94326A65E279E0CE0167
:1031B00080960E94074CBE016F5F7F4FCE018096C4
:1031C0000E94234B6FE476E00E940C4B6EE172E1AB
:1031D0000E94234BBC018EE192E10E948E4BCE01F6
:1031E00080960E94A34BCE0101960E94A34B62E3FE
:1031F00070E080E090E00C942110E090B302F09039
:10320000B40281E080932C0564E670E080E090E0F9
:103210000E9434860E948D3EC7010E9464780E94FD
:103220009DB120E034E0A901461B570BBA01CE0145
:1032300001960E942D5064E576E0CE0180960E94B2
:10324000074CBE016F5F7F4FCE0180960E94234BDB
:10325000BC018EE192E10E948E4BCE0180960E94CD
:10326000A34BCE0101960E94A34B60E087E00E9431
:10327000076A66EE74E0CE0101960E94F74B42E3C6
:1032800050E068E070E0CE0101960E94C48FCE014C
:1032900001960E94A34B6EE172E1CE0101960E945D
:1032A000FF4B42E350E06FEF7FEFCE0101960E94AB
:1032B0007C8DCE0101960E94A34B6BE576E0CAC0DF
:1032C0008091B1029091B2020E9464780E949DB1F7
:1032D0006B017C017093F10B6093F00B62E370E083
:1032E00080E090E00E943486B601CE0101960E94F3
:1032F0002D50BE016F5F7F4F8EE192E10E94C04A68
:10330000CE0101960E94A34B809176129091771284
:10331000892B09F45EC062E772E1CE0180960E94BB
:10332000FF4BBE01605E7F4FCE0101960E94FF4BB6
:1033300044E150E060E070E0CE0101960E94C48F4D
:10334000CE0101960E94A34B65E676E0CE01019680
:103350000E94074C6EE172E1CE0101960E94234B60
:10336000BC0188E192E10E948E4BCE0101960E9441
:10337000A34B68E172E1CE0101960E94FF4B44E14C
:1033800050E06FEF7FEFCE0101960E947C8DCE0161
:1033900001960E94A34BBE01605E7F4FCE01019655
:1033A0000E94FF4B68ED7BE0CE0101960E940C4B22
:1033B00068E172E10E94234BBC018EE192E10E9420
:1033C0008E4BCE0101960E94A34BCE0180960C94A9
:1033D000151060E776E088E192E10E94794B68E1A0
:1033E00072E1CE0101960E94FF4B44E150E060E0A3
:1033F00070E0CE0101960E94C48FCE0101960E941A
:10340000A34B64E576E0CE0101960E94074C6EE185
:1034100072E1CE0101960E94234BBC0188E192E14A
:103420000E948E4BCE0101960E94A34B68E172E18F
:10343000CE0101960E94FF4B44E150E06FEF7FEF19
:10344000CE0101960E947C8DCE0101960E94A34B75
:1034500065E676E0CE0101960E94074C6EE172E1CE
:10346000CE0101960E94234BBC018EE192E10E94A5
:103470008E4BCE0101960E94A34B0C9417108091A5
:103480000402882309F4C7C28091430C811104C04F
:1034900080911311882329F082E090E00E94684215
:1034A000BAC2C0905502D0905602E0905702F090F8
:1034B000580220E030E040E450E4C701B6010E9429
:1034C000F3B118166CF420E030E04AEF54E4C70181
:1034D000B6010E9413AF0E949DB16B017C0106C032
:1034E00040E3C42E45E7D42EE12CF12C0E948D3E02
:1034F00060E080E00E94076A67EF74E08FE193E18B
:103500000E94734C61E080E00E94076A6FEE74E0F5
:103510008FE193E10E94734C64E670E080E090E0FC
:103520000E9434860E9490876093EA0B7093EB0BA5
:103530008093EC0B9093ED0B0E9490878090EA0BA8
:103540009090EB0BA090EC0BB090ED0BDC01CB015D
:1035500088199909AA09BB098C159D05AE05BF05F7
:103560000CF059C283E090E00E9468420E9490876C
:1035700064E170E080E090E00E943486DDCF0E943C
:10358000F96187E39DE00E94FB4745C267E175E072
:1035900088E192E10E94344B68E172E1CE0101962C
:1035A0000E94FF4B4AE050E060E070E0CE010196DF
:1035B0000E94C48FCE0101960E94A34B3090B902A5
:1035C0008091FE0B811105C00E94908781E080935D
:1035D000FE0B8091F60B811105C00E94908781E05F
:1035E0008093F60B1092431310924213E090421313
:1035F000F090431358E2E516F1040CF07EC0832DE1
:103600000E94EA85F701EE0FFF1FE356F34F918307
:1036100080830E947D6B20E030E040EA50E40E940D
:1036200013AF20E030E040E85AE30E9413AF6B0193
:103630007C0140901D0250901E0260901F0270900D
:103640002002A30192016091190270911A028091E7
:103650001B0290911C020E943DB09B01AC0160E0F6
:1036600070E080EC90E40E943DB04B015C0120E0F2
:1036700030E0A9010E94AEAE20E030E040E650E428
:10368000811105C0C701B6010E9413AF1EC0C7015A
:10369000B6010E9413AFA30192010E943EB020E048
:1036A00030E040E850E40E943DB0A50194010E9442
:1036B00004B120E030E040EC50E40E9413AF20E081
:1036C00030E040E850E40E943EB06093F20B70930B
:1036D000F30B8093F40B9093F50B64E170E080E0C2
:1036E00090E00E943486809142139091431301969A
:1036F000909343138093421379CFC090F20BD090F4
:10370000F30BE090F40BF090F50B20E030E0A90112
:10371000C701B6010E94F3B187FD1EC022E0B701C8
:10372000A601CE0101960E94A84B64E776E0CE0187
:1037300080960E94074CBE016F5F7F4FCE0180963E
:103740000E94234BBC018EE192E10E948E4BCE0180
:1037500080960E94A34B49C168E075E08EE192E13A
:103760000E94344B46C180910402882309F453C15E
:103770008091430C81112BC080911311811127C0BE
:10378000C0905502D0905602E0905702F090580237
:1037900020E030E04AE754E4C701B6010E9413AFCD
:1037A0000E949DB14B015C0120E030E040EA50E412
:1037B000C701B6010E9413AF20E030E040EA50E4B8
:1037C0000E943EB00E949DB1A501940108C021E075
:1037D00030E040E050E06AE070E080E090E00E947D
:1037E0004E6519C1C7010E94F29115C1C7010E941F
:1037F0000B5D11C180919713882309F40CC165E614
:1038000075E0CE0101960E94F74BCE0101960E9411
:10381000BB70FDC080919B0C90919C0C892BA1F4F6
:1038200081E090E090939C0C80939B0C8EED93E054
:103830009093380C8093370C0E94E46D68EC70E034
:1038400080E090E00E94348668E575E0CE01019644
:103850000E94F74B44E650E06FEF7FEFCE010196F8
:103860000E947C8DCE0101960E94A34BE0E0F0E027
:103870001995D1C00E9428870E948D3E0E94FB7539
:10388000CAC09091181181E089278093181188236C
:1038900069F161E575E08EE192E10E94344B0E948E
:1038A000908760930F117093101180931111909372
:1038B000121180911B1190911C11181619065CF4BD
:1038C00020911D1130911E112817390724F01092F4
:1038D0001E1110921D1190911F1180911A119817AD
:1038E0005CF010921F111092201106C069E475E07F
:1038F0008EE192E10E94344B809118118093131154
:103900006EE172E1CE0101960E94FF4B4AE050E069
:1039100068E070E0CE0101960E94C48FCE0101964E
:103920000E94A34B6CE375E0CE0101960E94F74B19
:103930004AE050E06FEF7FEFCE0101960E947C8D50
:10394000CE0101960E94A34B6EE275E08EE192E1FA
:103950000E946A4A61E179E0CE0101960E94074C1B
:103960006EE172E1CE0101960E94234BBC018EE113
:1039700092E10E948E4BCE0101960E94A34B809152
:10398000430C809321118CE291E00E940A6E809199
:10399000430C882309F43FC06FEE77E08AE292E19E
:1039A0000E94794B86EE9FEF9093080C8093070C52
:1039B00032C0F092080CE092070C87E39DE00E9471
:1039C000FB4760E275E08EE192E10E94344B6FEBC1
:1039D00079E0CE0101960E94074C4AE050E060E099
:1039E00070E0CE0101960E94C48FCE0101960E9424
:1039F000A34B6EE172E1CE0101960E94FF4B4AE0BB
:103A000050E06FEF7FEFCE0101960E947C8DCE01DA
:103A100001960E94A34B809122129091231200974D
:103A2000A1F0419720F4023011050CF0A3C06EE123
:103A300072E1CE0101960E94FF4BCE0101960E94D9
:103A4000BB70CE0101960E94A34B64E670E080E05B
:103A500090E00E943486A1C00E94B13E0C94CB0E2F
:103A6000EC80F12CFE2CEE248D81E80EF11CCE8032
:103A7000D12CDC2CCC248F81C80ED11CA884B12C75
:103A8000BA2CAA248985A80EB11C21E02CAF0C9475
:103A9000061266EC73E08EE192E10E94344B6EE117
:103AA00072E1CE0180960E94FF4B4AE050E060E058
:103AB00070E0CE0180960E947C8DCE0180960E949F
:103AC000A34B63EB73E08EE192E10E94344B809153
:103AD0000D0C90910E0C029711F00C94DA121092CA
:103AE0000E0C10920D0C0C94DA1281E79EE00E94ED
:103AF0005D47892B71F081E79EE00E943B47E1E042
:103B0000F0E0EC0FFD1FEE0DFF1D80832FEFE21A9A
:103B1000F20A65E070E080E090E00E94348636E0D2
:103B2000E316F10401F5998188A198131CC09A81CC
:103B300089A1981318C09B818AA1981314C08D8104
:103B400090E0A0E0B0E0BA2FA92F982F88272C8111
:103B5000820F911DA11DB11D480E591E6A1E7B1EAC
:103B60004FEF241A340A5FEF851A950AA50AB50AA1
:103B70000C946F156EE172E1CE0101960E94FF4B2D
:103B80004AE050E06FEF7FEFCE0101960E947C8DFE
:103B9000CE0101960E94A34B4ACFCB5BDF4F0FB6FD
:103BA000F894DEBF0FBECDBFDF91CF911F910F9173
:103BB000FF90EF90DF90CF90BF90AF909F908F904D
:103BC0007F906F905F904F903F902F9008952F922D
:103BD0003F924F925F926F927F928F929F92AF929D
:103BE000BF92CF92DF92EF92FF920F931F93CF93EA
:103BF000DF93CDB7DEB728970FB6F894DEBF0FBEC0
:103C0000CDBFFC018DEB9FE0938782878091BA0F37
:103C100090E0958784878091871090E097878687CA
:103C20008091B70F853009F063C68091BF0F9091E6
:103C3000C00F885891098D35910588F48091BA0F8D
:103C4000843041F48091C10F9091C20F80974797C3
:103C500008F47DC08091BA0F843408F05EC0809172
:103C6000BA0F8A3108F4D5C08091BD0F9091BE0F74
:103C7000843F914050F4118610868FEF9FEFDC0156
:103C800084839583A683B7833CC08091BF0F9091B6
:103C9000C00F85974B9708F0BCC003ECE02E0FE0F7
:103CA000F02E82E090E040E050E0BA018C010F5F1E
:103CB0001F4F2091BA0F30E0021713076CF49701E1
:103CC00022503109D9012D913C91275031092730DB
:103CD000310508F47FC0C8010197959587959187B4
:103CE00080870C971CF41186108693C044835583FB
:103CF0006683778384E090E00DC0448355836683B8
:103D000077838BE090E006C0448355836683778396
:103D10008CE090E0918380831EC58091C10F9091CB
:103D2000C20F825491098E9708F099CF20E030E0BD
:103D3000C12CD12C7601A9014D53504FDA014D9180
:103D40005C91495051094930510598F088CF8091D4
:103D5000C30F9091C40F0997099708F07BCF118684
:103D600010868FEF9FEFDC0184839583A683B78352
:103D7000C2C5B9016B53704FDB014D915C91475146
:103D8000510942315105C0F4D701C601880F991F6E
:103D9000AA1FBB1F6C017D016894C0F82C5F3F4FC8
:103DA0002038310541F620E230E031872087C48297
:103DB000D582E682F7829FC5DB014D915C9146502A
:103DC00051094730510508F04ACFCC0CDD1CEE1CE0
:103DD000FF1CE4CFD7012D913C91235131092F30A5
:103DE000310550F4440F551F661F771F416002963E
:103DF000B4E0EB0EF11C5ACFD7012D913C912A5023
:103E000031092930310528F4440F551F661F771FEB
:103E1000EECF8091BA0F8A3108F460C08091BD0F57
:103E20009091BE0F8032934008F425CF8091BF0F50
:103E30009091C00FC697869708F050C08091C10F2F
:103E40009091C20FC697869708F048C0B5ECEB2E4C
:103E5000BFE0FB2E83E090E040E050E0BA018C012F
:103E60000F5F1F4F2091BA0F30E00217130764F461
:103E7000970122503109D9012D913C912C503109E3
:103E80002B30310560F0C801019795958795918792
:103E900080870C970CF031CF118610861FC0D70198
:103EA0002D913C91255231092B31310550F4440FAD
:103EB000551F661F771F41600296B4E0EB0EF11CA0
:103EC000CECFD7012D913C912C5031092A303105AC
:103ED00028F4440F551F661F771FEECF8091BA0F4D
:103EE000823208F452C08091BF0F9091C00F0697A4
:103EF000079708F04AC043ECC42E4FE0D42E82E06E
:103F000090E040E050E0BA018C010F5F1F4F20911C
:103F1000BA0F30E002171307F4F4D6011297ED90B0
:103F2000FC9011979D01BEE1EB1AF108A7E1EA169A
:103F3000F104E0F4440F551F661F771F4160D6015E
:103F40002D913C91B4E0CB0ED11C2350310925308A
:103F50003105C8F0C80101979595879591878087AD
:103F600040970CF0D1CE118610860FC0D9012D914B
:103F70003C912C5031092B30310538F4440F551F3A
:103F8000661F771FDCCF0296BFCF7F011C821B828A
:103F900081E090E09A8389838091BA0F8D3070F42C
:103FA0001C821B8281E090E09A838983F7018485DB
:103FB0009585181619060CF474C0D1C029E733E0B2
:103FC000AE014D5F5F4FBE016F5F7F4FC7010E9423
:103FD0004E99892B29F729E733E0AE014D5F5F4FFA
:103FE000BE016F5F7F4FC7010E944E990197C1F6D6
:103FF00029E733E0AE014D5F5F4FBE016F5F7F4F3A
:10400000C7010E944E99892B59F6812C912C54019D
:1040100000E010E08091BA0F90E029813A812817E2
:10402000390794F529E733E0AE014D5F5F4FBE01DC
:104030006F5F7F4FC7010E944E996C0129E733E003
:10404000AE014D5F5F4FBE016F5F7F4FC7010E94A2
:104050004E99F1E0CF16D10451F4892B09F0A0CF8D
:10406000880C991CAA1CBB1C689480F80AC0CD2837
:1040700009F096CF019709F093CF880C991CAA1CE0
:10408000BB1C0F5F1F4FC6CFD70119961C930E9311
:104090001897F70184829582A682B78281E090E02A
:1040A00039CE0284F385E02D82E090E09A83898303
:1040B0008281938189974E9708F051C083E090E008
:1040C0009A838983848195810B970A9708F047C06A
:1040D0002CEB31E0AE014D5F5F4FBE016F5F7F4F54
:1040E000C7010E944E99892BD1F52CEB31E0AE012E
:1040F0004D5F5F4FBE016F5F7F4FC7010E944E99BA
:10410000019769F5412C512C320100E010E0F701D4
:104110002485358589819A81821793070CF02FC1F8
:104120002CEB31E0AE014D5F5F4FBE016F5F7F4F03
:10413000C7010E944E995C010330110509F0E5C0EA
:104140002CEB31E0AE014D5F5F4FBE016F5F7F4FE3
:10415000C7010E944E99A816B90609F4D6C0D70126
:104160001A96ED91FC911B9782819381C697869751
:10417000E0F4848195814B974597B8F4DF0116965A
:104180006F0126ECC20ED11C20E030E040E050E090
:1041900060E070E080E090E00D911C911197095073
:1041A00011090830110508F4F4C08091BA0F893361
:1041B00070F182819381895791098335910508F4C3
:1041C0001BC125C0D90112966D917C911397665140
:1041D00071096131710508F037C1D501C401880F3B
:1041E000991FAA1FBB1F4C015D01689480F84E5FA8
:1041F0005F4F2C5F3F4F4B33510509F40CC1D90180
:104200006D917C916A50710969307105D8F2809185
:10421000BA0F823231F4828193810A97099708F4A8
:1042200023C1828193818957910983359105D0F407
:104230008091BA0F8132B0F084819581CA978997B5
:1042400088F49F012A5F3F4F812C912C540143E059
:1042500050E0D9016D917C916A5071096930710506
:1042600008F41EC1828193818C549109C59778F41A
:104270008091BA0F843031F484819581809747977B
:1042800008F46CC18091BA0F843408F04EC180915B
:10429000BA0F863460F1828193810C970B9708F4F2
:1042A000A9C125C0D90112966D917C9113976E51C9
:1042B00071096731710508F0D1C1D501C401880FBA
:1042C000991FAA1FBB1F4C015D01689480F84E5FC7
:1042D0005F4F2C5F3F4F4534510509F4A6C1D9010A
:1042E0006D917C916C5071096B307105D8F28091A1
:1042F000BA0F883508F4E4C1828193818558910909
:104300008B35910508F4BAC1DBC12CEB31E0AE016D
:104310004D5F5F4FBE016F5F7F4FC7010E944E9997
:104320006C010330110579F42CEB31E0AE014D5FE7
:104330005F4FBE016F5F7F4FC7010E944E99C81645
:10434000D90609F00CCFA114B10459F4CA94CD28B0
:1043500009F005CF440C551C661C771C689440F886
:104360000BC0AA94AB2809F0FACECD2809F0F7CEFD
:10437000440C551C661C771C0F5F1F4FC8CE11875D
:104380000087F701448255826682778282E090E05E
:10439000C1CC12960D911C911397015111090D304A
:1043A0001105E0F401E00E9480B321601496AC1581
:1043B000BD0509F0F1CEF701248335834683578389
:1043C00000E20E949BB32283338385E090E09183D7
:1043D000808380E390E091878087BDC112960D9124
:1043E0001C911397045011090530110508F0DDCE1A
:1043F00001E00E9480B3DACF84819581CA978997C2
:1044000008F005CF9F012A5F3F4F812C912C54016A
:1044100043E050E0F4CE9F012A583F4FD9012D913F
:104420003C912A5031092930310508F0F0CE2CE1B9
:1044300030E0F70131872087D70184829582A682F8
:10444000B7828AE090E085C1D90112966D917C9186
:104450001397665071096730710508F0D8CE880C43
:10446000991CAA1CBB1CC3CE2091BA0FCF01820F8E
:10447000911D820F911DDC0112978D919C910A97DD
:10448000099708F0CECEF701118610868FEF9FEFC7
:10449000DC0184839583A683B78386E090E03ACCE1
:1044A000D90112966D917C91139766517109613112
:1044B000710558F5D501C401880F991FAA1FBB1FAC
:1044C0004C015D01689480F84E5F5F4F2C5F3F4F59
:1044D0004332510509F0BDCE9F012A5B3F4FD90100
:1044E0002D913C912A5031092930310508F0BACE7E
:1044F00020E130E0F70131872087D701848295825F
:10450000A682B78286E090E024C1D90112966D910F
:104510007C911397665071096730710508F0A2CE3F
:10452000880C991CAA1CBB1CCFCF8481958189540F
:104530009109C39708F0ABCE9F012A5F3F4FAF01AF
:104540004A575F4F812C912C5401D9016D917C9178
:104550006950710969307105B8F099CE86819781EB
:104560000997099708F08ECED70119961C921E92D2
:1045700018978FEF9FEFDC01F70184839583A68363
:10458000B78387E090E0C6CBD90112966D917C91FC
:1045900013976651710961317105E0F4D501C401C9
:1045A000880F991FAA1FBB1F4C015D01689480F8FA
:1045B0002C5F3F4F2417350741F620E230E0F7012A
:1045C00031872087D70184829582A682B78287E0CF
:1045D00090E0BFC0D90112966D917C9113976650FF
:1045E00071096730710508F052CE880C991CAA1C1D
:1045F000BB1CDECF848195810997099708F077CE9F
:10460000868197818C974F9708F071CE8085918530
:1046100089974D9708F06BCE9F01265F3F4F812C05
:10462000912C540145E050E05ACE9F0126573F4F50
:10463000D9012D913C912C5031092B30310508F0D6
:1046400056CE20E230E0F70131872087D7018482FF
:104650009582A682B78288E090E07BC0D90112964D
:104660006D917C911397695071096930710508F05B
:104670003ECE880C991CAA1CBB1C29CE8481958136
:10468000825491098E97E0F48F01045C1F4F8DE1F5
:1046900090E040E050E02091BA0F30E02450310922
:1046A000821793070CF063C0980122503109D90199
:1046B0002D913C91295031092830310508F46EC004
:1046C0008091BA0F803209F07EC082819381069773
:1046D000069708F078C0848195810997099708F0BA
:1046E00072C09F012A5F3F4FAF01425C5F4F812C38
:1046F000912C5401D9016D917C91665071096630FD
:10470000710508F060C0D90112966D917C911397E4
:10471000695171096331710508F0D5C0D501C40133
:10472000880F991FAA1FBB1F4C015D01689480F878
:104730002C5F3F4F24173507E9F62EE030E0F701F4
:1047400031872087D70184829582A682B7828FE045
:1047500090E08D939C9381E090E0D0C0D8012D91A2
:104760003C91285131092231310550F1CB0101979B
:1047700095958795D70119969C938E9318978A974C
:104780000CF49ECF052E000C660B770BF7014483CB
:1047900055836683778389E090E0BCCABC016F5F74
:1047A0007F4FD8012D913C91275031092730310599
:1047B000A8F6440F551F416002960C5F1F4F6BCF48
:1047C000440F551FF9CFD7011C962D903C901D9793
:1047D000B6E02B1631040CF486C08F010E5F1F4F1C
:1047E00075EC872E7DE9972E7CE1A72E71E8B72E18
:1047F000E3E0CE2ED12CF801648175816080718058
:1048000080E090E00E94B2AE6D837E838F839887B4
:10481000B30180E090E00E94B2AE2B013C012DEC90
:104820003CEC4CE45FE30E9413AF9B01AC016D8153
:104830007E818F8198850E94AEAE87FD19C02DECD8
:104840003CEC4CE45FE36D817E818F8198850E9412
:1048500013AF9B01AC01C301B2010E94AEAEE82FC1
:10486000880FFF0BEE27FF0FEE1FFF27319602C0C8
:10487000E0E0F0E0A501940163E971E080E091E0FF
:104880000E9456B34F01FF0FAA08BB088626972641
:10489000A826B926FFEFCF1ADF0A0E5F1F4F2C1490
:1048A0003D0409F0A8CFD70114968D929D92AD9248
:1048B000BC92179780E290E019969C938E9318977C
:1048C0008FEF9FEF46CFD90112966D917C91139790
:1048D000695071096930710508F075CF880C991C11
:1048E000AA1CBB1C25CF82E08093B70F1092BA0F91
:1048F00080E090E003C083E090E00CCA28960FB6F9
:10490000F894DEBF0FBECDBFDF91CF911F910F9105
:10491000FF90EF90DF90CF90BF90AF909F908F90DF
:104920007F906F905F904F903F902F9008955F928F
:104930006F927F928F929F92AF92BF92CF92DF92AF
:10494000EF92FF920F931F93CF93DF93CDB7DEB714
:10495000E4970FB6F894DEBF0FBECDBF6CE372E1F3
:1049600086E392E10E948E4B0E942A8563E277E003
:10497000CE0101960E94074CBE016F5F7F4F86E318
:1049800092E10E940F85182FCE0101960E94A34B41
:10499000112309F476C026E030E045E050E06CE3F6
:1049A00072E1CE0101960E941B4CBE016F5F7F4FEA
:1049B00088E192E10E94C04ACE0101960E94A34B79
:1049C00088E192E10E94EE496B017C0164ED7AE09E
:1049D000CE0101960E94074CBE016F5F7F4F8CE3B2
:1049E00092E10E94BF84AC014F5F5F4F6CE372E1C4
:1049F000CE010B960E94D83EBE01655F7F4F88E1D5
:104A000092E10E94C04ACE010B960E94A34BCE01B8
:104A100001960E94A34B88E192E10E94EE499B011E
:104A2000E7E0F2E041E050E0A0910702B091080217
:104A3000A417B5075CF0A281B3812A173B0711F4D4
:104A4000138212824F5F5F4F3296EECF9601220F94
:104A5000331FF901E95FFD4F7183608382E090E0CD
:104A60000E9455776CE372E1CE0101960E94FF4BE4
:104A7000CE0101960E94988FCE0101960E94A34B11
:104A800031C069E277E0CE0101960E94074CBE0179
:104A90006F5F7F4F86E392E10E940F85182FCE0152
:104AA00001960E94A34B112349F1E7E0F2E081E077
:104AB00090E020910702309108022817390774F01E
:104AC000863091051CF49383828305C09C012E5F80
:104AD0003F4F3383228301963296EBCF82E090E002
:104AE0000E9455771092380C1092370C80E090E0BD
:104AF0000E94346E109254020C944F2F6FE277E0B4
:104B0000CE0101960E94074CBE016F5F7F4F86E386
:104B100092E10E940F85182FCE0101960E94A34BAF
:104B20001123F9F080919B0C90919C0C892BA1F49E
:104B300081E090E090939C0C80939B0C8EED93E031
:104B40009093380C8093370C0E94E46D68EC70E011
:104B500080E090E00E943486E0E0F0E019950C944B
:104B60004F2F66E377E0CE0101960E94074CBE010D
:104B70006F5F7F4F86E392E10E940F85182FCE0171
:104B800001960E94A34B1123B1F06EE377E0CE01B2
:104B900001960E94074C6DE073E1CE0101960E94E0
:104BA000234BBC018EE192E10E948E4BCE01019617
:104BB0000E94A34B20C068E477E0CE0101960E94DA
:104BC000074CBE016F5F7F4F86E392E10E940F8525
:104BD000182FCE0101960E94A34B112351F16CE5D1
:104BE00077E08EE192E10E94344B63E173E18EE164
:104BF00092E10E94BA4A61E179E0CE0101960E94F9
:104C0000074C6EE172E1CE0101960E94234BBC017C
:104C1000CE010B960E94FF4BCE010B960E94BB70FB
:104C2000CE010B960E94A34BCE0101960E94A34B8E
:104C300061CF6FE477E0CE0101960E94074CBE0180
:104C40006F5F7F4F86E392E10E940F85182FCE01A0
:104C500001960E94A34B112311F169E377E08EE1E5
:104C600092E10E94344B6EE172E1CE0101960E9406
:104C7000FF4BCE0101960E94BB70CE0101960E94AF
:104C8000A34B0E9494591092540265E577E08CE39F
:104C900092E10E94794B0E948C7E0C944F2F69E523
:104CA00077E0CE0101960E94074CBE016F5F7F4FF7
:104CB00086E392E10E940F85182FCE0101960E9493
:104CC000A34B112309F48CC064ED7AE0CE01019668
:104CD0000E94074CBE016F5F7F4F8CE392E10E9400
:104CE000BF84AC014F5F5F4F6CE372E1CE010B9666
:104CF0000E94D83EBE01655F7F4F88E192E10E942D
:104D0000C04ACE010B960E94A34BCE0101960E9491
:104D1000A34B88E192E10E94EE498B016CE277E0BF
:104D20008EE192E10E94344B80911811882331F07A
:104D300060E277E08EE192E10E94344B01151105AB
:104D400011F40C943B2FCE0101960E94E759CE013D
:104D500001960E94BB70CE0101960E94A34B0230C7
:104D600011050CF4C7CE67E775E0CE010B960E94E3
:104D7000F74BBE01655F7F4FCE0101960E94FF4B4E
:104D8000CE0101960E94BB70CE0101960E94A34BFA
:104D9000E12CF12C80911A11082E000C990BE816C9
:104DA000F9068CF4B701CE0101960E94F05BCE01AA
:104DB00001960E94BB70CE0101960E94A34BFFEFAB
:104DC000EF1AFF0AE7CFCE010B960E94A34B0230E9
:104DD000110509F48FCE8CE291E00E945E6E8ACEBE
:104DE00060E677E0CE0101960E94074CBE016F5F3E
:104DF0007F4F86E392E10E940F85182FCE01019626
:104E00000E94A34B112309F488C36CE372E1CE0125
:104E10008F960E94FF4B64ED7AE0CE0101960E94CE
:104E2000074CBE016F5F7F4FCE018F960E94BF84FB
:104E3000AC014F5F5F4FBE01615D7F4FCE01899630
:104E40000E94D83ECE0101960E94A34BBE01615D37
:104E50007F4FCE0101960E94FF4BCE0101960E942A
:104E6000988FCE0101960E94A34B64E677E0CE01B5
:104E700001960E94074CBE016F5F7F4FCE0189965D
:104E80000E9483848C01CE0101960E94A34B6FEB9C
:104E900079E0CE0183960E94074C6FEB79E0CE015A
:104EA0004D960E94074C1016110684F5A8014F5F1D
:104EB0005F4F8DA59EA54817590790F4BE01675D09
:104EC0007F4FCE0101960E94D83EBE016F5F7F4F9B
:104ED000CE0183960E94C04ACE0101960E94A34B48
:104EE000980140E050E0BE01675D7F4FCE01019622
:104EF0000E941B4CBE016F5F7F4FCE014D960E94FA
:104F0000C04ACE0101960E94A34B0DC06FEB79E021
:104F1000CE0183960E94794BBE01675D7F4FCE0123
:104F20004D960E948E4B89A19AA1892B09F4E6C265
:104F3000CE014D960E94EE498B01015011090831B6
:104F4000110514F007E110E017FF02C00FEF1FEF8B
:104F5000B801CE010B960E942D5066E677E0CE0197
:104F600001960E94074CBE01655F7F4FCE010196FE
:104F70000E94234BBC01CE0141960E94FF4BCE0103
:104F800041960E94988FCE0141960E94A34BCE017C
:104F900001960E94A34BCE010B960E94A34BBE012B
:104FA0006D5D7F4FCE0189960E948E4B64E677E05F
:104FB000CE0101960E94074CBE016F5F7F4FCE016C
:104FC00089960E9483847C01CE0101960E94A34BA6
:104FD0006FEB79E0CE0183960E94794B6FEB79E01D
:104FE000CE014D960E94794B1E141F040CF04EC04A
:104FF000A7014F5F5F4F8DA59EA54817590790F4F5
:10500000BE01675D7F4FCE0101960E94D83EBE0172
:105010006F5F7F4FCE0183960E94C04ACE010196FA
:105020000E94A34B970140E050E0BE01675D7F4FB7
:10503000CE0101960E941B4CBE016F5F7F4FCE01D7
:105040004D960E94C04ACE0101960E94A34BAE012C
:105050004F5F5F4F5A01E12CF12CA8014F5F5F4F6A
:105060008AE0849F9001859F300D1124F901E85E4C
:10507000FE4E6F01809F9001819F300D1124A90188
:105080004A5D5E4E3A018AE2582EC1C06FEB79E06C
:10509000CE0183960E94794BBE01675D7F4FCE01A2
:1050A0004D960E948E4BD3CFE114F10409F0BCC0A1
:1050B0000F3F8FEF180709F4B7C0CE014D960E943D
:1050C000F949C114D10439F044E050E0B601CE01F1
:1050D0004D960E949D84B601CE0141960E94074CD8
:1050E0006BE677E0CE010B960E94074CBE016F5E27
:1050F0007F4FCE010B960E94234BBC01CE014796F9
:105100000E94FF4BCE0147960E94988FCE01479692
:105110000E94A34BCE010B960E94A34BCE01419659
:105120000E94A34B89A19AA1029708F476C061E07E
:1051300070E0CE014D960E94594A082E000C990B42
:10514000803391050CF44C96E52DE81B8E2FF3016E
:105150008083FFEFEF1AFF0ABE016D5D7F4FCE0126
:1051600089960E948E4B64E677E0CE010B960E94F2
:10517000074CBE01655F7F4FCE0189960E948384F4
:105180004C01CE010B960E94A34B6FEB79E0CE0150
:1051900083960E94794B6FEB79E0CE014D960E9489
:1051A000794B181419040CF047C0A4014F5F5F4FEE
:1051B0008DA59EA54817590790F4BE01675D7F4FE6
:1051C000CE010B960E94D83EBE01655F7F4FCE0197
:1051D00083960E94C04ACE010B960E94A34B940175
:1051E00040E050E0BE01675D7F4FCE010B960E940C
:1051F0001B4CBE01655F7F4FCE014D960E94C04A99
:10520000CE010B960E94A34B52E0A50EB11C89A1C2
:105210009AA1892B09F048CF1DC0CE014D960E945E
:10522000EE49F301608395CFCE014D960E94EE4981
:10523000F501718360838DCF6FEB79E0CE018396AA
:105240000E94794BBE01675D7F4FCE014D960E9453
:105250008E4BDACF0F3F2FEF120709F07DC064E6C7
:1052600077E0CE010B960E94074CBE01655F7F4F31
:10527000CE0183960E9483848C01CE010B960E94FE
:10528000A34B17FF3BC109811A811016110634F494
:10529000093111052CF008E110E002C001E010E036
:1052A00000931A11B801CE0141960E942D5069E772
:1052B00077E0CE010B960E94074CBE016F5E7F4FD8
:1052C000CE010B960E94234BBC01CE0147960E9453
:1052D000FF4BCE0147960E94988FCE0147960E94C1
:1052E000A34BCE010B960E94A34BCE0141960E9488
:1052F000A34BE114F10459F18B819C8197FF02C00B
:1053000080E090E090931C1180931B1141E0E41623
:10531000F104E9F08D819E81181619062CF480178E
:10532000910724F48C0102C001E010E001500093C9
:105330001F1152E0E516F10451F08F81988518167F
:10534000190614F081E090E08150809320118CE2E6
:1053500091E00E940A6ED2C080911911082E000CB3
:10536000990B081719070CF083C0B701CE014196BD
:105370000E942D5063E877E0CE010B960E94074C07
:10538000BE016F5E7F4FCE010B960E94234BBC0186
:10539000CE0147960E94FF4BCE0147960E94988F00
:1053A000CE0147960E94A34BCE010B960E94A34BC1
:1053B000CE0141960E94A34B8AE0809FF001819F1D
:1053C000F00D1124E85EFE4E81E0878783E090E0D7
:1053D000918B808B938B828BE114F10409F48EC046
:1053E0008B819C818038910514F08FE790E08038A4
:1053F0002FEF920714F480E89FEF878741E0E416CF
:10540000F10409F47BC08AE0809FF001819FF00DD8
:105410001124E85EFE4E8D819E8197FF02C080E0E0
:1054200090E0918B808B52E0E516F10409F466C0A0
:105430008AE0809FF001819FF00D1124E85EFE4E0E
:105440008F81988597FF02C080E090E0938B828BDC
:1054500080911A11082E000C990B081719071CF0DF
:105460000F5F00931A118CE291E00E945E6E46C0BD
:10547000BE016D5D7F4FCE0147960E94FF4B60914C
:105480001911062E000C770BCE0141960E942D506B
:105490006BE877E0CE010B960E94074CBE01695E77
:1054A0007F4FCE010B960E94234B6CE977E00E9460
:1054B0000C4BBE016F5E7F4F0E94234BBC01CE019F
:1054C00047960E948E4BCE010B960E94A34BCE01B5
:1054D00041960E94A34BBE01695E7F4FCE010B96A1
:1054E0000E94FF4BCE010B960E94BB70CE010B9623
:1054F0000E94A34BCE0147960E94A34BCE014D962E
:105500000E94A34BCE0183960E94A34BCE018996A5
:105510000E94A34BCE018F9650C260EA77E0CE0185
:1055200001960E94074CBE016F5F7F4F86E392E1B8
:105530000E940F85182FCE0101960E94A34B1123C4
:10554000C9F164ED7AE0CE0101960E94074CBE01DC
:105550006F5F7F4F8CE392E10E94BF84AC014F5F8D
:105560005F4F6CE372E1CE010B960E94D83EBE0104
:10557000655F7F4F88E192E10E94C04ACE010B96A1
:105580000E94A34BCE0101960E94A34B88E192E1B9
:105590000E94EE496115710521F481E080932E058A
:1055A00006C06130710509F0A5CA10922E050E944F
:1055B0000B76A0CA65EA77E0CE0101960E94074CFF
:1055C000BE016F5F7F4F86E392E10E940F85182F27
:1055D000CE0101960E94A34B112309F452C143E06E
:1055E00050E06CE372E1CE0101960E94D83EBE010C
:1055F0006F5F7F4F88E192E10E94C04ACE01019621
:105600000E94A34B68E172E1CE0101960E94FF4B1C
:10561000CE0101960E94988FCE0101960E94A34B65
:105620001092380C1092370C68E172E1CE010196AD
:105630000E94FF4B60E0CE0101960E94994A8111C1
:1056400004C0CE0101960E94FA4ABE016F5F7F4FEF
:1056500089E193E10E948E4BCE0101960E94A34BFB
:1056600068E172E1CE0101960E94FF4B60E0CE013D
:1056700001960E94994A811104C0CE0101960E94B0
:10568000FA4ABE016F5F7F4F83E193E10E948E4B28
:10569000CE0101960E94A34B40911D1350911E1301
:1056A0004115510549F085EA90E1009729F0BC01C8
:1056B00089E193E10E949D84409117135091181342
:1056C0004115510549F083E091E1009729F0BC01B3
:1056D00083E193E10E949D848091370C9091380C76
:1056E0000E94346E6AEF76E0CE0101960E94074C6C
:1056F00068E172E1CE0101960E94234BBC01CE010C
:1057000041960E94FF4BCE0101960E94A34B8091CF
:10571000FF1090910011892B39F4BE016F5E7F4F0D
:1057200087E39DE00E94654C68EB7BE080E090E0C1
:105730000E9434868091FF1090910011029709F029
:1057400087C068E172E1CE0147960E94FF4B69EA8B
:1057500077E0CE0101960E94074CCE0101960E948F
:105760009BA9CE0101960E94A34B64EF71E080E0FB
:1057700090E00E9434866CEA77E0CE0101960E94A8
:10578000074CCE0101960E949BA9CE0101960E9472
:10579000A34B6CED75E080E090E00E94348665EBF1
:1057A00077E0CE0101960E94074CCE0101960E943F
:1057B0009BA9CE0101960E94A34B64EF71E080E0AB
:1057C00090E00E94348663EC77E0CE0101960E945F
:1057D000074CCE0101960E949BA9CE0101960E9422
:1057E000A34B64EF71E080E090E00E9434866AEFA2
:1057F00076E0CE0101960E94074CBE01695E7F4FA4
:10580000CE0101960E94234BBC01CE010B960E9453
:10581000FF4BCE0101960E94A34BCE010B960E9436
:10582000F949BE01655F7F4FCE0101960E94FF4B93
:10583000CE0101960E949BA9CE0101960E94A34B26
:10584000CE010B960E94A34BCE0147960E94A34B1C
:1058500068EB7BE080E090E00E94348665EA70E1CE
:10586000CE0101960E94074CCE0101960E94988FAE
:10587000CE0101960E94A34B10925402CE01419694
:105880009CC061ED77E0CE0101960E94074CBE01FD
:105890006F5F7F4F86E392E10E940F85182FCE0144
:1058A00001960E94A34B112309F48AC044E050E002
:1058B0006CE372E1CE0101960E94D83EBE016F5F9B
:1058C0007F4F88E192E10E94C04ACE0101960E947A
:1058D000A34B62E077E0CE0101960E94074C68E19D
:1058E00072E1CE0101960E94234BBC01CE010B96C2
:1058F0000E94FF4BCE0101960E94A34B8091FF10A6
:1059000090910011892B69F4BE01655F7F4F87E399
:105910009DE00E94654C68E873E180E090E00E94A1
:1059200034868091FF1090910011029709F041C0D8
:1059300066ED77E0CE0101960E94074C80911C1223
:1059400090911D12892B39F46FED77E0CE0101960D
:105950000E94794B15C0BE016F5F7F4FCE0141960B
:105960000E94FF4BCE0141960E949BA9CE01419619
:105970000E94A34B60ED77E080E090E00E943486C7
:10598000BE01655F7F4FCE0141960E94FF4BCE0165
:1059900041960E949BA9CE0141960E94A34B60EDC7
:1059A00077E080E090E00E943486CE0101960E946C
:1059B000A34B10925402CE010B960E94A34B6FC2D0
:1059C00068EE77E0CE0101960E94074CBE016F5F42
:1059D0007F4F86E392E10E940F85182FCE0101963A
:1059E0000E94A34B112309F462C06CE372E188E1C9
:1059F00092E10E948E4B81E0809354026CE372E14D
:105A0000CE0101960E94FF4BCE0101960E94988F15
:105A1000CE0101960E94A34B8091FF10909100113E
:105A2000029709F168E172E187E39DE00E94654C0D
:105A300068EB7BE080E090E00E943486CE01019626
:105A40000E946B75BE016F5F7F4F8CE392E10E94F5
:105A5000C04ACE0101960E94A34B60ED77E080E042
:105A600090E00E9434868091FF109091001102977F
:105A700071F468E172E1CE0101960E94FF4BCE0104
:105A800001960E949BA9CE0101960E94A34B809192
:105A9000401290914112892B09F42CC861E179E000
:105AA000CE0101960E94074C6CE372E1ACC86CEE2B
:105AB00077E0CE0101960E94074CBE016F5F7F4FD9
:105AC00086E392E10E940F85182FCE0101960E9475
:105AD000A34B112309F45CC08091FF109091001139
:105AE000019709F007C8CE0101960E947A608D8166
:105AF0009E81009709F4C9C1E981FA81208122239E
:105B000009F4C3C1079708F4C0C167E177E0CE018B
:105B10000B960E94F74B48EC50E06FEF7FEFCE0101
:105B20000B960E946990CE010B960E94A34BBE017A
:105B30006F5F7F4FCE010B960E94FF4B40ED57E009
:105B40006FEF7FEFCE010B960E947C8DCE010B96FE
:105B50000E94A34B62EF77E0CE010B960E94074CA8
:105B60006CE372E1CE010B960E94234BBC01CE0187
:105B700041960E94FF4BCE0141960E94BB70CE0120
:105B800041960E94A34BCE010B960E94A34B7DC170
:105B900060E078E0CE0101960E94074CBE016F5F85
:105BA0007F4F86E392E10E940F85182FCE01019668
:105BB0000E94A34B112361F125E030E044E050E066
:105BC0006CE372E1CE0101960E941B4CBE016F5F37
:105BD0007F4F88E192E10E94C04ACE0101960E9467
:105BE000A34B6CE372E1CE0101960E94FF4BCE0104
:105BF00001960E94988FCE0101960E94A34B88E1E6
:105C000092E10E94EE49CB010E9422910C947A25E8
:105C100065E078E0CE0101960E94074CBE016F5FFF
:105C20007F4F86E392E10E940F85182FCE010196E7
:105C30000E94A34B112361F127E030E046E050E0E1
:105C40006CE372E1CE0101960E941B4CBE016F5FB6
:105C50007F4F88E192E10E94C04ACE0101960E94E6
:105C6000A34B88E192E10E94EE49672B19F4109250
:105C7000971303C081E0809397136CE372E1CE0128
:105C800001960E94FF4BCE0101960E94988FFDC0A5
:105C90006CE078E0CE0101960E94074CBE016F5F78
:105CA0007F4F86E392E10E940F85182FCE01019667
:105CB0000E94A34B112309F476C080914012909169
:105CC0004112079708F4EBC046E050E06CE372E144
:105CD000CE0101960E94D83EBE016F5F7F4F88E1E2
:105CE00092E10E94C04ACE0101960E94A34B88E136
:105CF00092E10E94E34960935002709351028093B5
:105D000052029093530267E077E08EE192E10E94A5
:105D1000344B409150025091510260915202709167
:105D2000530221E0CE0101960E94A84BBE016F5F95
:105D30007F4FCE010B960E94FF4B6BED75E0CE01BD
:105D40000B960E940C4BBC018EE192E10E94BA4A74
:105D5000CE010B960E94A34BCE0101960E94A34B4D
:105D60006EE172E1CE0101960E94FF4BCE010196D9
:105D70000E94BB70CE0101960E94A34B0E949087A7
:105D800028EE33E040E050E00E940CB0CA01B901B7
:105D90000E94B2AE60933F0C7093400C8093410C14
:105DA0009093420C7CC063E178E0CE0101960E94A2
:105DB000074CBE016F5F7F4F86E392E10E940F8523
:105DC000182FCE0101960E94A34B112309F463C042
:105DD0008091401290914112079708F460C046E00C
:105DE00050E06CE372E1CE0101960E94D83EBE0104
:105DF0006F5F7F4F88E192E10E94C04ACE01019619
:105E00000E94A34B88E192E10E94E349609355020E
:105E100070935602809357029093580267EF76E092
:105E20008EE192E10E94344B40915502509156020E
:105E3000609157027091580221E0CE0101960E94B4
:105E4000A84BBE016F5F7F4FCE010B960E94FF4BA8
:105E50006BED75E0CE010B960E940C4BBC018EE100
:105E600092E10E94BA4ACE010B960E94A34BCE014A
:105E700001960E94A34B6EE172E1CE0101960E9451
:105E8000FF4BCE0101960E94BB70CE0101960E948D
:105E9000A34B0C947A25E9D5182F8823A1F01091F3
:105EA0005402112379F06CE372E1CE0101960E9455
:105EB000FF4BCE0101960E94988FCE0101960E9461
:105EC000A34B01C011E0812FE4960FB6F894DEBF1A
:105ED0000FBECDBFDF91CF911F910F91FF90EF903B
:105EE000DF90CF90BF90AF909F908F907F906F90FA
:105EF0005F9008954F925F926F927F929F92AF92C0
:105F0000BF92CF92DF92EF92FF920F931F93CF93A6
:105F1000DF93CDB7DEB7A9970FB6F894DEBF0FBEFB
:105F2000CDBF982E882351F080919713882331F0AC
:105F30006FEB79E08EE09FE00E945F6A0E94FB4F6A
:105F400060E08DE20E94565160E18DE20E94565160
:105F500068E08DE20E94565140908812509089125C
:105F600060908A1270908B12498E5A8E6B8E7C8E46
:105F7000C0908C12D0908D12E0908E12F0908F1203
:105F8000CD8EDE8EEF8EF8A28091901290919112BC
:105F9000A0919212B09193128EA39FA3A8A7B9A724
:105FA00089A39AA3ABA3BCA39920C9F180919713AD
:105FB0008823A9F164E47BE0CE0101960E94F74BAF
:105FC000CE0101960E94988FCE0101960E94A34BAC
:105FD0008E01075E1F4F5E0195E2A90EB11CD8012C
:105FE0006D917D918D919D918D0146E00E94A36AF6
:105FF00068ED7BE08EE09FE00E943E4DA016B1066A
:1060000071F76FEB79E0CE0101960E94074CCE014B
:1060100001960E94988FCE0101960E94A34B23E91E
:1060200038E144E85FE3C301B2010E9413AF2B01E2
:106030003C016D877E878F87988B22E430E645E8A8
:106040005FE3C701B6010E9413AF6B017C01698B4E
:106050007A8B8B8B9C8B25E83BEE41E95FE36EA14D
:106060007FA188A599A50E9413AF6D8B7E8B8F8B26
:10607000988F409288125092891260928A12709280
:106080008B12C0928C12D0928D12E0928E12F092EE
:106090008F1260939012709391128093921290934A
:1060A0009312992009F4A0C080919713882309F4D2
:1060B0009BC067E37BE0CE0101960E94F74BCE01C7
:1060C00001960E94988FCE0101960E94A34B8E01EB
:1060D000035F1F4F6E01B9E1CB0ED11C7801F801AF
:1060E00061917191819191918F0142E00E94A36A27
:1060F00068ED7BE08EE09FE00E943E4DC016D10629
:1061000071F76FEB79E0CE0101960E94074CCE014A
:1061100001960E94988FCE0101960E94A34B44E9FC
:1061200052E166E070E082E30E94F150A090941288
:10613000B0909512C0909612D0909712009198123C
:10614000109199126AE27BE08EE09FE00E94734C0E
:106150004AE050E0B5018EE09FE00E94F44C68ED0B
:106160007BE08EE09FE00E943E4D4AE050E0B601A9
:106170008EE09FE00E94F44C68ED7BE08EE09FE0B3
:106180000E943E4D4AE050E0B8018EE09FE00E9440
:10619000F44C6FEB79E08EE09FE00E945F6ACE01E5
:1061A00001960E94C35161E27BE08EE09FE00E9475
:1061B000734C8E010F5F1F4FD8016D917D918D91B2
:1061C0009D918D014AE00E94A36A68ED7BE08EE01C
:1061D0009FE00E943E4D0E151F0571F76FEB79E0B1
:1061E0008EE09FE00E945F6A61E08DE10E9456515F
:1061F0009920B1F080919713882391F06DE07BE0B6
:106200008EE09FE00E94734CAE014B5D5F4F61E0FA
:1062100070E08DE10E94F1508DA190E00E942A5122
:1062200062E08EE10E94565163E08FE10E94565178
:1062300064E080E20E945651992009F450C0809198
:106240009713882309F44BC061EF7AE08EE09FE05A
:106250000E94734CAE014B5D5F4F61E070E08EE1D8
:106260000E94F150CDA0D12CAE014B5D5F4F61E09B
:1062700070E08FE10E94F150EDA0F12CAE014B5D7A
:106280005F4F61E070E080E20E94F1500DA110E0EC
:106290004AE050E0B6018EE09FE00E94F44C68EDC9
:1062A0007BE08EE09FE00E943E4D4AE050E0B70167
:1062B0008EE09FE00E94F44C68ED7BE08EE09FE072
:1062C0000E943E4D4AE050E0B8018EE09FE00E94FF
:1062D000F44C6FEB79E08EE09FE00E945F6A65E02E
:1062E00081E20E9456519920B1F080919713882342
:1062F00091F06EED7AE08EE09FE00E94734CAE016B
:106300004B5D5F4F61E070E081E20E94F1508DA132
:1063100090E00E942A5166E082E20E945651992044
:10632000B1F080919713882391F066EC7AE08EE0CB
:106330009FE00E94734CAE014B5D5F4F61E070E0E7
:1063400082E20E94F1508DA190E00E942A5167E004
:1063500083E20E9456519920B1F0809197138823CF
:1063600091F060EB7AE08EE09FE00E94734CAE010A
:106370004B5D5F4F61E070E083E20E94F1508DA1C0
:1063800090E00E942A5168E084E20E9456519920D0
:10639000B1F080919713882391F068E97AE08EE05C
:1063A0009FE00E94734CAE014B5D5F4F61E070E077
:1063B00084E20E94F1508DA190E00E942A5169E090
:1063C00085E20E9456519920B1F08091971388235D
:1063D00091F06EE77AE08EE09FE00E94734CAE0190
:1063E0004B5D5F4F61E070E085E20E94F1508DA14E
:1063F00090E00E942A516AE086E20E94565199205C
:10640000B1F080919713882391F068E67AE08EE0EE
:106410009FE00E94734CAE014B5D5F4F61E070E006
:1064200086E20E94F1508DA190E00E942A516BE01B
:1064300088E20E9456519920B1F0809197138823E9
:1064400091F06FE47AE08EE09FE00E94734CAE0121
:106450004B5D5F4F61E070E088E20E94F1508DA1DA
:1064600090E00E942A516CE089E20E9456519920E6
:1064700009F479C080919713882309F474C067E305
:106480007AE08EE09FE00E94734CAE014B5D5F4F5F
:1064900061E070E089E20E94F1508DA190E00E94DD
:1064A0002A5160E27AE08EE09FE00E94734C66E041
:1064B00070E087E20E943C5190E00E942A5169E01E
:1064C0007AE08EE09FE00E94734C65E070E087E226
:1064D0000E943C5190E00E942A5162EF79E08EE0E8
:1064E0009FE00E94734C64E070E087E20E943C51A0
:1064F00090E00E942A5169ED79E08EE09FE00E94D1
:10650000734C62E070E087E20E943C5190E00E9490
:106510002A5160EC79E08EE09FE00E94734C61E0CC
:1065200070E087E20E943C5190E00E942A5167EAA5
:1065300079E08EE09FE00E94734C60E070E087E2BB
:106540000E943C5190E00E942A5166E979E08EE079
:106550009FE00E94734C63E070E087E20E943C5130
:1065600090E00E942A5141E067E070E087E20E94DB
:10657000695141E063E070E087E20E94695141E0C7
:1065800063E070E08AE20E946951992091F0809165
:106590009713882371F06DE779E08EE09FE00E9409
:1065A000734C63E070E08AE20E943C5190E00E94EC
:1065B0002A5140E063E070E08AE20E94695199202C
:1065C00091F080919713882371F063E679E08EE073
:1065D0009FE00E94734C63E070E08AE20E943C51AD
:1065E00090E00E942A5141E062E070E08AE20E945D
:1065F0006951992091F080919713882371F067E495
:1066000079E08EE09FE00E94734C62E070E08AE2E5
:106610000E943C5190E00E942A5140E062E070E00C
:106620008AE20E946951992091F080919713882302
:1066300071F06AE279E08EE09FE00E94734C62E0C4
:1066400070E08AE20E943C5190E00E942A5141E0B1
:1066500061E070E08AE20E946951992091F0809196
:106660009713882371F06EE079E08EE09FE00E943E
:10667000734C61E070E08AE20E943C5190E00E941D
:106680002A5140E061E070E08AE20E94695199205D
:1066900091F080919713882371F061EF78E08EE09C
:1066A0009FE00E94734C61E070E08AE20E943C51DE
:1066B00090E00E942A5141E060E070E08AE20E948E
:1066C0006951992091F080919713882371F065EDBD
:1066D00078E08EE09FE00E94734C60E070E08AE218
:1066E0000E943C5190E00E942A5140E060E070E03E
:1066F0008AE20E946951992091F080919713882332
:1067000071F068EB78E08EE09FE00E94734C60E0EF
:1067100070E08AE20E943C5190E00E942A5141E0E0
:1067200066E070E087E20E94695141E065E070E058
:1067300087E20E94695141E064E070E087E20E94D4
:10674000695140E062E070E087E20E94695140E0F8
:1067500061E070E087E20E94695140E060E070E033
:1067600087E20E946951992009F475C080919713BE
:10677000882309F470C060EA78E08EE09FE00E9410
:10678000734C66E070E08BE20E943C5190E00E9406
:106790002A5162E878E08EE09FE00E94734C65E049
:1067A00070E08BE20E943C5190E00E942A5164E626
:1067B00078E08EE09FE00E94734C64E070E08BE232
:1067C0000E943C5190E00E942A516BE478E08EE0F8
:1067D0009FE00E94734C62E070E08BE20E943C51AB
:1067E00090E00E942A5162E378E08EE09FE00E94F0
:1067F000734C61E070E08BE20E943C5190E00E949B
:106800002A5169E178E08EE09FE00E94734C60E0DD
:1068100070E08BE20E943C5190E00E942A5166E0B9
:1068200078E08EE09FE00E94734C63E070E08BE2C2
:106830000E943C5190E00E942A5161EF77E08EE087
:106840009FE00E94734C64E070E08CE20E943C5137
:1068500090E00E942A5140E064E070E08CE20E94E7
:106860006951AE014B5D5F4F61E070E08CE20E94C8
:10687000F1506DA1607F66608CE20E9456519920B4
:1068800009F45FC080919713882309F45AC06DED15
:1068900077E08EE09FE00E94734CAE014B5D5F4F4E
:1068A00061E070E08CE20E94F1506DA16F7070E0C9
:1068B00066507109072E000C880B990B0E94B4AE2C
:1068C0009B01AC0160E070E080E090E40E94ACB21B
:1068D00020E030E048EC50E40E9413AF0E94B45135
:1068E00066EC77E08EE09FE00E94734CAE014B5D5A
:1068F0005F4F61E070E080E30E94F1506DA14AE0DB
:1069000050E08EE09FE00E9499516EEA77E08EE0C1
:106910009FE00E94734C61E070E080E30E943C5174
:1069200090E00E942A5165E977E08EE09FE00E94A6
:10693000734C61E070E08FE20E943C5190E00E9455
:106940002A5141E061E070E08FE20E946951992094
:1069500091F080919713882371F06DE777E08EE0D6
:106960009FE00E94734C61E070E08EE20E943C5117
:1069700090E00E942A5141E061E070E08EE20E94C6
:10698000695140E067E070E081E30E94695199201D
:1069900009F455C080919713882309F450C06AE622
:1069A00077E08EE09FE00E94734C67E070E081E347
:1069B0000E943C5190E00E942A516AE178E08EE00A
:1069C0009FE00E943E4DAE014B5D5F4F61E070E085
:1069D00080E00E94F1508DA10E943E586FEB79E05B
:1069E0008EE09FE00E945F6A0DE110E06DE976E0C5
:1069F0008EE09FE00E943E4D40E150E0B8018EE005
:106A00009FE00E94F44C6EE178E08EE09FE00E94EF
:106A10003E4DAE014B5D5F4F61E070E0802F0E9404
:106A2000F1508DA10E943E586FEB79E08EE09FE01F
:106A30000E945F6A0F5F1F4F0A331105B9F6A996CE
:106A40000FB6F894DEBF0FBECDBFDF91CF911F917F
:106A50000F91FF90EF90DF90CF90BF90AF909F90FD
:106A60007F906F905F904F9008954F925F926F92DA
:106A70007F929F92AF92BF92CF92DF92EF92FF925E
:106A80000F931F93CF93DF93CDB7DEB7A8970FB6C1
:106A9000F894DEBF0FBECDBF6CE372E186E392E1F6
:106AA0000E948E4B0E942A856EE478E0CE0101960A
:106AB0000E94074CBE016F5F7F4F86E392E10E9408
:106AC0000F85182FCE0101960E94A34B112309F4C4
:106AD000E6C08091401290914112409718F080E0FA
:106AE0000C94763E42E050E06CE372E1CE010196F8
:106AF0000E94D83EBE016F5F7F4F88E192E10E9405
:106B0000C04ACE0101960E94A34B68E172E1CE011A
:106B100001960E94FF4BCE0101960E94988FCE01F4
:106B200001960E94A34B88E192E10E94E34920E094
:106B300030E048EC52E40E9413AF0E949DB1AB01DB
:106B4000BC0140934302509344026093450270930A
:106B50004602CE0101960E94326ACE0101960E9441
:106B6000988FCE0101960E94A34B609143027091D1
:106B7000440280914502909146028B019C0100598C
:106B80001F452140310901341C4921053105D0F050
:106B900061E278E0CE0101960E94074C68E172E163
:106BA000CE0101960E94234B64E378E00E940C4BD7
:106BB000BC018EE192E10E948E4BCE0101960E94B3
:106BC000A34B4EC01A821982FE01339626E0DF01E4
:106BD0001D922A95E9F70E94B4AE20E030E048EC1F
:106BE00052E40E9404B18E010F5F1F4F22E047E084
:106BF0000E941EAABC018EE192E10E94794B64E4DE
:106C000078E0CE0145960E94074C6EE172E1CE011C
:106C100045960E94234B61E578E00E940C4BBC0135
:106C20008EE192E10E948E4BCE0145960E94A34BCD
:106C30001092380C1092370C8091430290914402CC
:106C4000A0914502B09146028093891090938A10DA
:106C5000A0938B10B0938C1080E090E00E94346E73
:106C600061E179E0CE0101960E94074C6EE172E18C
:106C7000CE0101960E94234BBC01CE0145960E9495
:106C8000FF4BCE0145960E94BB70CE0145960E94F7
:106C9000A34BCE0101960E94A34B0C94733E66E574
:106CA00078E0CE0101960E94074CBE016F5F7F4FD6
:106CB00086E392E10E940F85182FCE0101960E9473
:106CC000A34B1123C1F126E030E044E050E06CE337
:106CD00072E1CE0101960E941B4CBE016F5F7F4F97
:106CE00088E192E10E94C04ACE0101960E94A34B26
:106CF00088E192E10E94EE497093021160930111C4
:106D000070932A02609329026CE372E1CE0101962E
:106D10000E94FF4BCE0101960E94988FCE010196F2
:106D20000E94A34B1092380C1092370C80E090E038
:106D30000E94346ED8C76BE578E0CE0101960E94C0
:106D4000074CBE016F5F7F4F86E392E10E940F8583
:106D5000182FCE0101960E94A34B112309F4C3C042
:106D60006EE578E0CE0101960E94074CBE016F5F90
:106D70007F4F86E392E10E940F85182FCE01019686
:106D80000E94A34B1123D1F184E090E00E94347E55
:106D900060931D0270931E0280931F029093200245
:106DA00060EC7CE08EE192E10E94344B40911D0248
:106DB00050911E0260911F027091200222E0CE01CC
:106DC00001960E94A84BBE016F5F7F4F8EE192E15A
:106DD0000E94BA4ACE0101960E94A34B80911D02E7
:106DE00090911E02A0911F02B09120028093AD10DD
:106DF0009093AE10A093AF10B093B01062E678E01D
:106E0000CE0101960E94074CBE016F5F7F4F86E363
:106E100092E10E940F85182FCE0101960E94A34B8C
:106E2000112309F442C08AE090E00E94347E60930E
:106E3000190270931A0280931B0290931C026FEA4E
:106E40007CE08EE192E10E94344B40911902509116
:106E50001A0260911B0270911C0222E0CE01019681
:106E60000E94A84BBE016F5F7F4F8EE192E10E94AE
:106E7000BA4ACE0101960E94A34B809119029091CB
:106E80001A02A0911B02B0911C028093B110909342
:106E9000B210A093B310B093B4101092380C1092AB
:106EA000370C80E090E00E94346E61E179E0CE0121
:106EB00001960E94074C6EE172E1CE0101960E949C
:106EC000234BBC01CE0145960E94FF4BCE01459657
:106ED0000E94BB70CE0145960E94A34BCE01019645
:106EE0000E94A34B02C767E678E0CE0101960E949C
:106EF000074CBE016F5F7F4F86E392E10E940F85D2
:106F0000182FCE0101960E94A34B112309F4B8C09B
:106F100080914012909141120797F0F046E050E0C6
:106F20006CE372E1CE01019643D7BE016F5F7F4FE4
:106F300088E192E10E94C04ACE0101960E94A34BD3
:106F400088E192E10E94E349609325027093260252
:106F5000809327029093280280915F0290916002B3
:106F600099270E9464782DE038E643E55BE30E94B0
:106F700013AF6B017C01209181023091820240911C
:106F80008302509184020E94AEAE18164CF06091BC
:106F9000690270916A0280916B0290916C021BC031
:106FA000209195023091960240919702509198025B
:106FB000C701B6010E94F3B187FF05C0C701B60142
:106FC0000E94A26C08C060917D0270917E02809147
:106FD0007F029091800220E030E048EC52E40E9471
:106FE00013AF6B017C0120E030E0A9010E94AEAE3E
:106FF000181634F0C12CD12C38EAE32E31E4F32EEC
:10700000C0922502D0922602E0922702F092280236
:10701000C092BD10D092BE10E092BF10F092C0108E
:1070200080919713882381F06DE97CE08EE09FE0EA
:107030000E94734C60912502709126028091270274
:10704000909128020E94B4511092380C1092370C83
:1070500080E090E00E94346E63E97CE08EE192E192
:107060000E94344B409125025091260260912702E4
:107070007091280222E0CE0101960E94A84B43C2E3
:107080006DE678E0CE0101960E94074CBE016F5F6D
:107090007F4F86E392E10E940F85182FCE01019663
:1070A0000E94A34B112309F46EC0B0905D0260E012
:1070B0008B2D0E94AE8509E110E0C12CD12C760108
:1070C0008B2D0E94EA85BC01990F880B990B0E94B9
:1070D000B4AE9B01AC01C701B6010E943EB06B018A
:1070E0007C016AE070E080E090E00E94348601500C
:1070F000110931F720E030E040EA50E4C701B60161
:107100000E9413AF20E030EC4FE754E40E9404B13A
:1071100020E030E048EC51E40E9404B16093210289
:107120007093220280932302909324026093D310E1
:107130007093D4108093D5109093D6101092380C81
:107140001092370C80E090E00E94346E60E87CE0A2
:107150008EE192E10E94344B409121025091220233
:10716000609123027091240222E0CE0101960E94D8
:10717000A84BBE016F5F7F4FCE0145960E94FF4B2B
:107180006DEC75E054C061E778E0CE0101960E9495
:10719000074CBE016F5F7F4F86E392E10E940F852F
:1071A000182FCE0101960E94A34B112309F454C05D
:1071B0008091B810082E000C990B0197039708F0E6
:1071C00044C089E390E00E9464782AE137E64CE904
:1071D00050E40E9413AF6093B9107093BA1080937B
:1071E000BB109093BC101092380C1092370C80E0BA
:1071F00090E00E94346E6FE57CE08EE192E10E94A7
:10720000344B4091B9105091BA106091BB107091FD
:10721000BC1022E0CE0101960E94A84BBE016F5F18
:107220007F4FCE0145960E94FF4B67E778E0CE0185
:1072300045960E940C4BBC018EE192E10E94BA4A35
:10724000CE0145960E94A34B65C169E37CE08EE1C7
:1072500092E10E94344B39C56AE778E0CE0101968D
:107260000E94074CBE016F5F7F4F86E392E10E9450
:107270000F85182FCE0101960E94A34B112309F40C
:107280004CC126E030E044E050E06CE372E1CE0116
:1072900001960E941B4CBE016F5F7F4F88E192E117
:1072A0000E94C04ACE0101960E94A34B88E192E160
:1072B0000E94EE496B017C015B0164ED7AE0CE0136
:1072C00001960E94074CBE016F5F7F4F8CE392E1F5
:1072D0000E94BF848E010B5E1F4FAC014F5F5F4F5A
:1072E0006CE372E1C80164D5B80188E192E10E94C3
:1072F000C04AC8010E94A34BCE0101960E94A34B35
:1073000090905B0288E192E10E94E3492B013C01ED
:10731000809197138823B9F062E57BE08EE09FE0CF
:107320000E94734C4AE050E0B6018EE09FE00E945C
:10733000F44C68ED7BE08EE09FE00E943E4DC3017F
:10734000B2010E94B451692DC8010E94E556188708
:107350000F831D821E82198289E08A8381E08B83DC
:107360008C831C8A1B8ACE0101960E94F253CE01A7
:1073700001960E948653CE0101960E94B7520E815B
:1073800010E00B30110514F00AE010E0BBE5CB165D
:10739000D10408F44CC02FE0C22E2CE0D22E5601AE
:1073A000412C512C3201E12CF12CE016F106BCF4F9
:1073B0006E2DCE0101960E9448529B01AC01F50151
:1073C00061937193819391935F01C301B2010E9414
:1073D0003EB02B013C01FFEFEF1AFF0AE6CFB801E8
:1073E000012E000C880B990B0E94B4AE9B01AC01DE
:1073F000C301B2010E9404B12B013C01E12CF12C2C
:10740000E016F1060CF05AC0D6012D913D914D9138
:107410005C91C301B2010E943DB0F601619371938A
:10742000819391936F01FFEFEF1AFF0AE9CF1A14CE
:107430001B0424F50A151B0524F041E0C41AD108E9
:1074400004C0680181E0C81AD1086C2DCE010196F4
:107450000E9448529B01AC018601000F111F000FD2
:10746000111F015F134FC301B2010E943DB0D8014B
:107470006D937D938D939C93139720C0AB28F1F46B
:107480008FE0C82E8CE0D82EE12CF12CE016F1060E
:10749000ACF46E2DCE0101960E9448529B01AC01C6
:1074A000C301B2010E943DB0F601619371938193D3
:1074B00091936F01FFEFEF1AFF0AE8CFEFE0FCE0D6
:1074C000A7EDB0E141915191619171914D935D931F
:1074D0006D937D934CE0E733F407A1F71092380CDD
:1074E0001092370C80E090E00E94346E68E17CE0FE
:1074F0008EE192E10E94344B44E050E06CE372E193
:10750000CE01019655D4BE016F5F7F4F8EE192E1AF
:107510000E94BA4ACE010196D6C36EE778E0CE014A
:1075200001960E94074CBE016F5F7F4F86E392E198
:107530000E940F85182FCE0101960E94A34B1123A4
:1075400009F424C127E030E046E050E06CE372E14A
:10755000CE0101960E941B4CBE016F5F7F4F88E1F8
:1075600092E10E94C04ACE0101960E94A34B88E19D
:1075700092E10E94EE498B016093B8108CE392E196
:107580000E94F94968ED7BE0CE0101960E94074C0C
:10759000BE016F5F7F4F8CE392E10E94BF84AC011C
:1075A0004F5F5F4F6CE372E1CE01459601D4CE018F
:1075B00045960E94E3496093B9107093BA10809386
:1075C000BB109093BC10CE0145960E94A34BCE01F8
:1075D00001960E94A34B67E07CE08EE192E10E945D
:1075E000344B0430110594F4023011050CF05BC0EB
:1075F00001151105B1F00130110509F09BC069EFCB
:107600007BE08EE192E10E946A4A77C00430110566
:1076100009F090C066EE7BE08EE192E10E946A4A3A
:10762000ACC020E030E0A9016091B9107091BA10AF
:107630008091BB109091BC100E94AEAE181664F001
:1076400080E090E0A0E8BFE38093B9109093BA1077
:10765000A093BB10B093BC102091B9103091BA1018
:107660004091BB105091BC1060E070E080EA90E463
:107670000E9404B1AB01BC0122E0CE0145960E94FC
:10768000A84B65E878E0CE0101960E94074CBE0148
:107690006B5E7F4FCE0101960E94234B64ED78E034
:1076A0000E940C4B5DC06DEE7BE08EE192E10E948A
:1076B0006A4A8AE0809FB001819F700D1124CE013B
:1076C00001960E942D50BE016F5F7F4FCE014596FF
:1076D0000E94FF4B6DEC78E0CE0145960E940C4B6A
:1076E000BC018EE192E10E94BA4ACE0145960E9409
:1076F000A34BCE0101960E94A34B20E030E048E46A
:1077000053E46091B9107091BA108091BB109091C0
:10771000BC100E94AEAE181684F180E090E4ACE19B
:10772000B5E48093B9109093BA10A093BB10B093B6
:10773000BC1023C06091B810062E000C770BCE0150
:1077400045960E942D5060E978E0CE0101960E9496
:10775000074CBE016B5E7F4FCE0101960E94234B0A
:10776000BC018EE192E10E94BA4ACE0101960E94CC
:10777000A34BCE0145960E94A34B1092380C109259
:10778000370C80E090E00E94346E9FC267E978E099
:10779000CE0101960E94074CBE016F5F7F4F86E3CA
:1077A00092E10E940F85182FCE0101960E94A34BF3
:1077B000112309F4CEC027E030E046E050E06CE34E
:1077C00072E1CE0101960E941B4CBE016F5F7F4F9C
:1077D00088E192E10E94C04ACE0101960E94A34B2B
:1077E00088E192E10E94EE496093B5108CE392E14A
:1077F0000E94F94988E192E10E94EE496115710504
:107800008105910519F485E090E007C061307105AC
:107810008105910539F489E190E09093B710809348
:10782000B61025C068ED7BE0CE0101960E94074CA2
:10783000BE016F5F7F4F8CE392E10E94BF84AC0179
:107840004F5F5F4F6CE372E1CE014596B1D2CE013E
:1078500045960E94EE497093B7106093B610CE0122
:1078600045960E94A34BCE0101960E94A34B109215
:10787000380C1092370C80E090E00E94346E65ED79
:107880007BE08EE192E10E94344B8091B510833011
:1078900044F56AEC7BE08EE192E10E946A4A6091D5
:1078A000B6107091B710CE0101960E942D50BE0106
:1078B0006F5F7F4FCE0145960E94FF4B62EB7BE0EE
:1078C000CE0145960E940C4BBC018EE192E10E94D4
:1078D000BA4ACE0145960E94A34BCE0101960E9462
:1078E000A34B8091B51083300CF4EFC16091B610BA
:1078F0007091B710CE0183960E942D506091B51003
:10790000062E000C770BCE0145960E942D5060E9A3
:1079100078E0CE0101960E94074CBE016B5E7F4F5E
:10792000CE0101960E94234BBE016D5D7F4F0E94E8
:10793000234BBC018EE192E10E94BA4ACE0101962E
:107940000E94A34BCE0145960E94A34BCE01839685
:10795000BAC16EE978E0CE0101960E94074CBE01E3
:107960006F5F7F4F86E392E10E940F85182FCE0153
:1079700001960E94A34B112309F456C0809159022D
:1079800090915A020E94757960932B0270932C0299
:1079900080932D0290932E026093A1107093A210F9
:1079A0008093A3109093A41080E090E5A3ECB7E43B
:1079B0008093330290933402A0933502B093360241
:1079C0008093991090939A10A0939B10B0939C1061
:1079D00080919713882381F06CEA7BE08EE09FE032
:1079E0000E94734C60912B0270912C0280912D02A9
:1079F00090912E020E94B4511092380C1092370CC4
:107A000080E090E00E94346E40912B0250912C0255
:107A100060912D0270912E0222E0CE0145960E94C7
:107A2000A84B62EA78E039C16DEA78E0CE010196B0
:107A30000E94074CBE016F5F7F4F86E392E10E9478
:107A40000F85182FCE0101960E94A34B112309F434
:107A500084C080914012909141120497F0F044E06C
:107A600050E06CE372E1CE010196A2D1BE016F5FDE
:107A70007F4F88E192E10E94C04ACE0101960E94A8
:107A8000A34B88E192E10E94E3496093370270932F
:107A900038028093390290933A0280913702909194
:107AA0003802A0913902B0913A02809395109093D8
:107AB0009610A0939710B0939810809197138823F5
:107AC00089F063E97BE08EE09FE00E94734C609157
:107AD0003702709138028091390290913A0242E067
:107AE0000E94A36A8091590290915A020E9475796E
:107AF00060932F0270933002809331029093320290
:107B000060939D1070939E1080939F109093A0108F
:107B100080919713882381F069E87BE08EE09FE0F5
:107B20000E94734C60912F0270913002809131025B
:107B3000909132020E94B4511092380C1092370C7E
:107B400080E090E00E94346E40912F02509130020C
:107B5000609131027091320299C069EB78E0CE01F8
:107B600001960E94074CBE016F5F7F4F86E392E152
:107B70000E940F85182FCE0101960E94A34B11235E
:107B800011F40C946F35809140129091411204973A
:107B9000F0F044E050E06CE372E1CE01019608D1D0
:107BA000BE016F5F7F4F88E192E10E94C04ACE0123
:107BB00001960E94A34B88E192E10E94E349609301
:107BC0003302709334028093350290933602809191
:107BD000330290913402A0913502B0913602809325
:107BE000991090939A10A0939B10B0939C10809141
:107BF0009713882389F060E77BE08EE09FE00E9486
:107C0000734C6091330270913402809135029091EF
:107C1000360242E00E94A36A8091590290915A0272
:107C20000E94757960932B0270932C0280932D0231
:107C300090932E026093A1107093A2108093A310D2
:107C40009093A41080919713882381F066E67BE0DF
:107C50008EE09FE00E94734C60912B0270912C0289
:107C600080912D0290912E020E94B4511092380CF6
:107C70001092370C80E090E00E94346E40912B020D
:107C800050912C0260912D0270912E0222E0CE01C3
:107C900045960E94A84B61EB78E0CE0101960E94C8
:107CA000074CBE016B5E7F4FCE0101960E94234BB5
:107CB000BC018EE192E10E948E4BCE0101960E94A2
:107CC000A34BCE0145960E94A34B6EE172E1CE011B
:107CD00001960E94FF4BCE0101960E94BB70CE011F
:107CE00001960E94A34B1092540281E0A8960FB611
:107CF000F894DEBF0FBECDBFDF91CF911F910F91E2
:107D0000FF90EF90DF90CF90BF90AF909F907F90CB
:107D10006F905F904F900895089580912E0588236D
:107D2000F9F080912D058823D9F081E00E94F66951
:107D30008BE39FE10197F1F760E080E00E94076A22
:107D40006CE97DE08FE193E10E94734C61E080E09B
:107D50000E94076A6CE87DE08FE193E10C94734C1C
:107D6000089580912E05882349F080912D05882360
:107D700029F060E08FE193E10C9439570895FF9268
:107D80000F931F93CF93DF93EC01F62E0881198197
:107D9000C8010E94CAAFF81621F06F2DC8010E94D9
:107DA000D2AFCE01DF91CF911F910F91FF90089537
:107DB000CF93DF93EC01FB01248135810E941B4CA2
:107DC000CE01DF91CF9108953F924F925F926F92D3
:107DD0007F928F929F92AF92BF92CF92DF92EF925B
:107DE000FF920F931F93CF93DF93CDB7DEB7E49746
:107DF0000FB6F894DEBF0FBECDBF80914413882329
:107E000019F0109244134CC381E0809344136FEB3C
:107E100079E0CE0185960E94074C6FEB79E0CE01A8
:107E20008B960E94074C00E010E082E0382E98EE1E
:107E3000C92E93E0D92EE12CF12CF8013197E031D5
:107E4000F10530F48827E856FF4F8F4F0C9478B334
:107E50006FEB79E0CE0185960E94794B8091FF10FF
:107E600090910011892B31F469E077E0CE0185967D
:107E70000E94794B8091FF1090910011019731F48D
:107E80006DE077E0CE0185960E94794B8091FF10DE
:107E900090910011029731F463E177E0CE0185966D
:107EA0000E94794B89A59AA5892B31F063E173E192
:107EB000CE0185960E94BA4A6DEB78E0CE0101961C
:107EC0000E94074C6DE073E1CE0101960E94234BA6
:107ED000BC01CE018B960E948E4BCE0101960E9472
:107EE000A34B8091FF1090910011019709F03BC2C4
:107EF000BE016B5D7F4FCE0101960E94FF4B48ECA7
:107F000050E06FEF7FEFCE0101960E94C48FCE014B
:107F100001960E94A34BBE01655D7F4FCE01019685
:107F20000E94FF4B40ED57E06FEF7FEFCE010196CF
:107F30000E947C8DCE0101960E94A34BCE0101963A
:107F40000E947A608D819E810097A1F0E981FA817B
:107F50002081222379F0079768F065E77FE0CE0162
:107F600085960E94344BBE016F5F7F4FCE018B968A
:107F70000E948E4BCE01019696C069E67FE0CE014D
:107F800085960E94344B0E9490874B015C010E94B1
:107F90009087A70196010E940CB0CA01B90120E8A0
:107FA00031E541E050E00E940CB020E13EE040E0CD
:107FB00050E00E94E0AF29AB3AAB4BAB5CAB2CE39B
:107FC00030E040E050E00E94E0AF29013A01AB010F
:107FD000BC01CE0101960E94326AB301A201CE011A
:107FE00007960E94326A49A95AA96BA97CA9CE01B9
:107FF0000D960E94326AC501B40120E03CE546E2DC
:1080000055E00E940CB0BA01A901CE0149960E9428
:10801000326ABE01675E7F4FCE0143960E94FF4BDE
:1080200062EC78E0CE0143960E940C4BBE01635F88
:108030007F4F0E94234B65EC78E00E940C4BBE0101
:10804000695F7F4F0E94234B68EC78E00E940C4BE5
:10805000BE016F5F7F4F0E94234B6BED75E00E9466
:108060000C4BBC01CE014F960E94FF4BCE014396B4
:108070000E94A34BCE0149960E94A34BCE010D96C0
:108080000E94A34BCE0107960E94A34BCE010196FE
:108090000E94A34BBE01615E7F4FCE018B960E9472
:1080A000C04ACE014F960E94A34B5DC180910D0C3A
:1080B00090910E0C019719F46AE57FE002C06CE420
:1080C0007FE0CE0185960E94344B6CE37FE047C190
:1080D0006CE27FE0CE0185960E94344B6FE17FE039
:1080E0003EC162E17FE0CE0185960E94344B67E09D
:1080F0007FE035C16BEF7EE0CE0185960E94344B68
:108100006AEE7EE02CC180910D0C90910E0C0397CD
:1081100019F46FED7EE002C065ED7EE0CE0185963C
:108120000E94344B6AEC7EE01AC16DEB7EE0CE011A
:1081300085960E94344B6EEA7EE011C163EA7EE0D0
:10814000CE0185960E94344B6091B6107091B710A5
:10815000CE0107960E942D5061EE7BE0CE01019684
:108160000E94074CBE01695F7F4FCE0101960E94BD
:10817000234B62EB7BE00E940C4BBC01CE01859649
:108180000E94BA4ACE0101960E94A34BCE010796E7
:108190000E94A34B66E97EE0E2C080910D0C9091B5
:1081A0000E0C029719F465E87EE002C065E77EE0F8
:1081B000CE0185960E94344B68E67EE0D0C06CE527
:1081C0007EE0CE0185960E94344B6CE47EE0C7C011
:1081D00061E47EE0CE0185960E94344B67E37EE049
:1081E000BEC06BE27EE0CE0185960E94344B6BE10F
:1081F0007EE0B5C0B090B81060E17EE0CE0185961B
:108200000E94344B83E08B1574F092E0B9160CF0A9
:1082100045C0BB2081F081E0B81261C06BEC78E012
:10822000CE01859659C094E0B91259C06FEC78E040
:108230008EE192E151C08090B9109090BA10A09058
:10824000BB10B090BC1020E030E048E452E4C5011F
:10825000B4010E94AEAE87FF02C033243394A5015F
:10826000940160E070E080EA90E40E9404B1AB0108
:10827000BC01232DCE0107960E94A84B69EF78E040
:10828000CE0101960E94074CBE01695F7F4FCE016F
:1082900001960E94234B64ED78E018C08B2D9AE084
:1082A0008902B0011124CE0107960E942D5061EE83
:1082B0007BE0CE0101960E94074CBE01695F7F4FB3
:1082C000CE0101960E94234B6DEC78E00E940C4B8E
:1082D000BC01CE0185961CC00E94AC4A23C06091AF
:1082E000B810062E000C770BCE0107960E942D5079
:1082F00067E97AE0CE0101960E94074CBE01695FF2
:108300007F4FCE0101960E94234BBC018EE192E18A
:108310000E94BA4ACE0101960E94A34BCE01079655
:108320000E94A34B60E07EE01AC063EF7DE0CE01C7
:1083300085960E94344B63EE7DE011C067ED7DE0D1
:10834000CE0185960E94344B68EC7DE008C06CEB52
:108350007DE0CE0185960E94344B6CEA7DE0CE0133
:108360008B960E94344BBE016B5D7F4FCE01019610
:108370000E94FF4B48EC50E06FEF7FEFCE0101967B
:108380000E946990CE0101960E94A34BBE01655DDB
:108390007F4FCE0101960E94FF4B48EC50E06FEFFB
:1083A0007FEFCE0101960E947C8DCE0101960E9446
:1083B000A34B0E940398982EA12CB12C91106DC054
:1083C0008FEFA81AB80A95E6A916B10451F00E94D9
:1083D0000398982E64E170E080E090E00E9434867B
:1083E000EDCF6FEB79E08CE392E10E94794BCE0107
:1083F00001960E942274BE016F5F7F4F8CE392E171
:108400000E94C04ACE0101960E94A34B8091401267
:1084100090914112892B89F461E070E0CE010196C0
:108420000E94388BBE016F5F7F4F8CE392E10E9408
:10843000C04ACE0101960E94A34B809140129091B8
:108440004112892B89F461E070E0CE0101960E940F
:10845000D689BE016F5F7F4F8CE392E10E94C04AD4
:10846000CE0101960E94A34B80914012909141123F
:10847000892B51F480914413882331F00F5F1F4FF3
:108480000131110509F0D9CCCE018B960E94A34B86
:10849000CE0185960E94A34B03C010924413F4CFE3
:1084A000E4960FB6F894DEBF0FBECDBFDF91CF913B
:1084B0001F910F91FF90EF90DF90CF90BF90AF9002
:1084C0009F908F907F906F905F904F903F90089516
:1084D0004F925F926F927F928F929F92AF92BF92D4
:1084E000CF92DF92EF92FF920F931F93CF93DF9380
:1084F000CDB7DEB7C654D1090FB6F894DEBF0FBEB4
:10850000CDBF8C016FEB79E0CE01C7960E94074C7E
:108510006FEB79E0CE01CD960E94074CBE016F5FF4
:108520007F4F89E592E154D68D889E88AF88B88CBC
:10853000498C5A8C6B8C7C8C8D8D9E8DAF8DB8A1A7
:1085400027968CAF9DAFAEAFBFAF2797C8010197FD
:10855000039708F0ADC1A3019201C501B401905881
:108560000E94B1B02BED3FE049EC5FE30E943EB0CA
:1085700020913F02309140024091410250914202CD
:108580000E943EB06B017C0120E030E0A9010E9416
:10859000AEAE87FD09C0C0924C0CD0924D0CE0925B
:1085A0004E0CF0924F0C10C02BED3FE049EC50E424
:1085B000C701B6010E943EB060934C0C70934D0C05
:1085C00080934E0C90934F0CC0904C0CD0904D0C5F
:1085D000E0904E0CF0904F0C2BED3FE049EC50E456
:1085E000C701B6010E94F3B1181684F42BED3FE0E9
:1085F00049EC50E4C701B6010E943DB060934C0CB9
:1086000070934D0C80934E0C90934F0C20E030E013
:1086100044E353E460914C0C70914D0C80914E0CEE
:1086200090914F0C0E9413AF2BED3FE049E450E4D2
:108630000E9404B16093480C7093490C80934A0CDB
:1086400090934B0C0E949DB1CE018B960E942D50B1
:1086500067ED78E0CE0185960E94074CBE01655D0E
:108660007F4FCE018596EFD761EE78E0D5D7BC017C
:1086700084E292E10E948E4BCE0185960E94A34B2C
:10868000CE018B960E94A34BC090480CD090490C11
:10869000E0904A0CF0904B0C20E030E044EB52E4C8
:1086A000C701B6010E94AEAE18168CF020E030E093
:1086B00040E05FE3C701B6010E943EB00E949DB159
:1086C000CE018B960E942D5068EE78E022C020E00B
:1086D00030E044E353E4C701B6010E94AEAE181681
:1086E0008CF1A701960160E070E884E393E40E94B6
:1086F0003DB06093480C7093490C80934A0C909362
:108700004B0C0E949DB1CE018B960E942D506BEEBA
:1087100078E0CE0185960E94074CBE01655D7F4FD3
:10872000CE01859690D7BC01CE01C796F7D7CE0172
:1087300085960E94A34BCE018B960E94A34B6AE2C2
:108740007BE05DC020E030E047E853E4C701B601BC
:108750000E94AEAE1816FCF020E030E044E353E493
:10876000C701B6010E943DB020E030E040E05FE389
:108770000E943EB06093480C7093490C80934A0C61
:1087800090934B0C0E949DB1CE018B960E942D5070
:108790006BEE78E01EC0A701960160E070E084EB0C
:1087A00093E40E943DB020E030E040E05FE30E94AF
:1087B0003EB06093480C7093490C80934A0C9093A0
:1087C0004B0C0E949DB1CE018B960E942D5068EEFD
:1087D00078E0CE0185960E94074CBE01655D7F4F13
:1087E000CE01859630D7BC01CE01C79697D7CE0172
:1087F0008596A9D7CE018B96A6D76EEE78E0CE01EE
:10880000CD9677D7BE01695C7F4FCE018596F7D7AD
:108810004AE050E060E070E0CE0185960E94C48F8F
:10882000CE01859690D70E949087C0909313D090E8
:108830009413E0909513F0909613A4E6CA0ED11C01
:10884000E11CF11CC616D706E806F90608F4E7C1D4
:108850000E9490870E94B2AE6B017C0160919313DD
:108860007091941380919513909196130E94B4AED9
:1088700020E030E048EC51E40E943EB09B01AC01A6
:10888000C701B6010E94AEAE87FDC9C168ED7BE0AD
:10889000CE018596BCD7BE01635C7F4FCE01859625
:1088A000D2D6BC01CE01C79665D6CE0185964BD7F0
:1088B000C8010297029708F08EC120E030E040E244
:1088C00051E4C501B4010E9413AF6B017C0120E0AB
:1088D00030E040E251E4C301B2010E9413AF4B010A
:1088E0005C0120E030E040E251E427966CAD7DADC4
:1088F0008EAD9FAD27970E9413AF2B013C010E94C4
:1089000090872091EA0B3091EB0B4091EC0B50914A
:10891000ED0B621B730B840B950B0E94B2AE20E033
:1089200030E04AE754E40E9404B1AB01BC0123E00B
:10893000CE018B960DD769EF78E0CE01859667D78B
:10894000BE01655D7F4FCE0185967DD66EEF7AE0E4
:1089500063D6BC0182E192E1E1D6CE018596F3D6E1
:10896000CE018B96F0D662E172E1CE01859647D7B3
:1089700064E272E1CE01859666D6BE01695C7F4FE6
:1089800062D6BC01CE01C796C9D6CE018596DBD68C
:1089900061E87DE08EE192E167D621E0B701A601B2
:1089A000CE018596D5D6BE016B5D7F4F8EE192E1FB
:1089B000E1D5CE018596C7D621E0B301A201CE0153
:1089C000C196C6D621E0B501A401CE018B96C0D6D2
:1089D00068ED7BE0CE0185961AD7BE01655D7F4FBD
:1089E000CE01859630D668ED7BE016D6BE016F5C71
:1089F0007F4F29D660EF78E00FD6BC018EE192E17F
:108A0000B9D5CE0185969FD6CE018B969CD6CE0148
:108A1000C19699D6A7019601C701B6010E9413AF6E
:108A20006B017C01A5019401C501B4010E9413AF43
:108A30009B01AC01C701B6010E943EB06B017C01F5
:108A4000A3019201C301B2010E9413AF9B01AC01CB
:108A5000C701B6010E943EB00E94FCB26B017C01CE
:108A60006093440C7093450C8093460C9093470C94
:108A700064EF78E08EE192E16FD521E0B701A601C5
:108A8000CE01859665D6BE016B5D7F4FCE018B967C
:108A9000B6D665E079E0CE018B96BED5BC0184E206
:108AA00092E13CD6CE018B964ED6CE0185964BD622
:108AB00064E272E18EE192E15DD5C090440CD09009
:108AC000450CE090460CF090470C20E030E04AE77F
:108AD00054E4C701B6010E94F3B187FD23C020E032
:108AE00030E04AE754E4C701B6010E9404B1AB018B
:108AF000BC0123E0CE0185962BD6BE016B5D7F4F76
:108B0000CE018B967CD666E079E0CE018B9684D53B
:108B1000BC0184E292E102D6CE018B9614D6CE013E
:108B2000859611D620E030E64AE656E46091440C82
:108B30007091450C8091460C9091470C0E94AEAE0E
:108B4000BE01695C7F4F87FF43C0CE01859657D633
:108B500068EF78E0CE0185965FD56EE172E173D55E
:108B6000BC018EE192E1DAD5CE018596ECD50330D9
:108B7000110589F46EE172E1CE01859640D6CE01F1
:108B800085960E94BB70CE018596DDD56FEB79E0AE
:108B90008EE192E1AED56BEF78E0CE01859637D6C7
:108BA00064E272E1CE0185964ED5BC01CE018B9672
:108BB00026D64AE050E06FEF7FEFCE018B960E9401
:108BC0007C8DCE018B96BFD5CE018596BCD503C0DA
:108BD0008EE192E1A3D56AE070E080E090E00E942F
:108BE0003486CE01CD96AFD5CE01C796ACD5CA5B43
:108BF000DF4F0FB6F894DEBF0FBECDBFDF91CF9130
:108C00001F910F91FF90EF90DF90CF90BF90AF90AA
:108C10009F908F907F906F905F904F9008956FEB33
:108C200079E0CE018596F3D5CE0185960E94F88D28
:108C3000CE01859688D5BE01635C7F4F8FE193E1BD
:108C400044D624CE1F93CF93DF93CDB7DEB7A8973A
:108C50000FB6F894DEBF0FBECDBF182F0E94FB4F9A
:108C60008EE10E94EC6962E08BEA9FE00E94F5557C
:108C700060E08BEA9FE00E94F5550E94E5698EE175
:108C80000E94EC6961E08BEA9FE00E94F55560E28A
:108C90008BEA9FE00E94F5550E94E56980E290E032
:108CA00090935D1280935C1280E090E8A9E8B4E4B0
:108CB0008093650290936602A0936702B093680266
:108CC00080E090E0A5E7B4E48093610290936202B3
:108CD000A0936302B0936402BE016F5F7F4F89E58A
:108CE00092E129D2112309F47CC066E57DE08EE093
:108CF0009FE0F9D58EE09FE00E94746966E47DE014
:108D00008EE09FE0F0D5BE016F5F7F4F8EE09FE069
:108D10000E945F6A66E37DE08EE09FE0E4D56D85AA
:108D20007E858F8598890E94706A66E27DE08EE07C
:108D30009FE0D9D569897A898B899C890E94706A5C
:108D400066E17DE08EE09FE0CED520E030E040E2BD
:108D500051E4698D7A8D8B8D9C8D0E9413AF42E01A
:108D60000E94A36A64E079E08EE09FE00E945F6A5F
:108D700066E07DE08EE09FE0B6D520E030E040E2A6
:108D800051E46D8D7E8D8F8D98A10E9413AF42E0CE
:108D90000E94A36A64E079E08EE09FE00E945F6A2F
:108DA00066EF7CE08EE09FE09ED520E030E040E280
:108DB00051E469A17AA18BA19CA10E9413AF42E06A
:108DC0000E94A36A64E079E08EE09FE00E945F6AFF
:108DD00060ED7CE08EE09FE086D58EE09FE00E9413
:108DE000746964EF71E080E090E00E943486A89698
:108DF0000FB6F894DEBF0FBECDBFDF91CF911F91AC
:108E000008950895CF92DF92EF92FF920F931F93F0
:108E1000CF93DF936C017A018B01C0E0D0E0CE15D7
:108E2000DF0581F0D8016D918D01D601ED91FC91A6
:108E30000190F081E02DC6011995892B11F0219642
:108E4000EECF7E01C701DF91CF911F910F91FF906F
:108E5000EF90DF90CF900895FC01538D448D252F26
:108E600030E0842F90E0821B930B541710F0CF96C4
:108E7000089501970895FC01918D828D981761F0F6
:108E8000828DDF01A80FB11D5D968C91928D9F5F41
:108E90009F73928F90E008958FEF9FEF0895FC01EC
:108EA000918D828D981731F0828DE80FF11D858D9F
:108EB00090E008958FEF9FEF0895FC01918D228D32
:108EC000892F90E0805C9F4F821B91098F739927B7
:108ED000089587E39DE0F1DF21E0892B09F420E08C
:108EE000822F089584ED9DE0E8DF21E0892B09F4CD
:108EF00020E0822F089581E79EE0DFDF21E0892BCB
:108F000009F420E0822F08958EE09FE0D6DF21E073
:108F1000892B09F420E0822F0895FC01848DDF0164
:108F2000A80FB11DA35ABF4F2C91848D90E00196DC
:108F30008F739927848FA689B7892C93A089B189CB
:108F40008C91837080648C93938D848D981306C06C
:108F50000288F389E02D80818F7D80830895EF92D0
:108F6000FF920F931F93CF93DF93EC0181E0888FE3
:108F70009B8D8C8D981305C0E889F989808185FDCA
:108F800025C0F62E0B8D10E00F5F1F4F0F731127BA
:108F9000E02E8C8DE8120BC00FB607FCFACFE889E3
:108FA000F989808185FFF5CFCE01B7DFF2CF8B8DB8
:108FB000FE01E80FF11DE35AFF4FF0829FB7F894CE
:108FC0000B8FEA89FB89808180620AC09FB7F89481
:108FD000EE89FF896083E889F989808183708064E4
:108FE00080839FBF81E090E0DF91CF911F910F912F
:108FF000FF90EF900895CF93DF93EC01888D882345
:10900000C1F0EA89FB89808185FD05C0A889B989FD
:109010008C9186FD0EC00FB607FCF5CF808185FFD1
:10902000F2CFA889B9898C9185FFEDCFCE0175DF8C
:10903000E8CFDF91CF91089580E090E0892B19F07F
:1090400063DF811116C080E090E0892B19F053DFB7
:10905000811112C080E090E0892B19F043DF81116B
:109060000EC080E090E0892B79F033DF81110AC0D7
:1090700008950E940000E7CF0E940000EBCF0E94FD
:109080000000EFCF0C94000008950E94CCB50F9320
:109090001F93CF93DF93EC0188819981009729F08A
:1090A0002A813B812617370788F48B016F5F7F4F3A
:1090B0000E94ECB4009761F0998388831B830A8334
:1090C0002C813D81232B11F4FC01108281E001C031
:1090D00080E0DF91CF911F910F910895EF92FF9261
:1090E0000F931F93CF93DF936115710511F480E007
:1090F0001BC041155105B9F07B01EC018C819D81AC
:109100008A01080F191FB801CE01C1DF882379F346
:10911000288139818C819D81B701820F931F0E9424
:1091200003B61D830C8381E0DF91CF911F910F91D6
:10913000FF90EF9008950F931F93CF93DF938C01CF
:10914000EB0188E2FB0111928A95E9F74BE050E0D0
:1091500068E079E0CE010E9418B61B8681E090E0BD
:10916000A0E0B0E08C879D87AE87BF87F801858936
:109170009689A789B08D888B998BAA8BBB8B82E04F
:1091800090E0A0E0B0E08C8B9D8BAE8BBF8B1CA2DF
:109190001DA21EA21FA280E090E0A8E4B4E4888F84
:1091A000998FAA8FBB8F80E090E0A8E4B4EC8C8FFD
:1091B0009D8FAE8FBF8F8DEC9CECACE4BEE388A39B
:1091C00099A3AAA3BBA3DF91CF911F910F910895FB
:1091D0004F925F926F927F928F929F92AF92BF92C7
:1091E000CF92DF92EF92FF920F931F93CF93DF9373
:1091F0008C01EB0184E2FB0111928A95E9F78EE183
:109200000E94EC6983E090E00E94E7690E94E569B2
:1092100066E08EE14DD780916D1390E020916E1342
:10922000821B910986309105ECF38BEA9FE00E9446
:10923000AD55882E8BEA9FE00E94AD55982E8BEAA3
:109240009FE00E94AD55682E8BEA9FE00E94AD55CD
:10925000782E8BEA9FE00E94AD55482E8BEA9FE066
:109260000E94AD55582EB82CA12CB5016929072EA6
:10927000000C880B990B0E94B4AE4B015C01F80105
:109280006583768387839087D42CC12CB6016529AA
:10929000072E000C880B990B0E94B4AEF801618771
:1092A000728783879487F62CE12CB7016729072EF4
:1092B000000C880B990B0E94B4AEF8016587768785
:1092C0008787908B118A128A138A148A84E290E02D
:1092D000A0E0B0E088839983AA83BB8385899689BF
:1092E000A789B08D8C839D83AE83BF8382E090E09D
:1092F000A0E0B0E088879987AA87BB87188A198A77
:109300001A8A1B8AC0906502D0906602E0906702BC
:10931000F0906802A7019601C501B4010E9404B152
:1093200020E030E048EC52E40E9413AF6C8B7D8B60
:109330008E8B9F8BA7019601F801618572858385CD
:1093400094850E9404B120E030E048EC52E40E9491
:1093500013AF688F798F8A8F9B8F20916102309134
:1093600062024091630250916402F801658576853E
:10937000878590890E9404B120E030E048EC52E4F7
:109380000E9413AF6C8F7D8F8E8F9F8F81E0DF9156
:10939000CF911F910F91FF90EF90DF90CF90BF90F2
:1093A000AF909F908F907F906F905F904F900895B7
:1093B000862F0C945885862F642F0C948085862FD9
:1093C000642F0C94AE85FC0180819181009711F08F
:1093D0000C943DAA60E070E0CB010895FC0180810F
:1093E0009181009711F00C9440AA60E070E0CB01ED
:1093F0000895AF92BF92CF92DF92EF92FF920F93B8
:109400001F93CF93DF93DC01CD90DC901197C114B3
:10941000D10409F443C01496CD91DC91159720979F
:10942000E9F18C0176015701BFEFAB1ABB0AF701D6
:109430008081082E000C990B0E947EAE892B11F0C2
:109440007501F1CF2197CC0DDD1D8881082E000C10
:10945000990B0E947EAE892B29F0CE15DF0510F006
:109460002197F3CFAE014F5F5F4F4E195F09D801CF
:1094700015965C934E931497CE14DF0420F4B70135
:10948000C6010E94F1B5D801ED91FC911197149697
:109490008D919C911597E80FF91F1082DF91CF9164
:1094A0001F910F91FF90EF90DF90CF90BF90AF9002
:1094B0000895FC01248135816217730748F4808187
:1094C0009181009729F0FC01E60FF71F8081089534
:1094D00080E00895EF92FF920F931F93CF93DF9355
:1094E0006115710511F480E01DC08B01EC01CB0109
:1094F0000E946DAA0097A9F02C813D817C01E20EAB
:10950000F31EB701CE01C3DD882369F328813981B9
:109510008C819D81B801820F931F0E9466AAFD82F3
:10952000EC8281E0DF91CF911F910F91FF90EF903E
:109530000895CF93DF931F921F92CDB7DEB7698353
:109540001A8241E050E0BE016F5F7F4FC7DD0F9090
:109550000F90DF91CF9108956115710549F0FB01DE
:1095600001900020E9F73197AF01461B570BB6CDAC
:1095700080E00895FB014481558160817181AECD09
:109580000F931F93CF93DF938C01EB01FC0180813C
:109590009181009739F06881798161157105A1F495
:1095A0000E9463B488819981F801918380838A81C4
:1095B0009B81938382838C819D819583848319828F
:1095C00018821B821A820FC0F801428153812C81BC
:1095D0003D814217530720F30E9403B68C819D8181
:1095E000F801958384831D821C82DF91CF911F91A6
:1095F0000F910895CF93DF93EC01888199810097B3
:1096000011F00E9463B4198218821D821C821B8291
:109610001A82DF91CF910895CF93DF93EC0161150A
:10962000710559F0FB0101900020E9F73197AF0176
:10963000461B570B53DD811102C0CE01DBDFCE018B
:10964000DF91CF910895CF93DF93EC01FB0144812B
:1096500055816081718142DD811102C0CE01CADF76
:10966000CE01DF91CF910895EF92FF920F931F9358
:10967000CF93DF93EC018B016115710549F0CB01AC
:109680000E946DAA7C01BC01CE0101DD811103C0E5
:10969000CE01B0DF07C0FD82EC82B80188819981DC
:1096A0000E9466AACE01DF91CF911F910F91FF908A
:1096B000EF900895EF92FF920F931F93CF93DF9354
:1096C000EC017B018A01BA01E2DC811103C0CE0109
:1096D00091DF07C01D830C83B701888199810E94A7
:1096E00003B6CE01DF91CF911F910F91FF90EF90C4
:1096F0000895CF93DF93EC016115710551F0FB01E3
:1097000001900020E9F73197AF01461B570BD2DFDC
:1097100001C070DFCE01DF91CF910895CF93DF9329
:10972000EC01FB018617970751F06081718161158B
:10973000710521F044815581BDDF01C05BDFCE01A1
:10974000DF91CF910895FC01808191810C9463B4E5
:10975000EF92FF920F931F93CF93DF93CDB7DEB7B6
:10976000A1970FB6F894DEBF0FBECDBF7C01CB0131
:10977000BA01F701118210821382128215821482BB
:1097800042E0420F8E010F5F1F4F0E941EAABC01D4
:10979000C701AFDFA1960FB6F894DEBF0FBECDBFF5
:1097A000DF91CF911F910F91FF90EF900895CF938C
:1097B000DF931F921F92CDB7DEB7FC01118210829A
:1097C000138212821582148269831A82BE016F5F2E
:1097D0007F4F8FDF0F900F90DF91CF910895FC01A5
:1097E000118210821382128215821482C9CEFC016A
:1097F00011821082138212821582148235CFFC01ED
:1098000011821082138212821582148287CFFC018A
:1098100011821082138212821582148261157105E1
:1098200049F0FB0101900020E9F73197AF01461B99
:10983000570B40CF0895BF92CF92DF92EF92FF92E5
:109840000F931F93CF93DF937C016B018A01E90192
:109850002417350720F4812F8901C42FD82F6FEBEF
:1098600079E0C701D4DFD60114968D919C911597AC
:1098700008171907C0F48C179D0708F4EC01D601EE
:10988000ED91FC911197EC0FFD1FB08010826D914E
:109890007C91600F711FC7012CDFD601ED91FC9107
:1098A000EC0FFD1FB082C701DF91CF911F910F9187
:1098B000FF90EF90DF90CF90BF900895DC01ED9185
:1098C000FC910190F081E02D1994DB0114964D91EB
:1098D0005C9115976D917C91DC01ED91FC9102807A
:1098E000F381E02D1994EF92FF920F931F93CF9382
:1098F000DF938C017B01C0E0D0E0F701EC0FFD1F8E
:109900006491662361F0D801ED91FC910190F081A2
:10991000E02DC8011995892B11F02196EECFCE01CB
:10992000DF91CF911F910F91FF90EF9008956115F6
:10993000710579F0FB0101900020E9F73197AF0143
:10994000461B570BDC01ED91FC910280F381E02D69
:10995000199480E090E008958F929F92AF92BF9209
:10996000EF92FF920F931F93CF93DF93CDB7DEB7A4
:10997000A1970FB6F894DEBF0FBECDBF7C01FA01F0
:10998000CB0119A2223008F42AE08E010F5D1F4F8F
:10999000822E912CA12CB12CBF01A50194010E9413
:1099A0000CB0F901CA01015011096A3014F4605D6C
:1099B00001C0695CD8016C93232B242B252B61F704
:1099C000B801C701B4DFA1960FB6F894DEBF0FBE91
:1099D000CDBFDF91CF911F910F91FF90EF90BF907E
:1099E000AF909F908F900895CF92DF92EF92FF9269
:1099F0000F931F93CF93DF934115510579F4DC0149
:109A0000ED91FC910190F081E02DDF91CF911F91BC
:109A10000F91FF90EF90DF90CF9019946B01770F2B
:109A2000EE08FF084A305105E9F4F7FE19C0EC01D1
:109A30006DE244DF8C0144275527BA014C195D09BA
:109A40006E097F092AE0CE0187DF800F911FDF9129
:109A5000CF911F910F91FF90EF90DF90CF900895DD
:109A60002AE001C0242FB701A601DF91CF911F91F9
:109A70000F91FF90EF90DF90CF906ECF58CF1F9255
:109A80000F920FB60F9211240BB60F922F933F93A4
:109A90004F935F936F937F938F939F93AF93BF93F6
:109AA000EF93FF9387E39DE038DAFF91EF91BF9149
:109AB000AF919F918F917F916F915F914F913F9166
:109AC0002F910F900BBE0F900FBE0F901F90189507
:109AD0001F920F920FB60F9211240BB60F922F9375
:109AE0003F934F935F936F937F938F939F93AF9326
:109AF000BF93EF93FF9387E39DE00E943F85FF9123
:109B0000EF91BF91AF919F918F917F916F915F91F5
:109B10004F913F912F910F900BBE0F900FBE0F9062
:109B20001F9018951F920F920FB60F9211240BB62B
:109B30000F922F933F934F935F936F937F938F93E6
:109B40009F93AF93BF93EF93FF9384ED9DE0E5D98F
:109B5000FF91EF91BF91AF919F918F917F916F9105
:109B60005F914F913F912F910F900BBE0F900FBEC1
:109B70000F901F9018951F920F920FB60F921124FD
:109B80000BB60F922F933F934F935F936F937F93F7
:109B90008F939F93AF93BF93EF93FF9384ED9DE0DB
:109BA0000E943F85FF91EF91BF91AF919F918F915F
:109BB0007F916F915F914F913F912F910F900BBECD
:109BC0000F900FBE0F901F9018951F920F920FB617
:109BD0000F9211240BB60F922F933F934F935F93E5
:109BE0006F937F938F939F93AF93BF93EF93FF9365
:109BF00081E79EE092D9FF91EF91BF91AF919F9144
:109C00008F917F916F915F914F913F912F910F9025
:109C10000BBE0F900FBE0F901F9018951F920F92C2
:109C20000FB60F9211240BB60F922F933F934F93C1
:109C30005F936F937F938F939F93AF93BF93EF93B4
:109C4000FF9381E79EE00E943F85FF91EF91BF91D6
:109C5000AF919F918F917F916F915F914F913F91C4
:109C60002F910F900BBE0F900FBE0F901F90189565
:109C70001F920F920FB60F9211240BB60F922F93D3
:109C80003F934F935F936F937F938F939F93AF9384
:109C9000BF93EF93FF938EE09FE03FD9FF91EF9149
:109CA000BF91AF919F918F917F916F915F914F91F4
:109CB0003F912F910F900BBE0F900FBE0F901F90F2
:109CC00018951F920F920FB60F9211240BB60F9298
:109CD0002F933F934F935F936F937F938F939F93B4
:109CE000AF93BF93EF93FF938EE09FE00E943F8579
:109CF000FF91EF91BF91AF919F918F917F916F9164
:109D00005F914F913F912F910F900BBE0F900FBE1F
:109D10000F901F901895DC0180E0615098F02D9114
:109D2000982F9227E92FEF70F0E0E258F04F24913E
:109D300092959F70E92FF0E0E257F04FE491822F67
:109D40008E27EBCF0895EF92FF920F931F93CF933F
:109D5000DF938C017B0140E065E5CDD7E70188E02A
:109D6000E80EF11C699140E0C801C5D7CE15DF05AA
:109D7000C9F7DF91CF911F910F91FF90EF90089558
:109D80006F927F928F929F92AF92BF92CF92DF920B
:109D9000EF92FF920F931F93CF93DF93EC017B0120
:109DA0008A018E819F81DAD7882389F1B7018E815C
:109DB0009F81C9DF40E06EEB8E819F819CD7780147
:109DC000680189E0C80ED11CAE80BF8088E0882E73
:109DD000912C712C66246394C5013AD781117628A1
:109DE000660CE1E08E1A9108B9F7F70171927F01D4
:109DF000EC15FD0549F78E819F81B0D7813039F48C
:109E000068E0C80188DF91E0F8012085281390E020
:109E1000892FDF91CF911F910F91FF90EF90DF90ED
:109E2000CF90BF90AF909F908F907F906F9008954C
:109E3000CF93DF93CDB7DEB729970FB6F894DEBF87
:109E40000FBECDBFAE014F5F5F4F9ADF882389F011
:109E50008D818F3361F020F48F3159F489E00CC08B
:109E60008F3519F08F3739F004C08BE005C08AE0D8
:109E700003C080E001C08CE029960FB6F894DEBFE5
:109E80000FBECDBFDF91CF910895BF92CF92DF92E9
:109E9000EF92FF920F931F93CF93DF93EC016B012F
:109EA0008D85811104C0CE0159D7811105C01B8653
:109EB0001D861C8680E05CC040E060EFCE011BD7B1
:109EC00001E0E12CB12C11E0CE01C2D6F82ECE017A
:109ED000BFD691E0F91203C08130B1F433C02E2D0A
:109EE00030E0F8121BC08B85181738F4FE01E20F22
:109EF000F31F8381802341F402C0811729F0F12CE4
:109F0000193058F41C8709C0FE01EE0DF11D838144
:109F1000802B8383FF24F39409C0B12EFE01E20F4E
:109F2000F31F9381802F8095892383836F2DCE012A
:109F3000B3D61F5F000F11F4E39401E087E08E15A4
:109F400008F0C2CF113408F4B2CFBB86B11002C002
:109F500081E08D878B81882309F4A9CFDE011396D8
:109F6000F6012B968D918193CA17DB07D9F781E013
:109F7000DF91CF911F910F91FF90EF90DF90CF90E5
:109F8000BF900895DF92EF92FF920F931F93CF93AC
:109F9000DF937C018B01D42EDC011696ED91FC91B0
:109FA0001797138615861486DF011B9633961E922B
:109FB000EA17FB07E1F7C0E0B801F7018681978156
:109FC00064DFD82F882369F0DC1208C067E0C8017D
:109FD000A2DED80117969C91891721F0CF5FDC167D
:109FE00058F7D0E08D2FDF91CF911F910F91FF9007
:109FF000EF90DF90089510926E1310926D131092EF
:10A00000150D1092360D1092130D81E08093120DF4
:10A010001092ED0C61E084E10E94808561E085E1B1
:10A020000E948085E9EBF0E080818E7F80838081D3
:10A030008D7F808388E48093B80085E48093BC00A2
:10A040008BE995E59093530C8093520C8CE995E540
:10A050009093510C8093500C08950F931F93CF93BE
:10A06000DF93CDB7DEB762970FB6F894DEBF0FBEB1
:10A07000CDBF8C01CB01F8011182108213821282B4
:10A08000158214824AE0BE016F5F7F4F0E9476AA5C
:10A09000BE016F5F7F4FC8012CDB62960FB6F8944C
:10A0A000DEBF0FBECDBFDF91CF911F910F910895FD
:10A0B000613208F060E20E94F08E10926E1380937D
:10A0C0006D130895AF92BF92CF92DF92EF92FF92FD
:10A0D0000F931F93CF93DF93C82FD62F1092801228
:10A0E0001092811210928212109283121092841296
:10A0F00061E00E94AE8560E08C2F0E9480856D2F0C
:10A1000070E080E090E00E94348660E08C2F0E9436
:10A11000AE858BE990E00197F1F700E911E08C2F13
:10A120000E945885892B31F401501109C1F78EEF37
:10A130009FEF4CC000E911E08C2F0E9458850197D9
:10A1400009F43FC018E2D0E800E090E9E92EFF24CE
:10A15000F3948C2F0E945885892B29F481E0E81A0A
:10A16000F108B9F7E4CF0E940F866B017C0180E90A
:10A17000A82EBB24B3948C2F0E945885019729F4F4
:10A1800081E0A81AB108B9F7D2CF0E940F86DC018E
:10A19000CB018C199D09AE09BF098997A105B105AD
:10A1A00038F0E02FF0E0E858FD4E80858D2B808759
:10A1B000D69511F40F5FD0E8115039F680E090E0A9
:10A1C00005C00150110909F0B7CFB1CFDF91CF9190
:10A1D0001F910F91FF90EF90DF90CF90BF90AF90C5
:10A1E0000895EF92FF920F931F93CF93DF93C82FA1
:10A1F0008B017A0183E50E94EC696C2F8BEA9FE06A
:10A20000F4D40E94E56983E50E94EC69B80183E516
:10A2100090E00E94328FE701CE018E199F093091A4
:10A220006D1320916E13321729F08BEA9FE095D4BD
:10A230008993F2CF0817190729F01092861281E04E
:10A2400080938712DF91CF911F910F91FF90EF9034
:10A250000C94E569CF93DF934AE050E0BC018EE0B7
:10A260009FE0C2DBEC018EE09FE00E9474698C0FDE
:10A270009D1FDF91CF9108951F93CF93DF931F927E
:10A28000CDB7DEB7162FAE014F5F5F4F61E070E0D4
:10A29000A8DF898190E002C0959587951A95E2F72D
:10A2A00081700F90DF91CF911F910895CF93DF932D
:10A2B000D82FC62F83E50E94EC696D2F8BEA9FE0B3
:10A2C00094D46C2F8BEA9FE090D4DF91CF910C94C3
:10A2D000E569FF920F931F93CF93DF931F92CDB742
:10A2E000DEB7182F062FF42EAE014F5F5F4F61E0EF
:10A2F00070E077DF4981FF2049F021E030E001C0C4
:10A30000220F0A95EAF7242B298309C081E090E007
:10A3100001C0880F0A95EAF78095842389836981B3
:10A32000812FC4DF0F90DF91CF911F910F91FF908C
:10A3300008950F931F93CF93DF93EC019A01452B60
:10A3400019F40E94AF4705C0462F50E060E070E06E
:10A3500003DB8C01CE010E947469800F911FDF9195
:10A36000CF911F910F910895CF93DF9342E00E9408
:10A37000A36AEC018EE09FE00E9474698C0F9D1F20
:10A38000DF91CF9108958F929F92AF92BF92CF921B
:10A39000DF92EF92FF920F931F93CF93DF9300D042
:10A3A00000D0CDB7DEB75C0144E952E166E070E071
:10A3B00082E317DF80919412909195129A8389839A
:10A3C00080919612909197129C838B838091981222
:10A3D000909199129E838D83CE0101966C0188E83D
:10A3E000E82E82E1F82E8501F601619171916F01ED
:10A3F000F70181909190A190B1907F01072E000C00
:10A40000880B990B0E94B4AEA50194010E9413AF72
:10A41000F80161937193819391938F01F4E9EF16A1
:10A42000F2E1FF0609F726960FB6F894DEBF0FBEDD
:10A43000CDBFDF91CF911F910F91FF90EF90DF90F3
:10A44000CF90BF90AF909F908F900895CF93DF9360
:10A45000C82F80910C130E94EC696C2F8BEA9FE04F
:10A46000C4D380E00E94896963E080910C1320DEF0
:10A470008BEA9FE072D3EC018BEA9FE06ED320E081
:10A4800030E0382FC9018C2B9D2BDF91CF9108959F
:10A490000F931F93CF93DF93CDB7DEB761970FB6BE
:10A4A000F894DEBF0FBECDBF8C01462FBE01665FA4
:10A4B0007F4F68DD811105C060E070E08EEF92ECA7
:10A4C0004BC0AE014F5F5F4FBE01665F7F4FC8015B
:10A4D00057DC882361F12A8130E0C901982F882751
:10A4E000990F990F990F698128E0629FB00111249B
:10A4F0009C01262B372B8A858031E1F4688570E03A
:10A500008F81AB01481B5109CA019695982F882766
:10A51000979587950E9465B360517109207F53E03C
:10A52000220F331F5A95E1F7620F731F04C060E8D2
:10A5300074EE01C0B901613854EE75070CF4BCCF5C
:10A54000072E000C880B990B0E94B4AE20E030E07F
:10A5500040E05CE30E9413AF61960FB6F894DEBF53
:10A560000FBECDBFDF91CF911F910F9108959F92A4
:10A57000AF92BF92CF92DF92EF92FF920F931F9311
:10A58000CF93DF93CDB7DEB761970FB6F894DEBFF8
:10A590000FBECDBF8C018CE0F8018183C12CD12C82
:10A5A0002FE5E22E3FE7B32E4FE1A42E5FE3952E79
:10A5B000F801848190E0C816D9060CF095C04C2DA6
:10A5C000BE01665F7F4FC801DDDCF8018181893003
:10A5D00038F0F82EFCE0F81728F49CE0F92E02C0C1
:10A5E00089E0F82E8A85803131F0BE01665F7F4FA9
:10A5F000C8011EDC01C08CE0F81609F471C0AE0180
:10A600004F5F5F4FBE01665F7F4FC801B9DB882394
:10A6100009F466C08A85803109F462C08BE0F816BF
:10A6200051F0ECE0FE1629F0FAE0FF1206C09D8220
:10A6300005C0BD8203C0ED8201C0AD82F8018681F4
:10A6400097818CD3BE01665F7F4FF8018681978129
:10A650007ADB40E06EE4F801868197814CD340E0DC
:10A660006B81F8018681978146D340E06C81F801C7
:10A670008681978140D38A85803131F040E06D81B9
:10A68000F8018681978137D3F8018681978166D357
:10A69000BE01665F7F4FF8018681978154DBF80128
:10A6A000408168E48681978126D364E170E080E090
:10A6B00090E00E943486F8018081882331F06AE0BE
:10A6C00070E080E090E00E943486F80186819781F6
:10A6D00045D3F80181818F1508F48F2DF80181830E
:10A6E000FFEFCF1ADF0A64CF61960FB6F894DEBF92
:10A6F0000FBECDBFDF91CF911F910F91FF90EF90D3
:10A70000DF90CF90BF90AF909F9008958F929F92CF
:10A71000AF92BF92CF92DF92EF92FF920F931F936F
:10A72000CF93DF93EC018E819F8118D340E06CECD6
:10A730008E819F81E0D2488164E48E819F81DBD24B
:10A740008A81882309F441C0E981E950E33040F46B
:10A75000F0E0EE0FFF1FEB5CFA4F0081118102C0A9
:10A760000EEE12E08B818823F1F0888181111BC0ED
:10A770000E9490874B015C016801110FEE08FF08F1
:10A780008E819F8165D2813001F10E949087DC012A
:10A79000CB018C199D09AE09BF0988159905AA0539
:10A7A000BB0570F312C0B801110F880B990BDF9134
:10A7B000CF911F910F91FF90EF90DF90CF90BF90BE
:10A7C000AF909F908F900C943486DF91CF911F9122
:10A7D0000F91FF90EF90DF90CF90BF90AF909F9040
:10A7E0008F900895EF92FF920F931F93CF93DF9373
:10A7F000CDB7DEB728970FB6F894DEBF0FBECDBF3A
:10A800008C01DC011696ED91FC9117971386158645
:10A810001486DF011B9633961E92EA17FB07E1F7B9
:10A82000F80114821582EE24E394BE016F5F7F4F1E
:10A83000D80116968D919C91179727DB882309F4F0
:10A840006DC067E0CE01019666DA98858913EDCF79
:10A85000F801808181111FC0868197817FD2BE015E
:10A860006F5F7F4FD80116968D919C9117976BDA89
:10A8700040E064EBF801868197813DD2D8011696BD
:10A880008D919C911797E4D1F82EF80186819781DC
:10A8900065D2FF20A1F1D8011196FC908981803109
:10A8A000C9F1BE016F5F7F4FC801C2DA8F1518F47E
:10A8B000F80181810AC08981803111F48CE005C0E2
:10A8C000BE016F5F7F4FC801B3DAD80111968C9338
:10A8D000119714968C9114978F5F14968C9389819D
:10A8E000883281F030F4803169F0823209F09DCFF6
:10A8F00009C08B3339F0823409F097CF03C0F801D7
:10A90000E082C9CFD80115968C9115978F5F159667
:10A910008C938BCFBCE0BF1558F2D0CF28960FB6E2
:10A92000F894DEBF0FBECDBFDF91CF911F910F9185
:10A93000FF90EF9008956F927F928F929F92AF92C7
:10A94000BF92CF92DF92EF92FF920F931F93CF931C
:10A95000DF93CDB7DEB72C970FB6F894DEBF0FBEEE
:10A96000CDBF7C015B014A016FEB79E00E94074C8F
:10A970006FEB79E0CE0107960E94074CC12CD12CD9
:10A9800035018FEF681A780A8E010F5F1F4FC814C8
:10A99000D9040CF084C0F701848195818615970550
:10A9A00008F07DC0B501C8010E94388BB801CE0106
:10A9B00007960E94C04AC8010E94A34B64E170E060
:10A9C00080E090E00E9434868B859C85892B61F421
:10A9D000B501C8010E94D689B801CE0107960E9430
:10A9E000C04AC8010E94A34B8B859C85892B79F0B6
:10A9F00060EF77E08F8198850E94FAB5892BD9F4B2
:10AA0000F701248135812115310569F514C064E110
:10AA100070E080E090E00E943486F70184819581A7
:10AA20008A159B0520F4EFEFCE1ADE0AB0CFF5E1D0
:10AA3000CF0ED11CACCFBE01695F7F4FC7010E9412
:10AA4000BA4AF2E3CF1AD108B701C8010E94FF4BFE
:10AA500042E350E06FEF7FEFC8010E947C8DC80198
:10AA60000E94A34BDACF2230310530F46FEB79E04E
:10AA7000C7010E94794BE5CF2150310940E050E0F9
:10AA8000B701C8010E941B4C0E151F0521F0B8012B
:10AA9000C7010E94C04AC8010E94A34BD2CFCE0179
:10AAA00007960E94A34BC7012C960FB6F894DEBF01
:10AAB0000FBECDBFDF91CF911F910F91FF90EF900F
:10AAC000DF90CF90BF90AF909F908F907F906F90CE
:10AAD000089585ED8093BC008091BC0084FDFCCF7F
:10AAE0001092130D08954091740C262F30E0240F1E
:10AAF000311D21323105DCF42091130D2430C9F4CD
:10AB0000FC0180E090E0861758F43091740C21919C
:10AB1000DC01AC5AB34FA30FB11D2C930196F3CFB8
:10AB20008091740C680F6093740C80E0089581E04C
:10AB3000089582E00895089508950895E0916E13B0
:10AB400080916D13E81730F4F0E0E159FC4E8081FC
:10AB500090E008958FEF9FEF089590916E1380918C
:10AB60006D13981750F4E92FF0E0E159FC4E208165
:10AB700030E09F5F90936E1302C02FEF3FEFC9014B
:10AB8000089580916D1390E020916E13821B9109BE
:10AB90000895CF92DF92EF92FF920F931F93CF937E
:10ABA000DF937C01CB018A012091140D222389F0CF
:10ABB000EB016B01C40ED51ECC15DD0561F069916A
:10ABC000D701ED91FC910190F081E02DC70119951D
:10ABD000F3CF642F88DFC801DF91CF911F910F91D0
:10ABE000FF90EF90DF90CF900895CF93DF931F9267
:10ABF000CDB7DEB769832091140D2223D1F02091C7
:10AC0000360D203240F021E030E0FC013383228316
:10AC100080E090E014C08091150DE82FF0E0EA5E2E
:10AC2000F24F998190838F5F8093150D8093360D3D
:10AC300004C061E0CE01019656DF81E090E00F9004
:10AC4000DF91CF91089580E090E008950C9463B473
:10AC5000FC0190810180F281E02DF8948181892BA3
:10AC600081832281892F809528232283A7E0B0E069
:10AC70001197F1F7218182238183A3E2B0E011973C
:10AC8000F1F780817894EFECF0E03197F1F79823B9
:10AC900081E009F480E00895FC0190810180F28157
:10ACA000E02D892F809560FF12C0F89422818223C5
:10ACB00082838181892B8183A3E2B0E01197F1F730
:10ACC0008281982B9283789487ED90E011C0F8945C
:10ACD0002281822382838181892B8183AFEFB0E03F
:10ACE0001197F1F78281982B928378948FE090E00E
:10ACF0000197F1F70895DF92EF92FF920F931F9360
:10AD0000CF93DF93EC01D62EE42E08E010E0FF2471
:10AD1000F39461E08D2D8F2109F460E0CE01BCDF5A
:10AD2000FF0C01501109A9F7E11010C0F894E98156
:10AD3000FA8191818881809589238183E981FA81D3
:10AD4000928188818095892382837894DF91CF9145
:10AD50001F910F91FF90EF90DF900895DC012C91EF
:10AD60001196ED91FC911297F8948181922F909514
:10AD70008923818378948DE743E050E0815021F16D
:10AD8000DA011197F1F730813223C1F3F89482810F
:10AD9000892382838181822B81837894ABE7B7E01A
:10ADA0001197F1F7F89481819823918383E191E0E1
:10ADB0000197F1F78081282381E009F080E0789401
:10ADC000E3E6F6E03197F1F708951F93CF93DF9311
:10ADD000EC01162F60E0812F0E94AE85612F70E09C
:10ADE000FB01E05BFC4EE491E883FB01E65FFC4E77
:10ADF000E491F0E0EE0FFF1FE051FD4E859194913C
:10AE00009A8389831B861D861C86FE013B962396AA
:10AE10001292EC17FD07E1F7DF91CF911F91089592
:10AE20001F93CF93DF93EC01162F8C810E94EC6966
:10AE30006B85812F862B90E00E94E769DF91CF918F
:10AE40001F910C94E5690F931F93CF938C01C62F2C
:10AE5000E7DF6C2F6460C801E3DF6C2F6B7FC801F4
:10AE6000DFDF83EC90E00197F1F7CF911F910F9115
:10AE700008950F931F93CF938C01C62F607F61605D
:10AE8000E2DF80E1C89FB00111246160C801DBDF0F
:10AE900081E090E0CF911F910F9108951F920F9242
:10AEA0000FB60F9211240BB60F922F933F934F932F
:10AEB0005F936F937F938F939F93AF93BF93EF9322
:10AEC000FF938091B80F0E9458852091BB0F30915D
:10AED000BC0F2F5F3F4F3093BC0F2093BB0F90915F
:10AEE000BA0F953618F096E09093B70F9091B70F80
:10AEF0009430C9F128F4923069F09330D1F05EC0FB
:10AF0000953009F451C0963009F058C091E0909303
:10AF1000871051C0811152C02091BB0F3091BC0FDE
:10AF20002436310508F442C0109287101092BA0FEF
:10AF30001CC0813009F042C0E091BA0F91E09E0F31
:10AF40009093BA0FF0E02091BB0F3091BC0FEE0F41
:10AF5000FF1FE354F04F318320831092BC0F1092F7
:10AF6000BB0F94E029C0811117C0E091BA0F91E0A6
:10AF70009E0F9093BA0FF0E02091BB0F3091BC0F61
:10AF8000EE0FFF1FE354F04F318320831092BC0F6C
:10AF90001092BB0F93E010C02091BB0F3091BC0FFB
:10AFA0002536310558F007C0811108C01092BC0F3A
:10AFB0001092BB0F03C095E09093B70F9091B90F1B
:10AFC000992329F0811102C02F9A01C02F98FF9177
:10AFD000EF91BF91AF919F918F917F916F915F9111
:10AFE0004F913F912F910F900BBE0F900FBE0F907E
:10AFF0001F901895CF92DF92EF92FF92CF93DF933D
:10B00000EC01072E000C880B990B0E94B4AE6B016B
:10B010007C0120E030E040E45FE30E9413AF20E0D9
:10B0200030E048E452E40E9404B10E949DB1C6178A
:10B03000D707D4F020E030E040EA5FE3C701B60173
:10B040000E9413AF20E030E048E452E40E9404B1D3
:10B0500020E030E040E85FE30E943EB00E949DB1F6
:10B0600021E06C177D070CF420E0822F90E0DF9147
:10B07000CF91FF90EF90DF90CF9008950F931F93A3
:10B08000CF93DF93082F60E476E08EE09FE00E948C
:10B090003E4DC7E0D0E010E0B8010C2E02C075951F
:10B0A00067950A94E2F76170772742E050E08EE0FE
:10B0B0009FE00E94F44C219778F7DF91CF911F9188
:10B0C0000F9108951F920F920FB60F9211240BB695
:10B0D0000F922F933F934F935F936F937F938F9331
:10B0E0009F93AF93BF93EF93FF938091B900887FB5
:10B0F000803609F49CC068F5883209F45BC090F48E
:10B10000803109F454C038F4882309F4F6C088303B
:10B1100009F44DC0F5C0883109F44CC0803209F4FF
:10B120005DC0EEC0803409F468C048F4803309F48F
:10B1300055C0883309F0E4C08093110DD8C0803524
:10B1400009F44FC0883509F45DC0883409F0D8C0CF
:10B15000D6C0883909F4C7C0A8F4883709F467C095
:10B1600038F4883609F463C0803709F460C0C8C079
:10B17000883809F4B8C0803909F45FC0803809F014
:10B18000BFC05BC0803B09F486C038F4803A09F444
:10B1900066C0883A09F47FC0B3C0803C09F4A7C0F8
:10B1A000883C09F4A4C0883B09F48AC0A9C08091F6
:10B1B000EE0C10C09091100D80910F0D981770F546
:10B1C000E091100D81E08E0F8093100DF0E0E151C1
:10B1D000F34F80818093BB0085EC86C08093110D76
:10B1E0008EC0E091100D81E08E0F8093100D809144
:10B1F000BB00F0E0E151F34F80839091100D8091FE
:10B200000F0D6EC0E091100D81E08E0F8093100D38
:10B210008091BB00F0E0E151F34F80838091120DEB
:10B2200081116DC081E08093ED0C84EA61C083E000
:10B230008093130D1092960CCFCF8091960C803294
:10B2400008F051C0E091960C81E08E0F8093960C2F
:10B250008091BB00F0E0EA58F34F8083BDCF85ECCE
:10B260008093BC001092130D8091960C803230F4C4
:10B27000E091960CF0E0EA58F34F10826091960C42
:10B2800070E0E091500CF091510C86E79CE019952C
:10B290001092960C35C084E08093130D1092750CBB
:10B2A0001092740CE091520CF091530C199580910E
:10B2B000740C811105C081E08093740C1092540CC1
:10B2C000E091750C81E08E0F8093750CF0E0EC5AE4
:10B2D000F34F80818093BB009091750C8091740C2A
:10B2E000981708F479CF85E88093BC0009C085ECF5
:10B2F0008093BC001092130D03C01092110DE9DB76
:10B30000FF91EF91BF91AF919F918F917F916F913D
:10B310005F914F913F912F910F900BBE0F900FBEF9
:10B320000F901F9018950895E9E8F0E114A215A276
:10B3300016A217A210A611A612A613A681E084A732
:10B3400029E130E036A725A787A780E090E0A0EAB2
:10B35000B0E480AB91ABA2ABB3AB80E090E0A8EAE5
:10B36000B1E484AB95ABA6ABB7AB809325029093C9
:10B370002602A0932702B093280280E090E0A0E884
:10B38000BFE38093D3109093D410A093D510B093C3
:10B39000D6108093210290932202A0932302B093AF
:10B3A0002402109200111092FF108BE090E0909315
:10B3B00002118093011190932A0280932902109226
:10B3C000380C1092370C80E090E00C94346EEF92C1
:10B3D000FF920F931F93CF93DF93CDB7DEB768979C
:10B3E0000FB6F894DEBF0FBECDBF8C0168ED7BE0D9
:10B3F000CE010D960E94074C60E179E0CE014396A4
:10B400000E94074C61EF7FE0C8010E94F74BBE012C
:10B410006D5E7F4FC8010E94BA4A68EE7FE0C801A6
:10B420000E946A4A88E1E82E81E1F82EF7016081E6
:10B4300070E0CE0101960E942D50BE016F5F7F4FDC
:10B44000CE0107960E94FF4BBE01635F7F4FCE0186
:10B4500007960E94234BBC01C8010E94BA4ACE0144
:10B4600007960E94A34BCE0101960E94A34B6BED61
:10B470007FE0C8010E946A4AF7016181062E000C34
:10B48000770BCE0101960E942D50BE016F5F7F4F5A
:10B49000CE0107960E94FF4BBE01635F7F4FCE0136
:10B4A00007960E94234BBC01C8010E94BA4ACE01F4
:10B4B00007960E94A34BCE0101960E94A34B61ED1B
:10B4C0007FE0C8010E946A4AF7016281062E000CE3
:10B4D000770BCE0101960E942D50BE016F5F7F4F0A
:10B4E000CE0107960E94FF4BBE01635F7F4FCE01E6
:10B4F00007960E94234BBC01C8010E94BA4ACE01A4
:10B5000007960E94A34BCE0101960E94A34B69ECC3
:10B510007FE0C8010E946A4AF70163817481CE010D
:10B5200001960E942D50BE016F5F7F4FCE0107969E
:10B530000E94FF4BBE016D5E7F4FCE0107960E94B9
:10B54000234BBC01C8010E94BA4ACE0107960E9453
:10B55000A34BCE0101960E94A34B62EB7FE0C80192
:10B560000E946A4AF70165817681CE0101960E94A8
:10B570002D50BE016F5F7F4FCE0107960E94FF4B9B
:10B58000BE01635F7F4FCE0107960E94234BBC0133
:10B59000C8010E94BA4ACE0107960E94A34BCE0171
:10B5A00001960E94A34B69EA7FE0C8010E946A4AA3
:10B5B000F7016781062E000C770B6F5F7F4FCE017E
:10B5C00001960E942D50BE016F5F7F4FCE010796FE
:10B5D0000E94FF4BBE01635F7F4FCE0107960E9422
:10B5E000234BBC01C8010E94BA4ACE0107960E94B3
:10B5F000A34BCE0101960E94A34B6EE97FE0C801E8
:10B600000E946A4AF7016085062E000C770BCE0176
:10B6100001960E942D50BE016F5F7F4FC8010E94AE
:10B62000BA4ACE0101960E94A34BCE0143960E94D6
:10B63000A34BCE010D960E94A34BC80168960FB68E
:10B64000F894DEBF0FBECDBFDF91CF911F910F9158
:10B65000FF90EF9008950F931F9360E08091020296
:10B660000E94808583E090E00197F1F761E080918E
:10B6700002020E94808583E290E00197F1F760E08A
:10B68000809102020E9480858091000290910102C7
:10B690009927FC01E05BFC4E6491FC01E65FFC4EE7
:10B6A000E491F0E0EE0FFF1FE051FD4E8591949183
:10B6B00000E412E42FE030E0462F0E94109A61155A
:10B6C00071058105910549F0DC01CB010196A11DB1
:10B6D000B11DBC01CD019F7003C060E070E0CB01E3
:10B6E0000E94B2AE20E030E048EC52E40E9404B187
:10B6F0002091970C3091980C4091990C50919A0C94
:10B700000E9413AF20E030E44CE156E40E9404B103
:10B7100020E030E040E05FE30E9413AF1F910F9103
:10B72000089523E333E948E853E40E9404B120E09C
:10B7300030E040E85FE30E943EB00E94FCB226E6A3
:10B7400036EA45EA53E40E9413AF6093970C709376
:10B75000980C8093990C90939A0C0895CF92DF9255
:10B76000EF92FF9278DF6B017C0120E030E040E057
:10B7700050E40E94F3B118161CF46DDF6B017C01DC
:10B7800020E030E040E050E4C701B6010E94F3B190
:10B7900018161CF460DF6B017C0120E030E040E013
:10B7A00050E4C701B6010E94F3B118161CF453DF30
:10B7B0006B017C0120E030E040E050E4C701B601BD
:10B7C0000E94F3B118162CF4FF90EF90DF90CF9009
:10B7D00042CFC701B601FF90EF90DF90CF90089560
:10B7E000BF92CF92DF92EF92FF920F931F93CF936E
:10B7F000DF93CDB7DEB762970FB6F894DEBF0FBE0A
:10B80000CDBF8C016B0168ED7BE0CE010D960E94EF
:10B81000074C67E370E1C8010E94F74B76012FEFF8
:10B82000E21AF20AB701CE0101960E942D50BE0124
:10B830006F5F7F4FCE0107960E94FF4B66E177E076
:10B84000CE0107960E940C4BBC01C8010E94BA4A67
:10B85000CE0107960E94A34BCE0101960E94A34BF6
:10B860008AE0B82EBE9CC001BF9C900D1124FC0143
:10B87000E85EFE4E7F018081082E000C990B0E942D
:10B88000E3B5892B09F4B2C0B701CE0101960E943D
:10B89000074CBE016F5F7F4FCE0107960E94FF4BA2
:10B8A00069EF7AE0CE0107960E940C4BBC01C801FB
:10B8B0000E94BA4ACE0107960E94A34BCE01019680
:10B8C0000E94A34BBC9CC001BD9C900D11249C0107
:10B8D000285E3E4E7901F9016685062E000C770B35
:10B8E000CE0101960E942D50BE016F5F7F4FCE01A9
:10B8F00007960E94FF4B63E179E0CE0107960E9414
:10B900000C4BBE01635F7F4F0E94234BBC01C801FB
:10B910000E94BA4ACE0107960E94A34BCE0101961F
:10B920000E94A34B60E370E1C8010E946A4AF701DC
:10B930006785062E000C770BCE0101960E942D50D4
:10B94000BE016F5F7F4FCE0107960E94FF4BBE0185
:10B95000635F7F4FCE0107960E94234BBC01C80155
:10B960000E94BA4ACE0107960E94A34BCE010196CF
:10B970000E94A34B6AE270E1C8010E946A4AF70183
:10B9800060897189CE0101960E942D50BE016F5FC2
:10B990007F4FCE0107960E94FF4BBE01635F7F4F32
:10B9A000CE0107960E94234BBC01C8010E94BA4AEF
:10B9B000CE0107960E94A34BCE0101960E94A34B95
:10B9C00065E270E1C8010E946A4AF70162897389E1
:10B9D000CE0101960E942D50BE016F5F7F4FC801BE
:10B9E0000E94BA4ACE0101960E94A34BCE010D9649
:10B9F0000E94A34BC80162960FB6F894DEBF0FBE3B
:10BA0000CDBFDF91CF911F910F91FF90EF90DF900D
:10BA1000CF90BF9008950F931F93CF93DF93CDB72F
:10BA2000DEB72C970FB6F894DEBF0FBECDBF8C01EA
:10BA30006FEB79E08CE392E10E94794B08301105BD
:10BA400009F0DFC066E271E1CE0101960E94F74B7A
:10BA500044E650E06FEF7FEFCE0101960E94C48F65
:10BA6000CE0101960E94A34B6AE171E1CE010196DD
:10BA70000E94F74B44E650E060E070E0CE01019692
:10BA80000E947C8DCE0101960E94A34B87E39DE02E
:10BA90000E94FB474CE251E061E070E0CE0101966C
:10BAA0000E949B54809197138823D1F065E179E03F
:10BAB000CE0107960E94074CBE016F5F7F4FCE01FB
:10BAC00007960E94234B61E277E00E940C4BBC0179
:10BAD0008EE09FE00E947869CE0107960E94A34BFA
:10BAE0006DEC78E0CE0107960E94074CBE01695FBD
:10BAF0007F4FCE0101960E940F85182FCE01079629
:10BB00000E94A34B112309F4A5C268E179E08CE3FC
:10BB100092E10E94794B88E090E09093080C80932A
:10BB2000070C0E943535182F6DE071E1CE010796A4
:10BB30000E94F74B44E650E060E070E0CE010796CB
:10BB40000E947C8DCE0107960E94A34B87E39DE067
:10BB50000E94FB4748E552E061E070E0CE010796A5
:10BB60000E949B54BE01695F7F4FCE0101960E94E7
:10BB7000C04ACE0107960E94A34B80919713882359
:10BB8000D1F065E179E0CE0107960E94074CBE0135
:10BB90006F5F7F4FCE0107960E94234B61E277E0F3
:10BBA0000E940C4BBC018EE09FE00E947869CE01A0
:10BBB00007960E94A34B60E476E0CE0107960E94B0
:10BBC000074CBE01695F7F4FCE0101960E940F8531
:10BBD000082FCE0107960E94A34B002309F43AC216
:10BBE0006DE179E08CE392E10E94794B0E9435355A
:10BBF000882309F42FC2112309F42CC260E071E1FB
:10BC0000F9C0093F2FEF120709F00BC16FEE70E189
:10BC1000CE0101960E94F74B44E650E06FEF7FEFB4
:10BC2000CE0101960E94C48FCE0101960E94A34BC3
:10BC300061EE70E1CE0101960E94F74B44E650E0C0
:10BC400060E070E0CE0101960E947C8DCE010196ED
:10BC50000E94A34B87E39DE00E94FB474CE251E02A
:10BC600064E070E0CE0101960E949B54809197138E
:10BC70008823D1F065E179E0CE0107960E94074C58
:10BC8000BE016F5F7F4FCE0107960E94234B61E29A
:10BC900077E00E940C4BBC018EE09FE00E94786927
:10BCA000CE0107960E94A34B60E070E0CE010196A2
:10BCB0000E94594A082E000C990BC0970A9708F069
:10BCC000CCC163E279E0CE0107960E94074CBE0129
:10BCD0006F5F7F4FCE0107960E94234BBC018CE320
:10BCE00092E10E948E4BCE0107960E94A34B89EFF2
:10BCF0009FEF9093080C8093070C0E943535182F06
:10BD000063ED70E1CE0107960E94F74B44E650E0E8
:10BD100060E070E0CE0107960E947C8DCE01079610
:10BD20000E94A34B87E39DE00E94FB4748E552E059
:10BD300065E070E0CE0107960E949B54BE01695FEA
:10BD40007F4FCE0101960E94C04ACE0107960E9405
:10BD5000A34B809197138823D1F065E179E0CE0160
:10BD600007960E94074CBE016F5F7F4FCE0107967A
:10BD70000E94234B61E277E00E940C4BBC018EE0F5
:10BD80009FE00E947869CE0107960E94A34B60E075
:10BD900070E0CE0101960E94594A082E000C990BC2
:10BDA000C0970A9708F059C168E279E0CE0107967A
:10BDB0000E94074CBE016F5F7F4FCE0107960E9425
:10BDC000234BBC018CE392E10E948E4BCE0107967F
:10BDD0000E94A34B89EF9FEF9093080C8093070C70
:10BDE0000E943535882309F438C1112309F435C17F
:10BDF00066EC70E1CE0107960E94F74B44E650E0F6
:10BE000060E070E0CE0107960E947C8DCE0107961F
:10BE10000E94A34B6FEB79E08CE392E10E94794B97
:10BE200014C165EB70E1CE0101960E94F74B44E628
:10BE300050E06FEF7FEFCE0101960E94C48FCE01DC
:10BE400001960E94A34B6FEB79E08CE392E10E9494
:10BE5000794B053F8FEF180749F46DE678E08CE3E6
:10BE600092E10E94794B6BEA70E126C0063F2FEF0A
:10BE7000120749F467E678E08CE392E10E94794B7F
:10BE800061EA70E119C0013F8FEF180749F461E7DB
:10BE900078E08CE392E10E94794B62E970E10CC09A
:10BEA000023F2FEF1207B9F46DE279E08CE392E1E3
:10BEB0000E94794B62E870E1CE0101960E94F74B37
:10BEC00044E650E06FEF7FEFCE0101960E947C8D3B
:10BED000CE010196C5C00230110509F07EC066E7AB
:10BEE00070E1CE0101960E94F74B44E650E06FEFFF
:10BEF0007FEFCE0101960E94C48FCE0101960E9471
:10BF0000A34B66E670E1CE0101960E94F74B44E632
:10BF100050E06FEF7FEFCE0101960E947C8DCE0145
:10BF200001960E94A34B44EF51E066E070E0CE0121
:10BF300001960E949B54BE016F5F7F4F8CE392E19C
:10BF40000E94C04ACE0101960E94A34B80914012EC
:10BF500090914112059708F486C060E070E08CE390
:10BF600092E10E94594A082E000C990BC0970A973B
:10BF700008F079C08CE392E10E94EE49613523EC30
:10BF80007207810591050CF46EC00E94B4AE20E0EA
:10BF900030E048EC52E40E9404B1AB01BC0122E065
:10BFA000CE0107960E94A84B6EE478E0CE01019680
:10BFB0000E94074CBE01695F7F4FCE0101960E942F
:10BFC000234BBC018CE392E10E948E4BCE01019683
:10BFD0000E94A34BCE01079643C06FE470E1CE01EF
:10BFE00001960E94F74B44E650E06FEF7FEFCE01E1
:10BFF00001960E947C8DCE0101960E94A34B6FEBAF
:10C0000079E08CE392E10E94794B0B3E8FEF1807A9
:10C0100009F465C08091401290914112892BE1F59D
:10C020005EC068EC70E080E090E00E94348669E3D6
:10C0300070E1CE0101960E94F74B44EF51E06FEFA3
:10C040007FEFCE0101960E947C8DCE0101960E9469
:10C05000A34B45C069EF70E1CDCE6FEB70E1CACE66
:10C060000E94A34BD7CF68E570E1CE0101960E94F4
:10C07000F74B48EE53E06FEF7FEFCE0101960E9441
:10C080007C8DCE0101960E94A34B6FEB79E08CE38F
:10C0900092E10E94794BBECF0E943535882309F288
:10C0A00068EC70E080E090E00E94348665E470E126
:10C0B000CE0101960E94F74B44EF51E06FEF7FEF06
:10C0C000CE0101960E947C8DCE0101960E94A34B69
:10C0D0001093080C0093070CC8010E94D70A2C96F5
:10C0E0000FB6F894DEBF0FBECDBFDF91CF911F9189
:10C0F0000F9108956F927F928F929F92AF92BF920D
:10C10000CF92DF92EF92FF920F931F93CF93DF9323
:10C11000CDB7DEB768970FB6F894DEBF0FBECDBFC0
:10C120006C018091FF1090910011019731F06FEB3D
:10C1300079E0C6010E94074C46C169E379E0CE016F
:10C140000D960E94074CBE01635F7F4F87E39DE021
:10C150000E94654C6CE271E080E090E00E943486C1
:10C16000CE0143960E946B7564E670E080E090E03B
:10C170000E943486E12CF12C85E0A82EB12C9AE0A7
:10C18000892E912C64E479E0CE0101960E94074C3F
:10C190008F89988D892B69F06B887C8869817A8179
:10C1A000C3010E9427B6009721F08C0106191709D8
:10C1B00002C00FEF1FEFCE0101960E94A34BA80112
:10C1C0004F5F5F4FBE016D5E7F4FCE0101960E94B3
:10C1D000D83EBE016F5F7F4FCE010D960E94C04AD0
:10C1E000CE0101960E94A34B89899A89892B69F017
:10C1F00060E070E0CE010D960E94594A082E000CB6
:10C20000990BC0970A9708F4C7C010E065E170E188
:10C21000CE0101960E94F74B44E150E06FEF7FEFB3
:10C22000CE0101960E946990CE0101960E94A34B17
:10C230008FEFE81AF80A62E370E080E090E00E9475
:10C240003486C701B5010E9465B3019771F5CE012F
:10C2500001960E9422748D819E81892B59F0BE0126
:10C260006F5F7F4F8CE392E10E948E4B0E948C7E29
:10C2700011E017C084E1E816F1049CF0C701B40195
:10C280000E9465B3892B69F4BE01635F7F4F87E32A
:10C290009DE00E94654C68EC70E080E090E00E94B8
:10C2A0003486CE0101960E94A34BCE0101960E94D6
:10C2B0006B75BE016F5F7F4FCE0143960E94C04AEF
:10C2C000CE0101960E94A34B62E370E080E090E013
:10C2D0000E94348684E6E816F10419F0112309F46B
:10C2E00051CF809197138823F1F061E179E0CE017D
:10C2F00001960E94074CBE01635F7F4FCE010196FD
:10C300000E94234BBC01CE0107960E94FF4BCE0139
:10C3100007960E94BB70CE0107960E94A34BCE01E8
:10C3200001960E94A34B89899A89892B61F060E06C
:10C3300070E0CE010D960E94594A082E000C990B10
:10C34000C0970A9730F066E479E0C6010E94074C76
:10C350001AC062E579E0CE0101960E94074CBE0149
:10C360006F5F7F4FCE010D960E940F85182FCE0173
:10C3700001960E94A34B1111E6CFBE01635F7F4F70
:10C38000C6010E94EF4BCE0143960E94A34BCE0103
:10C390000D960E94A34B17C062E579E0CE0101968D
:10C3A0000E94074CBE016F5F7F4FCE010D960E9429
:10C3B0000F85082FCE0101960E94A34B11E00023A8
:10C3C00009F424CF22CFC60168960FB6F894DEBFD9
:10C3D0000FBECDBFDF91CF911F910F91FF90EF90D6
:10C3E000DF90CF90BF90AF909F908F907F906F9095
:10C3F0000895AF92BF92CF92DF92EF92FF920F9388
:10C400001F93CF93DF93CDB7DEB72C970FB6F89479
:10C41000DEBF0FBECDBF8091430C811102C00E94D0
:10C420008D3E8091050290910602029751F0809115
:10C430000D0C90910E0C009709F48DC1039709F42F
:10C440008AC16FE571E188E192E10E94344B68E1B5
:10C4500072E1CE0101960E94FF4B44E150E060E0A2
:10C4600070E0CE0101960E94C48FCE0101960E9419
:10C47000A34B60E571E188E192E10E94344B68E1F1
:10C4800072E1CE0101960E94FF4B44E150E06FEF54
:10C490007FEFCE0101960E947C8DCE0101960E9415
:10C4A000A34B87E00E9426528C0186E00E94265210
:10C4B000BC0180E090E00E94B2AE2AE037ED43EA92
:10C4C0005CE30E9413AF23E333E948E853E40E949E
:10C4D0003DB06B017C0184E0A82EB12C20E030E05F
:10C4E00048EC52E4C701B6010E94F3B1181614F5E6
:10C4F00081E0A81AB10809F4F4C064E670E080E0B5
:10C5000090E00E94348686E00E942652BC0180E0C2
:10C5100090E00E94B2AE2AE037ED43EA5CE30E946D
:10C5200013AF23E333E948E853E40E943DB06B01C5
:10C530007C01D4CFB80180E090E00E94B2AE2AE046
:10C5400037ED43EA5CE30E9413AF23E333E948E8A5
:10C5500053E40E943DB0AB01BC0121E0CE01019645
:10C560000E94A84B6CE679E0CE0107960E94074C2A
:10C57000BE016F5F7F4FCE0107960E94234BBC0127
:10C580008EE192E10E948E4BCE0107960E94A34B52
:10C59000CE0101960E94A34B6EE172E1CE0101969D
:10C5A0000E94FF4B42E350E06FEF7FEFCE01019618
:10C5B0000E947C8DCE0101960E94A34B66E779E034
:10C5C000CE0101960E94074CCE0101960E94F88D83
:10C5D000CE0101960E94A34B65E779E08EE192E1DE
:10C5E0000E94AC4A21E0B701A601CE0101960E944B
:10C5F000A84B6DE07AE0CE0107960E94074CBE0181
:10C600006F5F7F4FCE0107960E94234BBC0184E2EF
:10C6100092E10E948E4BCE0107960E94A34BCE0161
:10C6200001960E94A34B68ED7BE0CE0101960E942B
:10C63000074C64E272E1CE0101960E94234BBC01DB
:10C6400088E192E10E948E4BCE0101960E94A34B9D
:10C6500068E172E1CE0101960E94FF4B4AE050E092
:10C6600060E070E0CE0101960E946990CE010196D3
:10C670000E94A34B66E779E0CE0101960E94074C29
:10C68000CE0101960E94F88DCE0101960E94A34B27
:10C6900065E779E084E292E10E94AC4A64E272E1EB
:10C6A000CE0101960E94FF4B68ED7BE0CE01019622
:10C6B0000E940C4B6EE172E10E94234BBC018EE1A3
:10C6C00092E10E948E4BCE0101960E94A34B809175
:10C6D0000D0C90910E0C039709F006C184E090E0D8
:10C6E000FFC065E471E188E192E10E94344B68E1AA
:10C6F00072E1CE0101960E94FF4B4AE050E060E0FB
:10C7000070E0CE0101960E94C48FCE0101960E9476
:10C71000A34B6AE579E0CE0101960E94074C68E1DF
:10C7200072E1CE0101960E94234BBC018EE192E1A1
:10C730000E948E4BCE0101960E94A34B80910D0C5E
:10C7400090910E0C049721F410920E0C10920D0C87
:10C7500081E090E018C184ED9DE00E94168E64E6B1
:10C7600070E080E090E00E94348665E871E188E145
:10C7700092E10E94344B68E172E1CE0101960E9481
:10C78000FF4B44E150E060E070E0CE0101960E9472
:10C79000C48FCE0101960E94A34B66E771E188E148
:10C7A00092E10E94344B68E172E1CE0101960E9451
:10C7B000FF4B44E150E06FEF7FEFCE0101960E9406
:10C7C0007C8DCE0101960E94A34B8CE40E94348E96
:10C7D0006B017C0104E010E0A7019601C701B601DE
:10C7E0000E943DB3811192C021E0B701A601CE01A4
:10C7F00007960E94A84B6CE679E0CE0101960E9454
:10C80000074CBE01695F7F4FCE0101960E94234B0A
:10C81000BC018EE192E10E948E4BCE0101960E94F6
:10C82000A34BCE0107960E94A34B6EE172E1CE01AD
:10C8300001960E94FF4B42E350E06FEF7FEFCE0185
:10C8400001960E947C8DCE0101960E94A34B66E763
:10C8500079E0CE0101960E94074CCE0101960E941C
:10C86000F88DCE0101960E94A34B65E779E08EE139
:10C8700092E10E94AC4A86E60E94348E6B017C01F4
:10C8800004E010E0A7019601C701B6010E943DB384
:10C89000882309F47DC00150110909F0E2C06FEB53
:10C8A00079E084E292E10E94794B64E272E1CE0188
:10C8B00001960E94FF4B68ED7BE0CE0101960E943D
:10C8C0000C4B6EE172E10E94234BBC018EE192E1C0
:10C8D0000E948E4BCE0101960E94A34B83E090E014
:10C8E00090930E0C80930D0C64E670E080E090E075
:10C8F0000E9434868091430C882309F4BEC060E214
:10C9000073E080E090E00E943486B7C001501109C6
:10C9100009F09BC06BE671E188E192E10E94344B23
:10C9200068E172E1CE0101960E94FF4B4AE050E0BF
:10C9300060E070E0CE0101960E94C48FCE010196A6
:10C940000E94A34B6AE579E0CE0101960E94074C54
:10C9500068E172E1CE0101960E94234BBC018EE199
:10C9600092E10E948E4BCE0101960E94A34B8091D2
:10C970000D0C90910E0C039721F410920E0C109256
:10C980000D0C82E090E09093060280930502ACCFFC
:10C9900021E0B701A601CE0107960E94A84B6DE0E9
:10C9A0007AE0CE0101960E94074CBE01695F7F4F7D
:10C9B000CE0101960E94234BBC0184E292E10E94C9
:10C9C0008E4BCE0101960E94A34BCE0107960E948A
:10C9D000A34B68ED7BE0CE0101960E94074C64E218
:10C9E00072E1CE0101960E94234BBC0188E192E1E5
:10C9F0000E948E4BCE0101960E94A34B68E172E12A
:10CA0000CE0101960E94FF4B4AE050E06FEF7FEFAE
:10CA1000CE0101960E946990CE0101960E94A34B1F
:10CA200066E779E0CE0101960E94074CCE0101969F
:10CA30000E94F88DCE0101960E94A34B65E779E034
:10CA400084E292E10E94AC4A30CF68EC70E080E072
:10CA500090E00E9434868CE40E94348E6B017C014D
:10CA6000BBCE68EC70E080E090E00E94348686E601
:10CA70000E94348E6B017C0105CF2C960FB6F89482
:10CA8000DEBF0FBECDBFDF91CF911F910F91FF9001
:10CA9000EF90DF90CF90BF90AF9008952F923F928C
:10CAA0004F925F926F927F928F929F92AF92BF92BE
:10CAB000CF92DF92EF92FF920F931F93CF93DF936A
:10CAC000CDB7DEB7C554D1090FB6F894DEBF0FBE9F
:10CAD000CDBF2B013C0169017A010E94908722960B
:10CAE0006CAF7DAF8EAF9FAF229720E9421621E059
:10CAF00052066104710434F090E9492E5524539490
:10CB0000612C712C30E1C31637E2D306E104F10445
:10CB10002CF4CDA6DEA6EFA6F8AA08C080E197E225
:10CB2000A0E0B0E08DA79EA7AFA7B8AB8091430C63
:10CB3000882321F0CDA6DEA6EFA6F8AA22966CAD3A
:10CB40007DAD8EAD9FAD229728EE33E040E050E002
:10CB50000E94E0AF26962CAF3DAF4EAF5FAF269759
:10CB600091E09DAB19A61AA61BA61CA68E01035F19
:10CB70001F4FCC24DD247601C418D508E608F70839
:10CB8000C9AADAAAEBAAFCAAC9A4DAA4EBA4FCA459
:10CB90002DA53EA54FA558A9C216D306E406F50655
:10CBA0000CF02BC3C701B6010E94B4AE20E030E008
:10CBB0004AE754E40E9404B1AB01BC0123E0C80180
:10CBC0000E94A84BB80188E192E10E94C04AC801C6
:10CBD0000E94A34B8DA59EA5AFA5B8A90A97A10554
:10CBE000B10584F426964CAD5DAD6EAD7FAD269754
:10CBF000C80138D4B80188E192E10E94C04AC80156
:10CC00000E94A34BCE0101960E94C35168E371E1DB
:10CC10008EE192E10E94344BDE0111961D01C12C80
:10CC2000D12C7601F10181909190A190B1901F01DA
:10CC3000A5019401C501B4010E9413AF9B01AC0191
:10CC4000C701B6010E943EB06B017C0123E0B50133
:10CC5000A401C8010E94A84BB801CE0143960E94CE
:10CC6000FF4B68ED7BE0CE0143960E940C4BBC016C
:10CC70008EE192E10E94BA4ACE0143960E94A34BF4
:10CC8000C8010E94A34B0215130561F6C701B60146
:10CC90000E94FCB26B017C01FDE24F16F1E05F06E1
:10CCA000610471042CF00E948D3E60E080E0AFD3FF
:10CCB00023E0B701A601CE0143960E94A84B68EF7E
:10CCC00078E0C8010E94074C68E172E1C8010E9447
:10CCD000234B68E779E00E940C4BBE016D5E7F4FED
:10CCE0000E94234B6DE779E00E940C4BBC018EE162
:10CCF00092E10E94BA4AC8010E94A34BCE0143961A
:10CD00000E94A34B2DEC3CEC4CE45FE3C701B60161
:10CD10000E94F3B129813A814B815C812DA33EA30E
:10CD20004FA358A718160CF0ACC12AE939E949E914
:10CD30005FE3C701B6010E94AEAE87FFA2C1CDA8D6
:10CD4000CC2009F49EC189849A84AB84BC8420E001
:10CD500030E0A901C501B4010E94AEAECD80DE80F5
:10CD6000EF80F884882309F12DA13EA14FA158A599
:10CD7000CA01B9010E9413AF6EAB7FAB88AF99AF08
:10CD8000A7019601C701B6010E9413AF9B01AC0138
:10CD90006EA97FA988AD99AD0E943EB00E94FCB2F9
:10CDA000A50194010E94B1B004C06BED7FE089EC55
:10CDB0009FE320EE3EE245E652E40E9413AF6EABE5
:10CDC0007FAB88AF99AF20E030E0A901C701B60181
:10CDD0000E94AEAE882309F12DA13EA14FA158A516
:10CDE000CA01B9010E9413AF6AAF7BAF8CAF9DAF90
:10CDF000A5019401C501B4010E9413AF9B01AC01D0
:10CE00006AAD7BAD8CAD9DAD0E943EB00E94FCB280
:10CE1000A70196010E94B1B004C06BED7FE089ECE0
:10CE20009FE320EE3EE245E652E40E9413AF6AAF74
:10CE30007BAF8CAF9DAF20E030E0A9016DA17EA15A
:10CE40008FA198A50E94AEAE8823F9F0A5019401A8
:10CE5000C501B4010E9413AF4B015C01A70196010B
:10CE6000C701B6010E9413AF9B01AC01C501B4011B
:10CE70000E943EB00E94FCB22DA13EA14FA158A538
:10CE80000E94B1B06B017C0108C08BEDC82E8FE011
:10CE9000D82E89ECE82E8FE3F82E69EF78E0C801F0
:10CEA0000E94074C68E172E1C8010E94234B60E8D0
:10CEB00079E00E940C4BBC018EE192E10E948E4B06
:10CEC000C8010E94A34B69EF78E0C8010E94074C9B
:10CED00068E172E1C8010E94234B6AE979E00E948F
:10CEE0000C4BBC0188E192E10E948E4BC8010E946C
:10CEF000A34B21E04EA95FA968AD79ADCE014F9655
:10CF00000E94A84B21E04AAD5BAD6CAD7DADCE017A
:10CF100049960E94A84B20EE3EE245E652E4C70146
:10CF2000B6010E9413AFAB01BC0121E0C8010E9411
:10CF3000A84BB801CE0143960E94FF4B68ED7BE001
:10CF4000CE0143960E940C4BBE01675E7F4F0E944C
:10CF5000234B68ED7BE00E940C4BBE01615E7F4F6E
:10CF60000E94234BBC0182E192E10E948E4BCE01D4
:10CF700043960E94A34BC8010E94A34BCE01499641
:10CF80000E94A34BCE014F960E94A34B2DE2421666
:10CF900021E052066104710474F469A57AA58BA599
:10CFA0009CA525E030E040E050E00E94E0AF672B18
:10CFB000682B692BC1F568E172E1C8010E94FF4B43
:10CFC00045E050E06FEF7FEFC8010E946990C80113
:10CFD0000E94A34B63EA79E0C8010E94074C45E038
:10CFE00050E061EF7FEFC8010E94C48FC8010E942A
:10CFF000A34B6FEB79E0C8010E94074CC8010E9467
:10D00000F88DC8010E94A34B62E172E1C8010E9441
:10D01000FF4B45E050E060E070E0C8010E947C8D6D
:10D02000C8010E94A34B62E172E18EE192E10E948D
:10D03000BA4A3FE1431651046104710434F4C9A4AF
:10D04000DAA4EBA4FCA4F7FC11C06EE172E1C80104
:10D050000E94FF4BC8010E94BB70C8010E94A34BF5
:10D060006FEB79E08EE192E10E94794BB201C3014E
:10D0700077FE04C069A97AA98BA99CA90E9434866D
:10D08000A9C023E04DA15EA16FA178A5CE01439672
:10D090000E94A84B69EF78E0C8010E94074C68E144
:10D0A00072E1C8010E94234B65EA79E00E940C4BB3
:10D0B000BE016D5E7F4F0E94234B6EE779E00E94B8
:10D0C0000C4BBC0188E192E10E948E4BC8010E948A
:10D0D000A34BCE0143960E94A34B49855A856B858D
:10D0E0007C8523E0CE0149960E94A84B4D815E814C
:10D0F0006F81788523E0C8010E94A84BB801CE015A
:10D1000043960E94FF4B6AEA79E0CE0143960E9463
:10D110000C4BBE01675E7F4F0E94234B6EE779E0A8
:10D120000E940C4BBC0182E192E10E948E4BCE0129
:10D1300043960E94A34BC8010E94A34BCE0149967F
:10D140000E94A34B2DE2421621E0520661047104B5
:10D1500074F469A57AA58BA59CA525E030E040E094
:10D1600050E00E94E0AF672B682B692BF1F468E177
:10D1700072E1C8010E94FF4B4AE050E06FEF7FEF81
:10D18000C8010E946990C8010E94A34B62E172E14C
:10D19000C8010E94FF4B4AE050E060E070E0C80127
:10D1A0000E947C8DC8010E94A34B6EE172E1C80110
:10D1B0000E94FF4BC801DFD7C8010E94A34B6FEB51
:10D1C00079E08EE192E10E94794BC301B2010E94A5
:10D1D00034861DAA0E9490876B017C0122962CAD9B
:10D1E0003DAD4EAD5FAD2297C21AD30AE40AF50AEF
:10D1F000C9A6DAA6EBA6FCA6C7CC68E172E1CE010F
:10D200000D960E94FF4B4AE050E06FEF7FEFCE019A
:10D210000D960E94C48FCE010D960E94A34BCDA8FF
:10D22000CC20B1F163EA79E0CE010D960E94074C63
:10D2300045E050E061EF7FEFCE010D960E94C48F74
:10D24000CE010D960E94A34B8091430C882391F050
:10D2500060E371E1CE010D960E94F74B45E050E08E
:10D2600060E070E0CE010D960E94C48FCE010D9655
:10D270000E94A34B6FEB79E0CE010D960E94074C04
:10D28000CE010D960E94F88DCE010D960E94A34B03
:10D2900062E172E1CE010D960E94FF4B4AE050E040
:10D2A0006FEF7FEFCE010D960E947C8DCE010D9623
:10D2B0000E94A34BCB5BDF4F0FB6F894DEBF0FBECF
:10D2C000CDBFDF91CF911F910F91FF90EF90DF9035
:10D2D000CF90BF90AF909F908F907F906F905F9016
:10D2E0004F903F902F9008956DEB79E00C94974C00
:10D2F0000F931F93CF93DF93EC010E94654C8C0139
:10D30000CE01F2DF800F911FDF91CF911F910F911E
:10D310000895282F3091360D313208F04AC080919F
:10D32000130D8111FCCF90912B1342E04093130D0C
:10D330002093120D2FEF2093110D1092100D3093AA
:10D340000F0DE6E1FDE0AFEEBCE020E0321721F08A
:10D3500041914D932F5FFACF1092EE0C2091EE0C7D
:10D36000990F922B9093EE0C9091ED0C913061F40B
:10D370001092ED0C9091EE0C9093BB009091BC003C
:10D3800093FDF8CF95EC01C095EE9093BC00909181
:10D39000130D9230E1F39091110D9F3F79F0809140
:10D3A000110D803241F08091110D803331F084E015
:10D3B00005C081E003C082E001C083E01092150D3A
:10D3C0001092360D1092140D089581E0A2CF682FAF
:10D3D0008BEA9FE00C94F55591E09093140D8093A7
:10D3E0002B131092150D1092360D0895CF93C82F60
:10D3F000682F607F8FE193E10E94235780E1C89FEF
:10D40000B00111248FE193E1CF910C942357CF9376
:10D41000DF93CDB7DEB728970FB6F894DEBF0FBE07
:10D42000CDBF98E0EBE3F5E0DE01119601900D929F
:10D430009A95E1F790912813961710F46FEF690F02
:10D44000FE013196E60FF11DE60FF11D9081890F67
:10D45000806828960FB6F894DEBF0FBECDBFDF916F
:10D46000CF91C4CF0F931F93CF93DF93CDB7DEB788
:10D47000A2970FB6F894DEBF0FBECDBF8C01CB01D3
:10D48000BA01F8011182108213821282158214826D
:10D490002AE0AE014F5F5F4F0E9480AABE016F5F1E
:10D4A0007F4FC8010E94794BA2960FB6F894DEBF59
:10D4B0000FBECDBFDF91CF911F910F9108950F93B4
:10D4C0001F93CF93DF93EC010E94974C8C01CE0108
:10D4D0000BDF800F911FDF91CF911F910F91089566
:10D4E000CF92DF92EF92FF92CF93DF936B017C019B
:10D4F00097FF15C06DE28EE09FE00E945E4CEC014C
:10D5000044275527BA014C195D096E097F092AE0A5
:10D510008EE09FE00E94AC4CC80FD91F08C02AE0E3
:10D52000AB01BC018EE09FE00E94AC4CEC018EE0B0
:10D530009FE0DADE8C0F9D1FDF91CF91FF90EF907F
:10D54000DF90CF9008958F929F92AF92BF92CF922B
:10D55000DF92EF92FF920F931F93CF93DF936B01B4
:10D560007C01142F9B01AC010E943DB3882319F06C
:10D5700060EC79E027C046015701E894B7F82FEF37
:10D580003FEF4FE75FE7C501B4010E943DB3811152
:10D590000DC02FEF3FEF4FE75FE7C501B4010E94D9
:10D5A000AEAE18161CF464EC79E00CC02FEF3FEF20
:10D5B0004FE75FE4C701B6010E94F3B1181694F477
:10D5C00068EC79E08EE09FE0DF91CF911F910F91A1
:10D5D000FF90EF90DF90CF90BF90AF909F908F9093
:10D5E0000C94974C2FEF3FEF4FE75FECC701B6016C
:10D5F0000E94AEAE87FDE4CF20E030E0A901C70174
:10D60000B6010E94AEAE87FF0BC06DE28EE09FE0D8
:10D610000E945E4CEC01F7FAF094F7F8F09402C027
:10D62000C0E0D0E000E060E070E080E09FE3101731
:10D6300041F020E030E040E251E40E9404B10F5F8D
:10D64000F6CFA70196010E943EB06B017C010E94BB
:10D65000A2B14B015C012AE0AB01BC018EE09FE06E
:10D660000E94AC4CC80FD91F1123C9F1C501B401E8
:10D670000E94B2AE9B01AC01C701B6010E943DB051
:10D680006B017C016EE28EE09FE00E945E4CC80F51
:10D69000D91F20E030E040E251E4C701B6010E940A
:10D6A00013AF4B015C010E94A2B16B01E12CF12C84
:10D6B0002AE0B701A6018EE09FE00E94AC4CC80FA3
:10D6C000D91FC701B6010E94B2AE9B01AC01C501D2
:10D6D000B4010E943DB06B017C011150D1F6CE0126
:10D6E000DF91CF911F910F91FF90EF90DF90CF903E
:10D6F000BF90AF909F908F9008952F923F924F923E
:10D700005F926F927F928F929F92AF92BF92CF92D1
:10D71000DF92EF92FF920F931F93CF93DF93CDB7DA
:10D72000DEB728970FB6F894DEBF0FBECDBFC0900E
:10D730009D0CD0909E0C40919F0C5091A00CC41653
:10D74000D5062CF43C2D2D2D6A01432F522FE1EAF2
:10D75000FCE060E070E0CB01019111910417150726
:10D7600054F44A01550FAA08BB08680D791D8A1D9B
:10D770009B1DA80115C0C016D10654F40D2C000C39
:10D78000EE08FF086C0D7D1D8E1D9F1D680108C0F1
:10D79000012E000C220B330B600F711F821F931F91
:10D7A0002CE0ED3EF207C1F60E94B4AE20E030E07E
:10D7B00048E152E40E9404B18B0188879F838DE980
:10D7C000E82E8CE0F82E812C912C5401D7016D911C
:10D7D0007D917D01072E000C880B990B0E94B4AE41
:10D7E000980148855F810E943DB09B01AC010E9479
:10D7F00013AF9B01AC01C501B4010E943EB04B01C7
:10D800005C01EDEEFCE0EE15FF0501F720E030E0F5
:10D810004CE152E40E9404B10E94FCB26B017C0115
:10D8200020E030E040E85FE30E94F3B118160CF00E
:10D8300069C02DE93CE03A832983212C312C412C0D
:10D84000512C3201A981BA818D919D91BA83A9830E
:10D850009C01990F440B550B2B833C834D835E83B6
:10D86000CA01B9010E94B4AE980148855F810E9447
:10D870003DB04B015C0120E030E0A9010E94F3B112
:10D88000181624F0B7FAB094B7F8B094A70196012F
:10D89000C501B4010E94AEAE87FF0BC08B819C8195
:10D8A000AD81BE81480E591E6A1E7B1E9FEF291A4C
:10D8B000390AADEEBCE0E981FA81AE17BF0711F677
:10D8C00020E030E040EC5FE3C701B6010E9413AFF7
:10D8D0006B017C01F5E02F1631040CF4AACFC301D3
:10D8E000B2010E94B4AE6B017C01B101330C880B14
:10D8F000990B0E94B4AE9B01AC01C701B6010E9416
:10D9000004B103C0B80188859F816B017C01C70108
:10D91000B60128960FB6F894DEBF0FBECDBFDF91DB
:10D92000CF911F910F91FF90EF90DF90CF90BF901C
:10D93000AF909F908F907F906F905F904F903F90AF
:10D940002F9008954F925F926F927F928F929F9245
:10D95000AF92BF92CF92DF92EF92FF921F93CF933D
:10D96000DF93CDB7DEB728970FB6F894DEBF0FBEB2
:10D97000CDBF4B015C0111E0612E712C9301220F90
:10D98000331F220F331F3A832983F901EF57FD4FCD
:10D99000C080D180E280F380A5019401C701B60167
:10D9A0000E94AEAE87FF02C01F5FE6CFA5019401C3
:10D9B000C701B6010E94AEAE49815A8147595D4FF9
:10D9C0005E834D83811106C0FA016081718182817D
:10D9D00093814DC0F1E06F1AF0EC7F0AC301880F0C
:10D9E000991F880F991FFC01EF57FD4F208131814E
:10D9F0004281538129833A834B835C83FC01E7593D
:10DA0000FD4F4080518062807380A3019201ED81BF
:10DA1000FE8160817181828193810E943DB06D831E
:10DA20007E838F83988729813A814B815C81C501F0
:10DA3000B4010E943DB09B01AC016D817E818F815C
:10DA400098850E9413AF4B015C0129813A814B817B
:10DA50005C81C701B6010E943DB09B01AC01C501CC
:10DA6000B4010E9404B1A30192010E943EB0289625
:10DA70000FB6F894DEBF0FBECDBFDF91CF911F91DF
:10DA8000FF90EF90DF90CF90BF90AF909F908F90DE
:10DA90007F906F905F904F9008950F931F930E9417
:10DAA00090876093DC0D7093DD0D8093DE0D909375
:10DAB000DF0D84ED9DE00E943B4797FF1FC00E9451
:10DAC00090870091DC0D1091DD0D2091DE0D3091DD
:10DAD000DF0DDC01CB01801B910BA20BB30B00917E
:10DAE000D80D1091D90D2091DA0D3091DB0D8017F2
:10DAF0009107A207B307E8F28FEF9FEF1F910F91F5
:10DB00000895CF92DF92EF92FF92CF93DF93EC01D3
:10DB10006A017B01E889F98982E080834115514ED1
:10DB200061057105B1F060E079E08DE390E0A70157
:10DB300096010E940CB0DA01C9010197A109B1094F
:10DB4000B695A795979587959C01211580E1380793
:10DB5000A8F0E889F989108260E874E88EE190E025
:10DB6000A70196010E940CB0DA01C9010197A10931
:10DB7000B109B695A795979587959C01EC85FD858C
:10DB80003083EE85FF852083188EEC89FD8986E041
:10DB90008083EA89FB89808180618083EA89FB89AF
:10DBA000808188608083EA89FB89808180688083A6
:10DBB000EA89FB8980818F7D8083DF91CF91FF90FF
:10DBC000EF90DF90CF9008950F931F93CF93DF9343
:10DBD0001F921F92CDB7DEB70BE91CE0F801608100
:10DBE0008EED93E09A838983CE0101960E94BF3E19
:10DBF000F80161818FED93E09A838983CE010196CC
:10DC00000E94BF3EC8010F900F90DF91CF911F91EE
:10DC10000F910895EF92FF920F931F93CF93DF938D
:10DC20001F921F92CDB7DEB708E111E188519141F3
:10DC30007C01C701800F911FF80161918F019A83C8
:10DC40008983CE0101960E94BF3EF1E102321F0797
:10DC500081F788E191E10F900F90DF91CF911F91B3
:10DC60000F91FF90EF900895EF92FF920F931F9303
:10DC7000CF93DF931F921F92CDB7DEB709E810E173
:10DC8000895890417C01C701800F911FF801619173
:10DC90008F019A838983CE0101960E94BF3EF1E1F4
:10DCA0000F301F0781F789E890E10F900F90DF9107
:10DCB000CF911F910F91FF90EF900895EF92FF92F7
:10DCC0000F931F93CF93DF931F921F92CDB7DEB7B1
:10DCD00008E111E1885191417C01C701800F911F3A
:10DCE000F80161918F019A838983CE0101960E9488
:10DCF000BF3EF2E102311F0781F788E191E10F9009
:10DD00000F90DF91CF911F910F91FF90EF900895A9
:10DD10008F929F92AF92BF92CF92DF92EF92FF923B
:10DD20000F931F93CF93DF938C01862F0B30110538
:10DD300009F06FC090918512992309F0F89462E17F
:10DD40000E94625020918512222309F07894009756
:10DD500009F072C0E0908012F09081126F2D70E097
:10DD600080E090E00E94B4AE2DEC3CEC4CEC5DE326
:10DD70000E9413AF4B015C016E2D70E080E090E0DB
:10DD80000E94B4AE9B01AC01C501B4010E943EB03B
:10DD9000609378127093791280937A1290937B1229
:10DDA000C0918212D09183126C2F6F7770E080E067
:10DDB00090E00E94B4AE4B015C016D2F70E080E0FA
:10DDC00090E00E94B4AE2DEC3CEC4CEC5DE30E9484
:10DDD00013AF9B01AC01C501B4010E943EB0C7FD69
:10DDE00009C060937C1270937D1280937E12909391
:10DDF0007F120BC0DC01CB01B05880937C12909352
:10DE00007D12A0937E12B0937F12FE0CCF0DCD0F2A
:10DE100071C00631110509F0B4C0909185129923A3
:10DE200009F0F89461E00E9462502091851222234B
:10DE300009F078940097A9F040E050EC69E774ECA1
:10DE4000409378125093791260937A1270937B12F8
:10DE500040937C1250937D1260937E1270937F12D8
:10DE600095C0F0908112D0918012609180127091D3
:10DE7000811276276727762780E090E00E94B2AE75
:10DE80002DEC3CEC4CEC5DE30E9413AF60937812F8
:10DE90007093791280937A1290937B12E0908312A0
:10DEA000C09182128C2F8F776E2D70E0782B80E0DE
:10DEB00090E00E94B2AE2DEC3CEC4CEC5DE30E9495
:10DEC00013AFC7FD09C060937C1270937D128093DD
:10DED0007E1290937F120BC0DC01CB01B05880936F
:10DEE0007C1290937D12A0937E12B0937F12DF0D6F
:10DEF000ED0ECE0D80918412C81346C0C0907812EA
:10DF0000D0907912E0907A12F0907B1220E030E00D
:10DF100048EC52E4C701B6010E94F3B118161CF098
:10DF2000C0E0D0E002C0CBEFDFEF20E030E0A9019D
:10DF3000C701B6010E94AEAE87FF02C0CAEFDFEF95
:10DF4000C0907C12D0907D12E0907E12F0907F12F3
:10DF500020E030E048EC52ECC701B6010E94AEAEC2
:10DF600087FF02C0C9EFDFEF20E030E040EF52E46E
:10DF7000C701B6010E94F3B11816ACF4C8EFDFEF89
:10DF800012C0CFEFDFEF0FC08FEF9FEF8F3FFFEF9C
:10DF90009F0709F4D3C0009709F4B0CF029609F4A3
:10DFA000D9C0CCEFDFEF0C30110509F0D6C08CE5FD
:10DFB00013DA80E090E00BDA08DA65E08CE50E9485
:10DFC0005850C82FD0E02097A1F0C530D105A4F05B
:10DFD0000CE213E18BEA9FE00E94AD55F8018087C7
:10DFE0000F5F1F4FC8018C5293418C179D0794F30C
:10DFF00006C0CEEFDFEFB1C0CDEFDFEFAEC0C09116
:10E00000341300913513602F70E080E090E00E949F
:10E01000B4AE2DEC3CEC4CEC5DE30E9413AF6B0115
:10E020007C016C2F70E080E090E00E94B4AE9B0118
:10E03000AC01C701B6010E943EB060932C137093EF
:10E040002D1380932E1390932F13D091361310918C
:10E0500037136D2F6F7770E080E090E00E94B4AED0
:10E060006B017C01612F70E080E090E00E94B4AE13
:10E070002DEC3CEC4CEC5DE30E9413AF9B01AC013A
:10E08000C701B6010E943EB0D7FF5BC0DC01CB01E7
:10E09000B0588093301390933113A0933213B09300
:10E0A00033138C2F800FC82FCD0FC10F80913813E1
:10E0B000C81344C0C0902C13D0902D13E0902E13A1
:10E0C000F0902F1320E030E048EC52E4C701B60195
:10E0D0000E94F3B118161CF0C0E0D0E002C0CBEFF4
:10E0E000DFEF20E030E040EA50E4C701B6010E94D3
:10E0F000AEAE87FF02C0CAEFDFEFC0903013D09002
:10E100003113E0903213F090331320E030E040EF11
:10E1100051ECC701B6010E94AEAE87FF02C0C9EF45
:10E12000DFEF20E030E040EF52E4C701B6010E948B
:10E13000F3B1181694F4C8EFDFEF0FC0CFEFDFEFA5
:10E140000CC060933013709331138093321390930B
:10E150003313A7CFCEEFDFEF26CFCE01DF91CF91E4
:10E160001F910F91FF90EF90DF90CF90BF90AF90F5
:10E170009F908F900895CF93DF93FC012481358188
:10E18000232B89F0EC01BC0187E39DE0B1D86EE15F
:10E1900070E080E090E00E943486BE018EE09FE057
:10E1A000DF91CF91A5C8DF91CF910895CF92DF92F3
:10E1B000EF92FF92CF93C091B810C430DCF4C1301D
:10E1C0000CF03FC0C11164C07FD720E030E040EACE
:10E1D00050E40E9413AF20E030EC4FE754E40E947B
:10E1E00004B12091B9103091BA104091BB105091F8
:10E1F000BC104BC0C43009F04BC066D720E030E003
:10E2000040EA50E40E9413AF20E030EC4FE754E4C2
:10E210000E9404B120E030E040EA50E40E9404B1E2
:10E2200020E030E040E851E40E9413AF20E030E00D
:10E2300040E850E40E943EB020E030E04AE754E479
:10E2400024C042D72AE137E64CE950E40E9413AFDC
:10E250002091B9103091BA104091BB105091BC1070
:10E260000E943DB06B017C01EC2FEE0FFF0BE955D6
:10E27000FA4F60817181072E000C880B990B0E9468
:10E28000B4AE9B01AC01C701B6010E9404B103C04A
:10E2900060E070E0CB01CF91FF90EF90DF90CF90E6
:10E2A00008958F929F92AF92BF92CF92DF92EF929A
:10E2B000FF92CF93DF93CDB7DEB72C970FB6F894CC
:10E2C000DEBF0FBECDBF66E472E1CE0101960E94B3
:10E2D000F74B4CE251E06FEF7FEFCE0101960E94C9
:10E2E0007C8DCE0101960E94A34B6091B502709186
:10E2F000B6028091290290912A020ADD84E1882EDB
:10E30000912CA12CB12CE12CF12C2FEFE21AF20A66
:10E31000C501B4010E9434866091B5027091B602C5
:10E320008091290290912A02F3DC23E0E216F104A5
:10E3300034F02AE0E216F10444F4892B49F084E138
:10E34000880E911CA11CB11CE0CF892B09F08BC158
:10E350008091290290912A028B309105C9F4809115
:10E360007C1290917D12A0917E12B0917F128093C9
:10E370003D1390933E13A0933F13B09340138091AD
:10E38000781290917912A0917A12B0917B121DC0EF
:10E390008631910521F30C9701F58091301390910E
:10E3A0003113A0913213B091331380933D139093A6
:10E3B0003E13A0933F13B093401380912C13909180
:10E3C0002D13A0912E13B0912F1380933913909396
:10E3D0003A13A0933B13B0933C1340913D135091DB
:10E3E0003E1360913F137091401321E0CE010796D8
:10E3F0000E94A84B6DE07AE0CE0101960E94074C86
:10E40000BE01695F7F4FCE0101960E94234BBC0184
:10E410008EE192E10E948E4BCE0101960E94A34BA9
:10E42000CE0107960E94A34B4091391350913A13A5
:10E4300060913B1370913C1321E0CE0107960E943E
:10E44000A84B62E476E0CE0101960E94074CBE0123
:10E45000695F7F4FCE0101960E94234BBC018EE184
:10E4600092E10E94BA4ACE0101960E94A34BCE01CE
:10E4700007960E94A34B64E076E08EE192E10E9451
:10E48000AC4A6FEB79E0CE0101960E94074C44E163
:10E4900050E060E070E0CE0101960E94C48FCE0192
:10E4A00001960E94A34BC0903D13D0903E13E09084
:10E4B0003F13F090401320E030E0A901C701B601FE
:10E4C0000E94F3B120E030E040E05FE387FD05C04B
:10E4D000C701B6010E943EB004C0C701B6010E9448
:10E4E0003DB00E949DB1AB01BC01CE0101960E94DE
:10E4F000326ABE016F5F7F4F88E192E10E94C04A9D
:10E50000CE0101960E94A34B60E087E00E94076A5B
:10E5100068E172E18FE193E10E94654C6FED8FE15C
:10E5200093E10E945E4C68E476E08FE193E10E9403
:10E530003E4D6091391370913A1380913B13909145
:10E540003C130E949DB14AE050E08FE193E10E94AC
:10E55000F44C64E076E08FE193E10E943E4D64E686
:10E5600070E080E090E00E943486C0903D13D0902F
:10E570003E13E0903F13F090401320E030E040EF76
:10E5800051E4C701B6010E94F3B187FD03C067E300
:10E5900072E154C020E030E040ED51E4C701B60123
:10E5A0000E94F3B187FD1FC067E272E1CE010196C0
:10E5B0000E94F74B4AE050E06FEF7FEFCE010196EB
:10E5C0000E947C8DCE0101960E94A34B8091470250
:10E5D000882331F06CED75E080E090E00E94348695
:10E5E00067E172E12BC020E030E040EB51E4C7016D
:10E5F000B6010E94F3B187FD03C069E072E11EC05D
:10E600006AEF71E1CE0101960E94F74B4AE050E0BB
:10E610006FEF7FEFCE0101960E947C8DCE010196B7
:10E620000E94A34B80914702882331F06CED75E086
:10E6300080E090E00E9434866CEE71E1CE0101969C
:10E640000E94F74B4AE050E06FEF7FEFCE0101965A
:10E650000E947C8DCE0101960E94A34B62E370E084
:10E6600080E090E0DCC00E948D3E6EE170E080E0D2
:10E6700090E00E9434860E94A3976B017C0164E6BF
:10E6800070E080E090E00E9434866DE07AE08EE1F8
:10E6900092E10E94794B21E0B701A601CE010196DB
:10E6A0000E94A84BBE016F5F7F4F8EE192E10E94F6
:10E6B000BA4ACE0101960E94A34B6EE172E1CE01EF
:10E6C00001960E94FF4B4AE050E060E070E0CE010E
:10E6D00001960E94C48FCE0101960E94A34B8091A7
:10E6E0002E05882379F080912D05882359F06FED50
:10E6F0008FE193E10E945E4C66E779E08FE193E160
:10E700000E943E4D65E779E08EE192E10E94AC4ABD
:10E71000C0923D13D0923E13E0923F13F09240130B
:10E7200020E030E040EF51E4C701B6010E94F3B1B0
:10E7300087FD03C06CED71E154C020E030E040ED96
:10E7400051E4C701B6010E94F3B187FD1FC06CEC14
:10E7500071E1CE0101960E94F74B4AE050E06FEF65
:10E760007FEFCE0101960E947C8DCE0101960E9422
:10E77000A34B80914702882331F06CED75E080E077
:10E7800090E00E9434866CEB71E12BC020E030E019
:10E7900040EB51E4C701B6010E94F3B187FD03C00D
:10E7A0006EEA71E11EC06FE971E1CE0101960E942F
:10E7B000F74B4AE050E06FEF7FEFCE0101960E94E9
:10E7C0007C8DCE0101960E94A34B80914702882345
:10E7D00031F06CED75E080E090E00E94348661E9F4
:10E7E00071E1CE0101960E94F74B4AE050E06FEFD5
:10E7F0007FEFCE0101960E947C8DCE0101960E9492
:10E80000A34B6CE271E080E090E00E94348680913E
:10E810004702882331F068EE73E080E090E00E94C8
:10E8200034862C960FB6F894DEBF0FBECDBFDF91B5
:10E83000CF91FF90EF90DF90CF90BF90AF909F90DF
:10E840008F900895DF92EF92FF920F931F93CF93D3
:10E85000DF93CDB7DEB762970FB6F894DEBF0FBE79
:10E86000CDBF8C01109241136FEB79E0CE010D9674
:10E870000E94074CFF24F3948EE09FE00E945D47C6
:10E880002091411318161906DCF5211139C08EE0CC
:10E890009FE00E943B478A3041F08D3031F0682F75
:10E8A000CE010D960E94994A24C089899A89892BA4
:10E8B00001F1F09241136CEC79E0CE0101960E94D7
:10E8C000074CBE01635F7F4FCE0101960E94234B30
:10E8D000BC01CE0107960E94FF4BCE0107960E9415
:10E8E000988FCE0107960E94A34BCE0101960E94FD
:10E8F000A34B6AE070E080E090E00E943486BCCFD9
:10E90000211185C0E12CF12CDD24D39487E39DE017
:10E910000E945D471816190614F587E39DE00E94D2
:10E920003B478A3079F08D3069F090914113911115
:10E9300009C0682FCE010D960E94994A8FEFE81A00
:10E94000F80A06C089899A89892B11F0D09241135F
:10E9500065E070E080E090E00E943486D7CF64E10B
:10E9600070E080E090E00E943486EF28D1F1898940
:10E970009A89892BB1F180919713882361F161E124
:10E9800079E0CE0101960E94074CBE016F5F7F4F78
:10E99000CE010D960E940F85F82ECE0101960E94A1
:10E9A000A34BF11018C065ED79E08EE09FE00E9466
:10E9B0003E4DBE01635F7F4FCE0101960E94FF4B2B
:10E9C000BE016F5F7F4F8EE09FE00E947869CE01AD
:10E9D00001960E94A34B64E170E080E090E00E9409
:10E9E000348680914113811112C089899A89892BBB
:10E9F00071F464E670E080E090E00E9434860E944A
:10EA000090876FEB79E0C8010E94074C51C089895B
:10EA10009A89019709F046C06BED75E0CE01079623
:10EA20000E94074CBE01695F7F4FCE010D960E9488
:10EA30000F85811116C06EE577E0CE0101960E9428
:10EA4000074CBE016F5F7F4FCE010D960E940F8570
:10EA5000FF24F3948111F12CCE0101960E94A34B67
:10EA600001C0F12CCE0107960E94A34BFF20A1F01C
:10EA700040E050E0BE01635F7F4FCE0101960E94EF
:10EA8000D83EBE016F5F7F4F8AE292E10E94C04A8A
:10EA9000CE0101960E94A34B64E170E080E090E01B
:10EAA0000E943486BE01635F7F4FC8010E94EF4B16
:10EAB000CE010D960E94A34BC80162960FB6F89442
:10EAC000DEBF0FBECDBFDF91CF911F910F91FF90A1
:10EAD000EF90DF900895DF92EF92FF920F931F93D4
:10EAE000CF93DF93CDB7DEB72C970FB6F894DEBF88
:10EAF0000FBECDBF8C01109241136FEB79E0CE01B8
:10EB000007960E94074CE12CF12CDD24D39487E377
:10EB10009DE00E945D471816190614F58091411377
:10EB200081111EC087E39DE00E943B478A3059F067
:10EB30008D3049F0682FCE0107960E94994A8FEFD9
:10EB4000E81AF80A06C08B859C85892B11F0D092B3
:10EB500041136FE070E080E090E00E943486D7CFF0
:10EB600062E370E080E090E00E943486EF2851F08C
:10EB700087E39DE00E94FB4764E670E080E090E060
:10EB80000E9434868091411381110AC08B859C8537
:10EB9000892B31F46FEB79E0C8010E94074C18C053
:10EBA00080919713882371F0BE01695F7F4FCE017A
:10EBB00001960E94FF4BCE010196DDDACE0101964F
:10EBC0000E94A34BBE01695F7F4FC8010E94EF4BBB
:10EBD000CE0107960E94A34BC8012C960FB6F8945D
:10EBE000DEBF0FBECDBFDF91CF911F910F91FF9080
:10EBF000EF90DF90089581E080932D0580912E05A0
:10EC0000882341F088E080932A1360E08FE193E14C
:10EC10000C941057089580912E0581110FC081E04A
:10EC200080932E0580932D0580912513982F946055
:10EC3000909325138C600E94F66918C080912D0571
:10EC40008823A1F010922A1360E08FE193E10E94E3
:10EC5000105710922D05809125138B7F80932513DB
:10EC600088600E94F66910922E050895C4CF2F92F5
:10EC70003F924F925F926F927F928F929F92AF924C
:10EC8000BF92CF92DF92EF92FF920F931F93CF9399
:10EC9000DF93CDB7DEB766970FB6F894DEBF0FBE31
:10ECA000CDBF1C0181E79EE00E94168E40E855E230
:10ECB00060E070E081E79EE00E94816D64E670E0B4
:10ECC00080E090E00E9434868CED95E0A0E0B0E01A
:10ECD0008093750E9093760EA093770EB093780E76
:10ECE00064E670E080E090E00E9434868FEF8A87CF
:10ECF00081E08B8786E88C871D861E861F86188A92
:10ED0000198A89E78A8BC101880F991F9E8B8D8B89
:10ED1000C12CD12CE12CF12C412C512C320181E75A
:10ED20009EE0E214F3046CF5ED89FE89CE16DF0651
:10ED300044F50E942C4708974CF049E050E0BE0192
:10ED4000665F7F4F81E79EE00E94024765E070E0CA
:10ED500080E090E00E94348600E010E0812C912C4D
:10ED6000540181E79EE00E945D47892B31F4F4E075
:10ED70008F169104A104B104ACF50230110594F58D
:10ED800035C00E94168EE114F10409F47101C3012B
:10ED9000B2010E94B4AE4B015C01B701FF0C880BBD
:10EDA000990B0E94B4AE9B01AC01C501B4010E9455
:10EDB00004B166960FB6F894DEBF0FBECDBFDF91EB
:10EDC000CF911F910F91FF90EF90DF90CF90BF9068
:10EDD000AF909F908F907F906F905F904F903F90FB
:10EDE0002F9008958FEFC81AD80A99CF81E79EE037
:10EDF0000E945D47892B69F081E79EE00E943B47B6
:10EE0000E1E0F0E0EC0FFD1FE00FF11F80830F5FEA
:10EE10001F4F65E070E080E090E00E943486023091
:10EE2000110569F599818A85981329C09A818C8585
:10EE3000981325C0CE0103969C8B8B8B81E79EE0B7
:10EE40000E945D47892B31F494E089169104A10456
:10EE5000B1043CF509301105C1F48B8190E0982F85
:10EE600088272C81820F911D092E000CAA0BBB0B49
:10EE7000480E591E6A1E7B1EEFEFEE1AFE0AFFEFC8
:10EE80008F1A9F0AAF0ABF0A6CCF81E79EE00E94EB
:10EE90003B47EB89FC898193FC8BEB8B0F5F1F4F0A
:10EEA000CDCF0430110544F3D8CF2F923F924F922B
:10EEB0005F926F927F928F929F92AF92BF92CF920A
:10EEC000DF92EF92FF920F931F93CF93DF936C012A
:10EED000CFEAD5E089E0882E82E0982E09E810E19B
:10EEE000EE24E394F12C22E1222E312C33E1432E47
:10EEF000512C40E1642E712C51E1A52EB12C809152
:10EF00000702909108028E159F050CF4CAC021E0FB
:10EF1000C216D10439F4F80182AD93ADF4019183A6
:10EF200080830AC0F2E0CF16D10431F4F40180816D
:10EF30009181F80193AF82AFF401808191810097B4
:10EF400039F48A819B819093B8028093B70222C0E2
:10EF50008130910539F48A819B819093B602809328
:10EF6000B50218C08230910539F48A819B81909353
:10EF7000B4028093B3020EC0039761F48A819B812F
:10EF80009093B2028093B1026FEB79E082E792E155
:10EF90000E94794BF401819191914F018430910548
:10EFA00039F42A813B813093BA022093B90212C00E
:10EFB0008530910539F42A813B8130935A022093A0
:10EFC000590208C086309105C9F00EC08A309105FB
:10EFD00009F448C08531910589F42A813B81309339
:10EFE0005E0220935D023EC08730910579F72A8149
:10EFF0003B813093600220935F020AC08631910505
:10F0000039F42A813B8130935C0220935B022AC051
:10F010008731910539F52A813B812830310549F442
:10F020007092030260920202B0920102A09200026A
:10F0300019C02730310549F43092030220920202B0
:10F0400050920102409200020DC02630310551F469
:10F0500021E030E03093030220930202109201027B
:10F06000109200029C012B5031092A30310590F496
:10F070002A813B813093B2022093B10239E1389F5B
:10F08000B001399F700D112465547D4F82E792E1E4
:10F090000E94794B8FEFE81AF80A22960E5F1F4FF5
:10F0A0002ECFDF91CF911F910F91FF90EF90DF90C6
:10F0B000CF90BF90AF909F908F907F906F905F9018
:10F0C0004F903F902F9008954F925F926F927F9252
:10F0D0009F92AF92BF92CF92DF92EF92FF920F93E7
:10F0E0001F93CF93DF93982E8EE0A82EB12CEE24A1
:10F0F000EA9493E0F92ECFEFD3E0C12CD12C00E0BD
:10F1000010E0412C512C3201892D0E94EA8508170C
:10F11000190728F0C816D90618F46C0101C08C0133
:10F120008C179D0728F08E159F0518F47C0101C0EF
:10F13000EC01BC0180E090E00E94B2AE9B01AC010A
:10F14000C301B2010E943EB02B013C0165E070E0BA
:10F1500080E090E00E94348681E0A81AB108A1F610
:10F16000B6016E0D7F1D600F711FC60FD71FBE0148
:10F1700080E090E00E94B2AE9B01AC01C301B201FD
:10F180000E943DB020E030E040E251E40E9404B132
:10F19000DF91CF911F910F91FF90EF90DF90CF9073
:10F1A000BF90AF909F907F906F905F904F90089529
:10F1B0004F925F926F927F92AF92BF92CF92DF9207
:10F1C000FF920F931F93CF93DF9300D000D0CDB762
:10F1D000DEB75C0181E79EE00E94168E40E052ECB3
:10F1E00061E070E081E79EE00E94816D8CED95E02A
:10F1F000A0E0B0E08093750E9093760EA093770E0A
:10F20000B093780E64E670E080E090E00E9434866F
:10F21000C12CD12CF12CCA14DB040CF051C065E0D8
:10F2200070E080E090E00E94348600E010E0412C25
:10F23000512C3201F1100FC081E79EE00E945D4722
:10F24000892B31F485E148165104610471041CF4E2
:10F250000330110554F08FEFC81AD80A64E670E045
:10F2600080E090E00E943486D6CF81E79EE00E9445
:10F270005D47892B69F081E79EE00E943B47E1E012
:10F28000F0E0EC0FFD1FE00FF11F80830F5F1F4FB9
:10F2900065E070E080E090E00E9434860230110565
:10F2A0004CF089818B3B31F4FF24F3948A818A3AB4
:10F2B00009F0F12C8FEF481A580A680A780ABACF79
:10F2C0008F2D26960FB6F894DEBF0FBECDBFDF910F
:10F2D000CF911F910F91FF90DF90CF90BF90AF9093
:10F2E0007F906F905F904F9008951F93CF93DF931F
:10F2F000182FCDE9DCE0812F0E94EA85899399934C
:10F300006CE370E080E090E00E9434868CE0CD3EBB
:10F31000D80789F70E947D6B20E030E040EA50E496
:10F320000E9413AF20E030E040E85AE30E9413AFA0
:10F33000DF91CF911F9108954F925F926F927F92CC
:10F340008F929F92AF92BF92CF92DF92EF92FF92F5
:10F35000CF93DF93CDB7DEB768970FB6F894DEBFD3
:10F360000FBECDBF6B017C010E949087698B7A8BA9
:10F370008B8B9C8B84ED9DE00E94168E61E08091CA
:10F3800002020E94AE8560E0809100020E94AE857C
:10F390000E94A3970E94915B0E94AE5B6D877E875F
:10F3A0008F87988B0E940F864B015C016AE070E0AA
:10F3B00080E090E00E9434866CED79E08EE192E18D
:10F3C0000E94794B20E030E04AE754E4C701B601DF
:10F3D0000E9413AF6D8B7E8B8F8B988F412C512C9D
:10F3E0003201C12CD12C7601C701B6010E94B4AE06
:10F3F0002D893E894F89588D0E94AEAE87FF85C109
:10F400000E94908729893A894B895C89621B730B1A
:10F41000840B950B0E94B2AE20E030E04AE754E442
:10F420000E9404B1AB01BC0123E0CE0101960E9411
:10F43000A84BBE016F5F7F4F88E192E10E94C04AF6
:10F44000CE0101960E94A34B0E94AE5B6B017C0132
:10F450000E940F869B01AC01281939094A095B09F2
:10F4600049015A0131ED831637E09306A104B10436
:10F470000CF441C020E030E0A901C701B6010E94B0
:10F48000F3B118165CF426EA3BE944EC5BE3C701F0
:10F49000B6010E94AEAE87FF0BC02DC026EA3BE945
:10F4A00044EC5BEBC701B6010E94F3B118161CF1E6
:10F4B000C501B40128EE33E040E050E00E94E0AF27
:10F4C000CA01B9010E94B4AE4B015C012D853E8595
:10F4D0004F855889C701B6010E943DB020E030E059
:10F4E0004AE754E40E9413AFA50194010E9404B1BD
:10F4F0004B015C0103C0812C912C540168E172E145
:10F50000CE0101960E94FF4B6BED75E0CE01019696
:10F510000E940C4BBC0188E192E10E948E4BCE010F
:10F5200001960E94A34B23E0B701A601CE010196EC
:10F530000E94A84BBE016F5F7F4FCE0107960E94CD
:10F54000FF4B68EC78E0CE0107960E940C4BBC01A3
:10F5500082E192E10E948E4BCE0107960E94A34B5E
:10F56000CE0101960E94A34B22E0B501A401CE0179
:10F5700007960E94A84B69EF78E0CE0101960E94A1
:10F58000074C68E172E1CE0101960E94234B6AEFBD
:10F5900079E00E940C4B62E172E10E94234B6EED18
:10F5A00075E00E940C4BBE01695F7F4F0E94234BA8
:10F5B00069ED75E00E940C4BBC018EE192E10E9466
:10F5C000BA4ACE0101960E94A34BCE0107960E9433
:10F5D000A34B20E030E0A901C501B4010E94F3B1C2
:10F5E00087FD06C068ED7BE082E192E10E94AC4AB3
:10F5F00022E0B501A401CE0101960E94A84BBE01F4
:10F600006F5F7F4FCE0107960E94FF4B69ED75E05B
:10F61000CE0107960E940C4BBC0182E192E10E9450
:10F62000BA4ACE0107960E94A34BCE0101960E94D2
:10F63000A34B6EE172E1CE0101960E94FF4BCE0119
:10F6400001960E94BB70CE0101960E94A34BC3019C
:10F65000B20125E030E040E050E00E94E0AF672BCF
:10F66000682B692B21F56CE772E1CE0101960E94AF
:10F67000F74B45E050E060E070E0CE0101960E945B
:10F68000C48FCE0101960E94A34B62E172E1CE01CC
:10F6900001960E94FF4B45E050E06FEF7FEFCE01F7
:10F6A00001960E947C8DCE0101960E94A34B6FEBC8
:10F6B00079E08EE192E10E94794B65E070E080E0B4
:10F6C00090E00E9434860E9490876B017C0129891A
:10F6D0003A894B895C89C21AD30AE40AF50A0E9466
:10F6E000AE5B6D877E878F87988B0E940F864B015C
:10F6F0005C016AE070E080E090E00E9434863FEFB9
:10F70000431A530A630A730A6FCE60E080910202C3
:10F710000E94AE8568960FB6F894DEBF0FBECDBFCF
:10F72000DF91CF91FF90EF90DF90CF90BF90AF909F
:10F730009F908F907F906F905F904F9008954F9221
:10F740005F926F927F92AF92BF92CF92DF92EF92D1
:10F75000FF920F931F93CF93DF93CDB7DEB7EA9756
:10F760000FB6F894DEBF0FBECDBFF82E6FEB79E079
:10F77000CE01C5960E94074C8E010B5E1F4F6F2D68
:10F78000C8010E94E55618870F831D821E821982C8
:10F7900089E08A8381E08B838C831C8A1B8ACE015B
:10F7A00001960E94F253CE0101960E948653CE012B
:10F7B00001960E94B7520E8110E00330110509F442
:10F7C0006EC162E772E1CE01C5960E94344B6FEBC9
:10F7D00079E08EE192E10E94794BBE016B5C7F4F34
:10F7E000CE0183960E94FF4B4AE050E060E070E05B
:10F7F000CE0183960E94C48FCE0183960E94A34BB4
:10F8000061E080E00E94076A6DE07AE0CE01C59673
:10F810000E94794B8FE0A82E8CE0B82ECC24C394A4
:10F82000D12CE12CF12CE016F1060CF0EEC06E2D7F
:10F83000CE0101960E944852F501219131914191EA
:10F8400051915F010E943EB02B013C0120E030E06D
:10F850004CEF52EC0E94AEAE87FF24C0B601CE0141
:10F8600089960E942D506AEA77E0CE0183960E9425
:10F87000074CBE01675D7F4FCE0183960E94234BEC
:10F880006EEF79E00E940C4BBC018EE192E10E9488
:10F89000BA4ACE0183960E94A34BCE0189960E945C
:10F8A000A34B48C022E0B301A201CE018F960E9473
:10F8B000A84BB601CE0189960E942D506AEA77E0E6
:10F8C000CE0183960E94074CBE01675D7F4FCE013B
:10F8D00083960E94234B64ED7AE00E940C4BBE019C
:10F8E000615D7F4F0E94234BBC0182E192E10E9447
:10F8F0008E4BCE0183960E94A34BCE0189960E9427
:10F90000A34BCE018F960E94A34B62E172E1CE0120
:10F9100083960E94FF4B68ED7BE0CE0183960E94A8
:10F920000C4BBC018EE192E10E94BA4ACE01839653
:10F930000E94A34B0130110559F4E114F10409F0C0
:10F940005DC06EE172E1CE01C5960E948E4B56C03D
:10F950000230110511F522E0B301A201CE01839618
:10F960000E94A84BBE016D5D7F4FCE0189960E941B
:10F97000FF4B68ED7BE0CE0189960E940C4BBC01E9
:10F98000CE01C5960E94BA4ACE0189960E94A34B29
:10F99000CE0183960E94A34B31C00330110571F153
:10F9A00062E172E1CE0183960E94FF4B44E150E098
:10F9B0006FEF7FEFCE0183960E947C8DCE01839600
:10F9C0000E94A34B66E779E0CE0183960E94074C24
:10F9D000CE0183960E94F88DCE0183960E94A34BA0
:10F9E00080912E05882351F080912D05882331F0D8
:10F9F00060ED77E080E090E00E943486FFEFEF1A40
:10FA0000FF0A8FEFC81AD80A0ECFCE01C5960E9402
:10FA1000F9498EE192E10E94F94901151105C9F4F5
:10FA20006FE572E18EE192E10E94344B64E572E190
:10FA3000CE0183960E94F74B4AE050E06FEF7FEFD4
:10FA4000CE0183960E947C8DCE0183960E94A34BAB
:10FA5000EBC0043011050CF000C1BE016B5C7F4FA0
:10FA6000CE0183960E94FF4B4AE050E06FEF7FEF9C
:10FA7000CE0183960E947C8DCE0183960E94A34B7B
:10FA800066E779E0CE0183960E94074CCE0183960B
:10FA90000E94F88DCE0183960E94A34BDEC06AE0DF
:10FAA0007AE0CE01C5960E94794BBE016B5C7F4F18
:10FAB000CE0183960E94FF4B4AE050E060E070E088
:10FAC000CE0183960E94C48FCE0183960E94A34BE1
:10FAD0006FEB79E08EE192E10E94794B6EE172E189
:10FAE000CE01C5960E948E4B00E010E0602FCE0143
:10FAF00001960E9448526B017C0122E0AB01BC01DF
:10FB0000CE0183960115110551F40E94A84BBE0148
:10FB10006D5D7F4F8FE193E10E94654C18C00E949C
:10FB2000A84BBE016D5D7F4FCE0189960E94FF4BB1
:10FB300068ED7BE0CE0189960E940C4BBC01CE01A2
:10FB4000C5960E94BA4ACE0189960E94A34BCE0167
:10FB500083960E94A34B22E0B701A601CE018396B3
:10FB60000E94A84BBE016D5D7F4FCE0189960E9419
:10FB7000FF4B68ED7BE0CE0189960E940C4BBC01E7
:10FB80008EE192E10E94BA4ACE0189960E94A34B6F
:10FB9000CE0183960E94A34B0F5F1F4F03301105C8
:10FBA00009F0A4CFCE01C5960E94F949BE016B5C55
:10FBB0007F4FCE0183960E94FF4B4AE050E06FEFEB
:10FBC0007FEFCE0183960E947C8DCE0183960E94AA
:10FBD000A34B66E779E0CE0183960E94074CCE01E5
:10FBE00083960E94F88DCE0183960E94A34B8EE1EE
:10FBF00092E10E94F94960E17AE0CE0183960E9489
:10FC0000074C6EE172E1CE0183960E94234B6AE1BC
:10FC10007AE00E940C4BBC018EE192E10E948E4B77
:10FC2000CE0183960E94A34BCE01C5960E94A34BA2
:10FC3000EA960FB6F894DEBF0FBECDBFDF91CF912D
:10FC40001F910F91FF90EF90DF90CF90BF90AF90FA
:10FC50007F906F905F904F9008956AE17AE08EE117
:10FC600092E10E94AC4AE0CF0F931F93CF93DF93B2
:10FC70008C011092431310924213C0914213D09101
:10FC80004313C832D10584F48091B902A3D7FE0191
:10FC9000EE0FFF1FE356F34F918380832196D0939D
:10FCA0004313C0934213E9CF0E947D6B20E030E004
:10FCB00040EA50E40E9413AF20E030E040E85AE30D
:10FCC0000E9413AF0430110569F420E030E040E6F3
:10FCD00050E40E9413AF9B01AC0160E070E080E84B
:10FCE00090E40FC00A30110579F420E030E040E6DE
:10FCF00050E40E9413AF9B01AC0160E070E080E231
:10FD000091E40E943DB003C060E070E0CB01DF9160
:10FD1000CF911F910F910895AF92BF92CF92DF9232
:10FD2000EF92FF920F931F93CF93DF93CDB7DEB780
:10FD3000A4970FB6F894DEBF0FBECDBF80914413D9
:10FD4000882319F01092441377C580914012909146
:10FD50004112049708F03FC060EF77E0CE010196B2
:10FD60000E94074CBE016F5F7F4F86E392E157D63A
:10FD7000182FCE0101960E94A34B112361F161E07F
:10FD800070E08CE392E10E94594A80330CF4845E67
:10FD90006AE270E0681B710987FD7395CE010196D8
:10FDA0000E942D50BE016F5F7F4F8CE392E10E9455
:10FDB000C04ACE0101960E94A34B6CE372E18AE235
:10FDC00092E10E948E4B8CE392E10E94EE49CB01BE
:10FDD0000E94D70A31C561E577E0CE0101960E9405
:10FDE000074CBE016F5F7F4F86E392E118D6182F54
:10FDF000CE0101960E94A34B112309F482C36DE248
:10FE00007AE0CE0101960E94074CCE0101960E9435
:10FE1000BB70CE0101960E94A34B69E37AE0CE014C
:10FE200007960E94074C63E173E1CE0107960E949A
:10FE3000234BBC01CE0101960E94FF4BCE010196DF
:10FE40000E94BB70CE0101960E94A34BCE01079683
:10FE50000E94A34B6091430270914402809145023D
:10FE6000909146020E94B4AE20E030E048EC52E4AB
:10FE70000E9404B1AB01BC0122E0CE0107960E94B2
:10FE8000A84B6FE47AE0CE010D960E94074CBE01AC
:10FE9000695F7F4FCE010D960E94234B62E578E0AB
:10FEA0000E940C4BBC01CE0101960E94FF4BCE017B
:10FEB00001960E94BB70CE0101960E94A34BCE0119
:10FEC0000D960E94A34BCE0107960E94A34B409132
:10FED0003F0250914002609141027091420224E041
:10FEE000CE0107960E94A84B64E67AE0CE010D96FB
:10FEF0000E94074CBE01695F7F4FCE010D960E94A4
:10FF0000234BBC01CE0101960E94FF4BCE0101960E
:10FF10000E94BB70CE0101960E94A34BCE010D96AC
:10FF20000E94A34BCE0107960E94A34B409133023F
:10FF300050913402609135027091360222E0CE0178
:10FF400007960E94A84B40912B0250912C02609181
:10FF50002D0270912E0223E0CE010D960E94A84B37
:10FF600040913702509138026091390270913A0203
:10FF700022E0CE0143960E94A84B40912F0250915F
:10FF80003002609131027091320223E0CE01499635
:10FF90000E94A84B61E87AE0CE014F960E94074C80
:10FFA000BE01675E7F4FCE014F960E94234B66E9EC
:10FFB0007AE00E940C4BBE016D5E7F4F0E94234B86
:10FFC00069E97AE00E940C4BBE01635F7F4F0E949B
:10FFD000234B66E97AE00E940C4BBE01695F7F4FBC
:10FFE0000E94234B6FE97AE00E940C4BBC01CE01CA
:10FFF00001960E94FF4BCE0101960E94BB70CE017C
:020000021000EC
:1000000001960E94A34BCE014F960E94A34BCE01B6
:1000100049960E94A34BCE0143960E94A34BCE016A
:100020000D960E94A34BCE0107960E94A34B6BEA4C
:1000300072E1CE0149960E94F74BF090B8100F2D57
:100040000F2C000C110B01151105A1F52091B91011
:100050003091BA104091BB105091BC1060E070E03C
:1000600080EA90E40E9404B1AB01BC0122E0CE0121
:1000700001960E94A84B65E878E0CE0107960E94A1
:10008000074CBE016F5F7F4FCE0107960E94234B46
:1000900064ED78E00E940C4BBC01CE0149960E94B1
:1000A000BA4ACE0107960E94A34BCE0101960E9448
:1000B000A34B09C00130110531F46DE972E1CE01A5
:1000C00049960E946A4AC8010297029738F58F2D17
:1000D0009AE08902B0011124CE0101960E942D50B0
:1000E00064EA7AE0CE0107960E94074CBE016F5F7A
:1000F0007F4FCE0107960E94234B6DEC78E00E9463
:100100000C4BBC01CE0149960E94BA4ACE0107961B
:100110000E94A34BCE0101960E94A34B043011050F
:1001200019F46BE872E105C00530110534F063E89D
:1001300072E1CE0149960E946A4ABE01675E7F4F16
:10014000CE0101960E94FF4BCE0101960E94BB702A
:10015000CE0101960E94A34B60EB7AE0CE01499656
:100160000E94794B8091B5106091B6107091B710D4
:1001700083300CF04FC3CE0101960E942D506BEAE4
:100180007AE0CE0107960E94074CBE016F5F7F4F59
:10019000CE0107960E94234B62EB7BE00E940C4B42
:1001A000BC01CE0149960E94BA4ACE0107960E9430
:1001B000A34BCE0101960E94A34BBE01675E7F4F09
:1001C000CE0101960E94FF4BCE0101960E94BB70AA
:1001D000CE0101960E94A34B4091BD105091BE10DC
:1001E0006091BF107091C01022E0CE0107960E946E
:1001F000A84B60EC7AE0CE010D960E94074CBE0140
:10020000695F7F4FCE010D960E94234B66ED7AE029
:100210000E940C4BBC01CE0101960E94FF4BCE0107
:1002200001960E94BB70CE0101960E94A34BCE01A5
:100230000D960E94A34BCE0107960E94A34B4091BE
:10024000D3105091D4106091D5107091D61022E047
:10025000CE0107960E94A84B6DED7AE0CE010D9677
:100260000E94074CBE01695F7F4FCE010D960E9430
:10027000234B6DEC75E00E940C4BBC01CE01019646
:100280000E94FF4BCE0101960E94BB70CE010196E9
:100290000E94A34BCE010D960E94A34BCE01079660
:1002A0000E94A34B89E0C82E82E0D82E01E010E026
:1002B00099E1F92E80910702909108028017910729
:1002C0000CF44DC0F601A190B1906F01B501CE01C3
:1002D00007960E942D50B801CE010D960E942D5018
:1002E00060EF7AE0CE0143960E94074CBE01635F47
:1002F0007F4FCE0143960E94234B68EF7AE00E9425
:100300000C4BBE01695F7F4F0E94234B6BEF7AE07D
:100310000E940C4BFA9CB001FB9C700D112465549B
:100320007D4F0E940C4BBC01CE0101960E94FF4BF9
:10033000CE0101960E94BB70CE0101960E94A34B94
:10034000CE0143960E94A34BCE010D960E94A34B73
:10035000CE0107960E94A34B0F5F1F4FABCF80913A
:10036000FF1090910011892B71F461E07BE0CE01C8
:1003700001960E94074CCE0101960E94BB70CE01EF
:1003800001960E94A34B8091FF109091001101975C
:1003900071F460E17BE0CE0101960E94074CCE0132
:1003A00001960E94BB70CE0101960E94A34B8091E2
:1003B000FF1090910011029771F46AE17BE0CE0189
:1003C00001960E94074CCE0101960E94BB70CE019F
:1003D00001960E94A34B6091290270912A02CE01DE
:1003E00007960E942D506CE27BE0CE010D960E9494
:1003F000074CBE01695F7F4FCE010D960E94234BD3
:10040000BC01CE0101960E94FF4BCE0101960E94D5
:10041000BB70CE0101960E94A34BCE010D960E94A7
:10042000A34BCE0107960E94A34B409150025091DE
:100430005102609152027091530222E0CE01079660
:100440000E94A84B69E47BE0CE010D960E94074C08
:10045000BE01695F7F4FCE010D960E94234B6BED6D
:1004600075E00E940C4BBC01CE0101960E94FF4B2F
:10047000CE0101960E94BB70CE0101960E94A34B53
:10048000CE010D960E94A34BCE0107960E94A34B6E
:100490004091550250915602609157027091580256
:1004A00022E0CE0107960E94A84B69E57BE0CE01D1
:1004B0000D960E94074CBE01695F7F4FCE010D96DD
:1004C0000E94234B6BED75E00E940C4BBC01CE01EA
:1004D00001960E94FF4BCE0101960E94BB70CE0197
:1004E00001960E94A34BCE010D960E94A34BCE0114
:1004F00007960E94A34B10925402CE0149960E9487
:10050000A34B80914012909141128330910508F0E5
:100510006FC18130910541F460E070E08CE392E1BD
:100520000E94594AE82E57C0029709F054C060EF64
:1005300077E0CE0101960E94074CBE016F5F7F4FAE
:1005400086E392E16CD2182FCE0101960E94A34B54
:10055000112309F440C061E070E08CE392E10E9455
:10056000594A682FCE0101960E94D74BBE016F5F9A
:100570007F4F8AE292E10E94C04ACE0101960E941A
:10058000A34B60E070E08CE392E10E94594AE82EB0
:10059000809197138823F9F069E67BE0CE010196FC
:1005A0000E94074C6CE372E1CE0101960E94234B3E
:1005B00068ED7BE00E940C4BBC018EE09FE00E9446
:1005C000654CCE0101960E94A34B6AE272E18EE077
:1005D0009FE00E9478698E2DEE0C990B0E94D0B599
:1005E000892BB1F00E94FB750E948D3E68ED7BE087
:1005F000CE0101960E94074C4AE050E060E070E0B6
:10060000CE0101960E946990CE0101960E94A34BF3
:100610006CE372E1CE0107960E94FF4B60E070E050
:10062000CE0107960E94594A823409F474C0D4F46A
:10063000803309F490C07CF4833209F483C08A3299
:1006400009F0A9C062E87BE08CE392E10E94794B5B
:100650008FEF9FEF8EC0813309F48EC0813409F48F
:100660004FC099C0813609F44BC034F4833409F487
:100670005DC0843449F08FC0833609F457C00CF450
:100680004AC0843609F087C080912E1290912F12B3
:10069000892B09F49FC061E070E0CE0107960E94AB
:1006A000594A182F80919713882361F06FE67BE0F9
:1006B0008EE09FE00E943E4D6AE272E18EE09FE094
:1006C0000E94786910330CF4145E6AE270E0611BDA
:1006D000710917FD7395CE0101960E942D50BE0140
:1006E0006F5F7F4F8AE292E10E94C04ACE0101967D
:1006F0000E94A34B8AE292E10E94EE49CB0139C0ED
:1007000066E77BE08CE392E10E94794B8091070CD5
:100710009091080C2EC069E77BE08CE392E10E9487
:10072000794B1092430C8CEF9FEF23C06CE77BE07A
:100730008CE392E10E94794B81E08093430C8DEF32
:100740009FEF17C06FE77BE08CE392E10E94794B4B
:100750008EEF9FEF0EC068E579E08AE292E10E9499
:10076000794B68E579E08CE392E10E94794B80E077
:1007700090E00E94D70A2EC063E87BE08AE292E113
:100780000E94794B63E87BE08CE392E10E94794B15
:1007900081E090E0EECFBE01695F7F4F8AE292E197
:1007A0000E948E4B60E070E08AE292E10E94594A1A
:1007B000082E000C990BC0970A9738F48AE292E150
:1007C0000E94EE49CB010E94D70A64E670E080E007
:1007D00090E04AD2CE0107960E94A34BA1D360932A
:1007E000390C70933A0C80933B0C90933C0C02C0F4
:1007F0000E94972495D36093390C70933A0C8093A0
:100800003B0C90933C0C6FEB79E08CE392E10E94FF
:10081000794B12C0CE0101960E942D5065E87BE015
:10082000CE0107960E94074CBE016F5F7F4FCE013D
:1008300007960E94234BB4CCA4960FB6F894DEBF63
:100840000FBECDBFDF91CF911F910F91FF90EF9021
:10085000DF90CF90BF90AF90089590E0FC0131976A
:10086000E231F10508F04EC08827E855FF4F8F4F61
:100870000C9478B3809180008F7703C080918000C2
:100880008F7D80938000089580918000877FF9CFCD
:1008900084B58F7702C084B58F7D84BD0895809123
:1008A000B0008F7703C08091B0008F7D8093B0003F
:1008B0000895809190008F7707C0809190008F7D80
:1008C00003C080919000877F80939000089580916D
:1008D000A0008F7707C08091A0008F7D03C080911A
:1008E000A000877F8093A0000895809120018F77DA
:1008F00007C0809120018F7D03C080912001877FF8
:10090000809320010895CF93DF93FC0124813581EA
:10091000232B71F0FB01DC01CD91DC9160817181B1
:10092000CE010E9427B6009719F08C1B9D0B02C0C8
:100930008FEF9FEFDF91CF9108950F931F93CF9388
:10094000DF93FC01C481D581209719F4FB0110824B
:1009500011C0415051094C175D0708F4EA018B01A1
:10096000FC0160817181AE01C8010E9418B6C00F00
:10097000D11F1882DF91CF911F910F910895AF92EF
:10098000BF92CF92DF92EF92FF920F931F93CF937C
:10099000DF93FC0124813581FB014481558189016C
:1009A000041B150B4115510551F12115310539F184
:1009B0002417350720F10217130718F08901015099
:1009C00011097B01FC01A080B180C501DFEFCFEFF1
:1009D0006501C00ED11EC816D906A0F0F7016081CE
:1009E00071810E9427B6009769F09C012A193B0982
:1009F0000217130710F0D22FC32F0196ECCF8FEF01
:100A00009FEF02C08D2F9C2FDF91CF911F910F91EF
:100A1000FF90EF90DF90CF90BF90AF900895FB01D3
:100A200044815581FC01248135812417350778F0F4
:100A300080819181009759F0FB016081718161157E
:100A4000710529F00E940AB621E0892B09F020E007
:100A5000822F0895CF93DF93C0913612D091371231
:100A6000209751F08881882339F0082E000C990BCB
:100A70000E94E9B58993F6CFDF91CF910895FC01EB
:100A8000A089B1898C91A689B78982FD0FC09C91FC
:100A9000818D8F5F8F73228D821749F0218DDF0149
:100AA000A20FB11D5D969C93818F08958C9108953E
:100AB000CF93DF93282F30E0F901EA56FC4E849162
:100AC000F901E05BFC4ED491F901E65FFC4EC49164
:100AD000CC2389F08111C1DEEC2FF0E0EE0FFF1F77
:100AE000E051FD4EA591B491EC91ED2381E090E0B1
:100AF00021F480E002C080E090E0DF91CF91089582
:100B00001F93CF93DF93282F30E0F901EA56FC4E74
:100B10008491F901E05BFC4ED491F901E65FFC4E53
:100B2000C491CC23B9F0162F811197DEEC2FF0E0A1
:100B3000EE0FFF1FEA52FD4EA591B4919FB7F894B6
:100B4000111104C08C91D095D82302C0EC91DE2BFA
:100B5000DC939FBFDF91CF911F910895CF93DF93D7
:100B600090E0FC01E05BFC4E2491FC01E65FFC4E52
:100B70008491882361F190E0880F991FFC01E4546F
:100B8000FD4EC591D491FC01EA52FD4EA591B49160
:100B9000611109C09FB7F8948881209582238883CA
:100BA000EC912E230BC0623061F49FB7F8948881DA
:100BB000322F309583238883EC912E2B2C939FBF6B
:100BC00006C08FB7F894E8812E2B28838FBFDF9162
:100BD000CF910895863308F0865390917B00282F9B
:100BE0002870977F922B90937B0020912C0590E4A6
:100BF000299F900111248770822B80937C00809123
:100C00007A00806480937A0080917A0086FDFCCF20
:100C1000809178002091790090E0922B08953FB761
:100C2000F8948091491390914A13A0914B13B0917D
:100C30004C1326B5A89B05C02F3F19F00196A11DA6
:100C4000B11D3FBFBA2FA92F982F8827820F911D62
:100C5000A11DB11DBC01CD0142E0660F771F881FA9
:100C6000991F4A95D1F708958F929F92AF92BF92A4
:100C7000CF92DF92EF92FF926B017C01D0DF4B01AC
:100C80005C01C114D104E104F104E9F0C8DFDC0126
:100C9000CB0188199909AA09BB09883E9340A1058F
:100CA000B10578F321E0C21AD108E108F10888EE15
:100CB000880E83E0981EA11CB11CC114D104E1046C
:100CC000F10421F7DECFFF90EF90DF90CF90BF903F
:100CD000AF909F908F900895FF920F931F93CF93A3
:100CE000DF93CDB7DEB72B970FB6F894DEBF0FBEFC
:100CF000CDBF81E79EE09AD740E855E260E070E022
:100D000081E79EE00E94816D64E670E080E090E003
:100D1000ABDF8CED95E0A0E0B0E08093750E909392
:100D2000760EA093770EB093780E64E670E080E0C4
:100D300090E09ADF8FEF898381E08A8386E88B8356
:100D40001C821D821E821F82188689E7898781E79F
:100D50009EE00E94FB4762E370E080E090E084DF69
:100D600081E79EE00E942C4708974CF049E050E054
:100D7000BE016F5F7F4F81E79EE00E94024762E302
:100D800070E080E090E070DF81E79EE00E945D47C8
:100D9000892B01F181E79EE00E942C47089784F49B
:100DA00065E070E080E090E05FDF00E010E0F12CB3
:100DB00081E79EE00E945D4702301105A4F50CC05A
:100DC00049E050E0BE016F5F7F4F81E79EE00E94E7
:100DD0000247E6CFF12C27C081E79EE00E945D47E5
:100DE000892B99F465E070E080E090E03DDF02300F
:100DF0001105F1F69A8589819813DACF9B858B814D
:100E00009813D6CFFF24F394D3CF81E79EE00E94BE
:100E10003B47EAE0F0E0EC0FFD1FE00FF11F80839D
:100E20000F5F1F4FDFCF62E370E080E090E01CDFD8
:100E300081E79EE0FBD68F2D2B960FB6F894DEBF90
:100E40000FBECDBFDF91CF911F910F91FF900895FD
:100E5000CF93DF930E94FB4F1092241380912813AD
:100E6000823018F098E090932413909129139923DD
:100E700039F0813029F48091241384608093241305
:100E800062E370E080E090E0EFDE60912A138FE192
:100E900093E10E94105768EE73E080E090E0E4DE9A
:100EA00060E38FE193E10E942357CBE4D6E4CE01C7
:100EB0000197F1F760E38FE193E10E9423572197B7
:100EC000F1F760E38FE193E10E94235783E592E01D
:100ED0000197F1F760E28FE193E10E94235780913F
:100EE000241380620E94F66984E0809325138CE0CD
:100EF0000E94F66981E00E94F669CBE3DFE1CE0152
:100F00000197F1F782E08093261386E00E94F6694C
:100F100082E00E94F6692197F1F7DF91CF91089561
:100F20002FB7F89460914513709146138091471341
:100F3000909148132FBF08952F923F924F925F9246
:100F40006F927F928F929F92AF92BF92CF92DF92D9
:100F5000EF92FF920F931F93CF93DF93CDB7DEB73E
:100F600066970FB6F894DEBF0FBECDBF7C016D8BC8
:100F70007E8B5C8B4B8B19016FEB79E00E94074CE9
:100F80008EE1882E912C8E010F5F1F4F2101032CC3
:100F9000000C66087708CD88DE88A12CB12CA2143D
:100FA000B3040CF07BC0B501CE010D960E942D500C
:100FB000BE01635F7F4FCE0107960E94FF4B66E143
:100FC00077E0CE0107960E940C4B6B897C890E94CA
:100FD000234BB6010E94234BBC01C8010E94FF4B6A
:100FE00040ED57E060E070E0C80186D5C8010E947E
:100FF000A34BCE0107960E94A34BCE010D960E94F3
:10100000A34B44E150E061E070E0C8010E949B54B2
:101010000E151F0521F0B801C7010E94C04AC80182
:101020000E94A34BF70184819581892BA9F160E08F
:1010300070E0C7010E94594A082E000C990BC09716
:101040000A9740F4C7010E94EE49641575058605AC
:1010500097054CF066E779E0F701808191810E9465
:10106000FAB5892B59F481E0FFEFAF1ABF0A96E079
:10107000C90ED11C882309F492CF15C06CED73E121
:10108000C8010E94F74B40ED57E060E070E0C801F6
:1010900033D5C8010E94A34B80E0E6CFE1E08E1A71
:1010A000910809F078CFC70166960FB6F894DEBFB5
:1010B0000FBECDBFDF91CF911F910F91FF90EF90A9
:1010C000DF90CF90BF90AF909F908F907F906F9068
:1010D0005F904F903F902F900895CF93DF93EC0156
:1010E000483085E058076105710509F441C108F0F1
:1010F0008DC0493481E058076105710509F43BC191
:10110000E0F5443481E058076105710509F424C114
:10111000E8F4413481E058076105710509F413C111
:1011200038F4403451406105710509F409C135C1F5
:10113000423481E058076105710509F407C1433461
:1011400051406105710509F404C127C1463481E0AD
:1011500058076105710509F405C108F400C1473459
:1011600081E058076105710509F4FFC0483451401A
:101170006105710509F4FCC010C1423085E05807D3
:101180006105710509F4E2C0E8F4443781E05807CD
:101190006105710509F4F5C038F442375140610525
:1011A000710509F4F1C0F9C0411585E058076105E2
:1011B000710509F4C5C0413055406105710509F458
:1011C000C2C0EBC0453085E058076105710509F4E0
:1011D000C6C070F4433085E058076105710509F415
:1011E000B8C0443055406105710509F4B5C0D5C09B
:1011F000463085E058076105710509F4B3C04730F2
:1012000055406105710509F4B0C0C7C04D3B82E48B
:1012100058078FEF6807710509F4BCC008F045C096
:101220004F3E80E158078FEF6807710509F49DC0B4
:10123000E8F4423385E058076105710509F4A4C05C
:1012400038F4493055406105710509F494C0A5C0D2
:10125000443385E058076105710509F492C04D3F9C
:1012600052406F4F710509F48FC097C04D3D82E227
:1012700058078FEF6807710509F483C038F4473EBB
:1012800058416F4F710509F46AC087C04F3C80E335
:1012900058078FEF6807710509F45EC0473C584353
:1012A0006F4F710509F464C078C0473988E6580764
:1012B0008FEF6807710509F446C000F54D3A82E5E5
:1012C00058078FEF6807710509F461C030F4453B9A
:1012D0005A446F4F7105A1F160C0453A8AE558073D
:1012E0008FEF6807710509F446C04D3952466F4FBC
:1012F000710509F052C066E779E051C0473588EAC8
:1013000058078FEF68077105C9F168F445388AE717
:1013100058078FEF6807710529F1473658496F4F15
:101320007105A1F03AC04F3480EB58078FEF680782
:10133000710579F04D33524C6F4F710529F12DC075
:1013400068E579E02CC063E87BE029C060E87BE0D9
:1013500026C06DE77BE023C06AE77BE020C067E73B
:101360007BE01DC06EE87BE01AC06BEB79E017C034
:1013700060E97BE014C062E97BE011C060EF77E0D8
:101380000EC060E476E00BC06DEC78E008C061E16F
:1013900079E005C064E97BE002C06FEB79E0CE0143
:1013A0000E94074CCE01DF91CF9108954F925F923A
:1013B0006F927F928F929F92AF92BF92EF92FF9225
:1013C0000F931F93CF93DF93CDB7DEB762970FB61E
:1013D000F894DEBF0FBECDBF7C015B018DE593E1CC
:1013E0000E94E71D892B31F46FEB79E0C7010E9461
:1013F000074C28C1409161135091621360916313AF
:1014000070916413CE01079668DE8091971388234C
:1014100059F166E97BE0CE0101960E94074CBE01BE
:10142000695F7F4FCE0101960E94234B66E177E012
:101430000E940C4BBC018EE09FE00E94654CCE01E7
:1014400001960E94A34B40916113509162136091E9
:1014500063137091641320E18EE09FE00E94AC4C16
:101460008EE09FE00E94746960E070E0CE01079614
:101470000E94594A182F8A3211F01092441350DDFD
:101480006093390C70933A0C80933B0C90933C0C16
:101490006FEB79E0CE010D960E94074C812F110F62
:1014A000990BC0970A9708F05CC0CE0107960E947E
:1014B000EE4963307105810591050CF094C001E09F
:1014C00010E082E0982E0A151B050CF08CC06CE22F
:1014D00071E080E090E0C8DB9092B70F1092BA0FF5
:1014E000412C512C32018DE493E10E94E71D892BA0
:1014F00041F48EE1481651046104710409F08CC076
:101500001CC08EE14816510461047104B1F0409191
:101510005113509152136091531370915413CE0193
:101520000196DBDDBE016F5F7F4FCE010D960E94FD
:10153000C04ACE0101960E94A34B89899A89892BC2
:1015400039F0BE01635F7F4FCE0107960E94BA4A11
:101550000F5F1F4F6FEB79E0CE010D960E94794B24
:10156000B2CF6CE271E080E090E07EDB82E08093BD
:10157000B70F1092BA0F812C912C54018DE493E196
:101580000E94E71D892B41F48EE188169104A10485
:10159000B10409F04CC01CC08EE188169104A1046E
:1015A000B104B1F040915113509152136091531313
:1015B00070915413CE01019690DDBE016F5F7F4F95
:1015C000CE010D960E94C04ACE0101960E94A34B07
:1015D00089899A89892B39F0BE01635F7F4FCE01DB
:1015E00007960E94BA4A64E670E080E090E03CDB37
:1015F00082E08093B70F1092BA0FBE01695F7F4FF0
:10160000C7010E94EF4BCE010D960E94A34BCE0165
:1016100007960E94A34B16C06EE170E080E090E058
:1016200023DB8FEF481A580A680A780A5CCF6EE10C
:1016300070E080E090E018DB8FEF881A980AA80A23
:10164000B80A9CCFC70162960FB6F894DEBF0FBEF2
:10165000CDBFDF91CF911F910F91FF90EF90BF9081
:10166000AF909F908F907F906F905F904F90089574
:10167000AF92BF92CF92DF92EF92FF920F931F93A0
:10168000CF93DF93CDB7DEB72C970FB6F894DEBFBC
:101690000FBECDBF7C015B010E940398182F811102
:1016A00006C06FEB79E0C7010E94074C99C08A32EF
:1016B00011F01092441334DC6093390C70933A0C9F
:1016C00080933B0C90933C0C612FCE0107960E94B7
:1016D000D74B812F012E000C990BC0970A9750F51C
:1016E000CE0107960E94EE49633071058105910590
:1016F0000CF04BC001E010E00A151B050CF045C0D2
:1017000062E370E080E090E0AFDA0E940398C12CC1
:10171000D12C811152C08FEFC81AD80A85E1C816A2
:10172000D10499F16EE170E080E090E09DDA0E94D2
:101730000398EFCF612FCE0101960E94D74BBE01D7
:101740006F5F7F4FCE0107960E94C04ACE0101967F
:101750000E94A34B62E370E080E090E085DA0E9493
:10176000039800E010E08823D9F0682FCE0101969D
:101770000E94D74BBE016F5F7F4FCE0107960E943C
:10178000BA4ACE0101960E94A34BBE01695F7F4F0A
:10179000C7010E94EF4BCE0107960E94A34B20C0C9
:1017A0000F5F1F4F0F31110581F36EE170E080E094
:1017B00090E05ADA0E940398D6CF682FCE010196A6
:1017C0000E94D74BBE016F5F7F4FCE0107960E94EC
:1017D000BA4ACE0101960E94A34B0F5F1F4F8CCFD8
:1017E000C7012C960FB6F894DEBF0FBECDBFDF91B8
:1017F000CF911F910F91FF90EF90DF90CF90BF900E
:10180000AF9008954F925F926F927F928F929F92C6
:10181000AF92BF92CF92DF92EF92FF92CF93DF937E
:10182000CDB7DEB72C970FB6F894DEBF0FBECDBF95
:101830000E948D3E0E94D1952B013C010E94A397EE
:101840004B015C016091430270914402809145021A
:10185000909146020E94B4AE6B017C010E94D1952A
:101860000E94B4AEA70196010E9404B121E03EEDB2
:1018700042E45EE30E94ACB29B01AC0160E070E028
:1018800080E89FE30E943DB020E03AE24DE257E459
:101890000E9413AF6B017C01C301B2010E94B4AE80
:1018A00020E030E048EC52E40E9404B1AB01BC01FE
:1018B00022E0CE0101960E94A84BBE016F5F7F4FD0
:1018C00082E192E10E94C04ACE0101960E94A34BA0
:1018D00062E578E082E192E10E94AC4A62E172E165
:1018E00088E192E10E948E4B6EE478E0CE01019691
:1018F0000E94074C62E172E1CE0101960E94234BE7
:10190000BC0182E192E10E948E4BCE0101960E94C1
:10191000A34B6DE07AE08EE192E10E94794B21E0E9
:10192000B501A401CE0101960E94A84BBE016F5FD4
:101930007F4F8EE192E10E94BA4ACE0101960E9449
:10194000A34B6BE97BE08EE192E10E94AC4A21E07F
:10195000B701A601CE0101960E94A84BBE016F5FA0
:101960007F4FCE0107960E94FF4B67EF75E0CE01D7
:1019700007960E940C4BBC018EE192E10E94BA4A8C
:10198000CE0107960E94A34BCE0101960E94A34B65
:1019900062E172E1CE0101960E94FF4B68ED7BE0AF
:1019A000CE0101960E940C4B6EE172E10E94234B26
:1019B000BC018EE192E10E948E4BCE0101960E9405
:1019C000A34B21E0B501A401CE0101960E94A84BD2
:1019D000BE016F5F7F4F84E292E10E94C04ACE0158
:1019E00001960E94A34B64E272E1CE0101960E942F
:1019F000FF4B4AE050E060E070E0CE010196C4D2B7
:101A0000CE0101960E94A34B65E070E080E090E07B
:101A10002BD966E779E0CE0101960E94074CCE01F2
:101A20000196E6D0CE0101960E94A34B68E172E1D7
:101A3000CE0101960E94FF4B4AE050E06FEF7FEF2E
:101A4000CE01019659D0CE0101960E94A34B20E011
:101A5000B701A601CE0101960E94A84BBE016F5F9F
:101A60007F4FCE0107960E94FF4B67EF75E0CE01D6
:101A700007960E940C4BBC0184E292E10E948E4BBF
:101A8000CE0107960E94A34BCE0101960E94A34B64
:101A900064E272E1CE0101960E94FF4B4AE050E001
:101AA00064EF7FEFCE01019627D0CE0101960E9410
:101AB000A34B65E070E080E090E0D6D88091430CC5
:101AC000882329F068E572E080E090E0CDD82C967C
:101AD0000FB6F894DEBF0FBECDBFDF91CF91FF9060
:101AE000EF90DF90CF90BF90AF909F908F907F90BE
:101AF0006F905F904F9008958F929F92AF92BF9298
:101B0000EF92FF920F931F93CF93DF9320912E05B7
:101B1000222309F462C020912D05222309F45DC01F
:101B20008A01EB017C0177FF18C0C095D09561E078
:101B30008C2F0E94076AB7018FE193E10E94654CE8
:101B40006AEF73E18FE193E10E94734CF7018481A6
:101B500061E08C0F0E94076A31C0E2D980908F1338
:101B600090909013A0909113B090921324E6820E5F
:101B7000911CA11CB11C86169706A806B90668F52B
:101B800061E08C2F0E94076AB7018FE193E10E9408
:101B9000654C69EE73E18FE193E10E94734CF701AC
:101BA000848161E08C0F0E94076ABAD960938F1319
:101BB000709390138093911390939213B801110F27
:101BC000880B990BDF91CF911F910F91FF90EF90B0
:101BD000BF90AF909F908F9047C8DF91CF911F919A
:101BE0000F91FF90EF90BF90AF909F908F900895CE
:101BF000CF93DF9320912E052223A9F020912D056C
:101C0000222389F0EC016FED8FE193E10E945E4C9D
